:20000000F05B002045AF00009B2D00000B400000000000000000000000000000000000006E
:2000200000000000000000000000000067410000000000000000000067420000BF4F000061
:2000400050B2000050B2000050B2000050B2000050B2000050B2000050B2000050B2000090
:2000600050B20000E14F000050B2000050B2000050B2000050B2000050B2000050B2000042
:2000800050B2000050B2000050B2000050B2000050B2000050B2000050B2000050B2000050
:2000A00050B2000050B2000050B2000050B2000050B2000050B2000050B2000050B2000030
:2000C00048573031424C30313031000032313A30333A353900000000466562202034203255
:2000E0003032350000000000574B2D4B3836000000000000000000000000000000000000E1
:20010000FFFFFFFFFFFFFFFFFFFFFFFFFFFFFFFFFFFFFFFFFFFFFFFFFFFFFFFFFFFFFFFFFF
:20012000FFFFFFFFFFFFFFFFFFFFFFFFFFFFFFFFFFFFFFFFFFFFFFFFFFFFFFFFFFFFFFFFDF
:20014000FFFFFFFFFFFFFFFFFFFFFFFFFFFFFFFFFFFFFFFFFFFFFFFFFFFFFFFFFFFFFFFFBF
:20016000FFFFFFFFFFFFFFFFFFFFFFFFFFFFFFFFFFFFFFFFFFFFFFFFFFFFFFFFFFFFFFFF9F
:20018000FFFFFFFFFFFFFFFFFFFFFFFFFFFFFFFFFFFFFFFFFFFFFFFFFFFFFFFFFFFFFFFF7F
:2001A000FFFFFFFFFFFFFFFFFFFFFFFFFFFFFFFFFFFFFFFFFFFFFFFFFFFFFFFFFFFFFFFF5F
:2001C000FFFFFFFFFFFFFFFFFFFFFFFFFFFFFFFFFFFFFFFFFFFFFFFFFFFFFFFFFFFFFFFF3F
:2001E000FFFFFFFFFFFFFFFFFFFFFFFFFFFFFFFFFFFFFFFFFFFFFFFFFFFFFFFFFFFFFFFF1F
:20020000FFFFFFFFFFFFFFFFFFFFFFFFFFFFFFFFFFFFFFFFFFFFFFFFFFFFFFFFFFFFFFFFFE
:20022000FFFFFFFFFFFFFFFFFFFFFFFFFFFFFFFFFFFFFFFFFFFFFFFFFFFFFFFFFFFFFFFFDE
:20024000FFFFFFFFFFFFFFFFFFFFFFFFFFFFFFFFFFFFFFFFFFFFFFFFFFFFFFFFFFFFFFFFBE
:20026000FFFFFFFFFFFFFFFFFFFFFFFFFFFFFFFFFFFFFFFFFFFFFFFFFFFFFFFFFFFFFFFF9E
:20028000FFFFFFFFFFFFFFFFFFFFFFFFFFFFFFFFFFFFFFFFFFFFFFFFFFFFFFFFFFFFFFFF7E
:2002A000FFFFFFFFFFFFFFFFFFFFFFFFFFFFFFFFFFFFFFFFFFFFFFFFFFFFFFFFFFFFFFFF5E
:2002C000FFFFFFFFFFFFFFFFFFFFFFFFFFFFFFFFFFFFFFFFFFFFFFFFFFFFFFFFFFFFFFFF3E
:2002E000FFFFFFFFFFFFFFFFFFFFFFFFFFFFFFFFFFFFFFFFFFFFFFFFFFFFFFFFFFFFFFFF1E
:20030000FFFFFFFFFFFFFFFFFFFFFFFFFFFFFFFFFFFFFFFFFFFFFFFFFFFFFFFFFFFFFFFFFD
:20032000FFFFFFFFFFFFFFFFFFFFFFFFFFFFFFFFFFFFFFFFFFFFFFFFFFFFFFFFFFFFFFFFDD
:20034000FFFFFFFFFFFFFFFFFFFFFFFFFFFFFFFFFFFFFFFFFFFFFFFFFFFFFFFFFFFFFFFFBD
:20036000FFFFFFFFFFFFFFFFFFFFFFFFFFFFFFFFFFFFFFFFFFFFFFFFFFFFFFFFFFFFFFFF9D
:20038000FFFFFFFFFFFFFFFFFFFFFFFFFFFFFFFFFFFFFFFFFFFFFFFFFFFFFFFFFFFFFFFF7D
:2003A000FFFFFFFFFFFFFFFFFFFFFFFFFFFFFFFFFFFFFFFFFFFFFFFFFFFFFFFFFFFFFFFF5D
:2003C000FFFFFFFFFFFFFFFFFFFFFFFFFFFFFFFFFFFFFFFFFFFFFFFFFFFFFFFFFFFFFFFF3D
:2003E000FFFFFFFFFFFFFFFFFFFFFFFFFFFFFFFFFFFFFFFFFFFFFFFFFFFFFFFFFFFFFFFF1D
:2004000027C08FD2A0D34DDC000000000000FFFFBFFFFFFFFFFFFFFFFE88E6BE30A25B8E5D
:2004200000B5020093680120DB680340DBB2002B0AD093681B6A9B081840C0B2002803D0E9
:20044000D0690860012000E0002000BDF2B584B00200002001009468E66801239E430123AC
:200460000D00EDB21D403543E560049E3678002E51D0D169294CA14201D1010012E0D16986
:20048000274CA14201D219000CE0D169254CA14201D2022106E0D169234CA14201D2032141
:2004A00000E004210C00E4B2042C01D1002033E06C46617094680194019CE4680C25AC4343
:2004C0006D466D78AD000C262E4026430396039C019DEC606C4620709068C4681025AC4322
:2004E0006D462D782D011026354025430295029CC4601C009568EE680127BE432700FFB29A
:200500001F403743EF609068006A840818002040C0B20028F7D0012005B0F0BD00093D0023
:2005200001127A0001366E01015A620200B502009068006A43081800C007C00FC0B200281D
:2005400003D090690860012000E0002000BDF2B584B005000026A86801244169200008403C
:20056000C0B200286AD0A868016A20000840C0B2002863D0A8688069010920000840C0B21A
:20058000002802D0012806D00BE069462800FFF747FF060005E069462800FFF7C7FF0600E0
:2005A000FFE73000C0B2002801D1002048E02700A8684069000A8007800FC0B2002805D002
:2005C000022808D004D3032808D00AE0270008E00220070005E00420070002E008200700FC
:2005E000FFE7A868406940084006400EC0B2002802D18020029000E00290A8684069C00AEC
:200600004007400FC0B2002802D10820019000E00190A8684069810A20000840C0B2401C33
:2006200003900098029948430399484301997943490002F05AFB0499086026003000C0B28F
:2006400005B0F0BDFCB502000020040095686E6901239E4301232700FFB21F40374301971B
:20066000019E6E611E006F463E704E78002E02D0012E0FD01DE004009568AF691026B74371
:20068000BC462600F6B2360110273E4067463E43AE6111E01C009568AF691026B743BC460D
:2006A0002600F6B2360110273E4067463E43AE6102E004006D462C706C462478002C01D1C2
:2006C000002093E0CC68012C01D104000FE0CC68022C01D11C000AE0CC68042C01D10224CB
:2006E00005E0CC68082C01D1032400E0FF242500EDB2FF2D01D1002078E06D466C709568EB
:200700006E69834F3740BC466E4676783702C026B6003E4067463E436E614F88002F1CD0D3
:200720004D88812D19DA4D88802D01D1050000E04D8896680196019E7769FE26B743BC4601
:200740002E00F6B27700FE263E4067463E43019F7E610F69002F02D11AE0002046E00D69CD
:20076000092D15D20D69082D00D0086995686E69B04F3740BC460600F6B2F702E026B601C0
:200780003E4067463E436E618F68012F02D104E000202BE08868022813D18868401E95688C
:2007A0006E69A54F3740BC460600F6B2B6028027FF003E4067463E436E610F78002F02D1E5
:2007C00012E0002012E0180095686E690127BE430700FFB21F4037436F619068056A180020
:2007E0002840C0B20028F8D068460078F6BDF3B581B0070000242600009478690125C06968
:20080000010928000840C0B2002818D069463800FFF706FE06003000C0B200280FD078696B
:20082000C069000A4007400F85402900412905D2009802F05AFA0299086000E026003000A9
:20084000C0B2FEBDFEB5020000206B4618706B4658705369DE691024E443264010256F4636
:200860007F783F012F403743DF618E88012E01D103001EE08B88022B01D1012319E08B88BE
:20088000042B01D1022314E08B88082B01D103230FE08B88102B01D104230AE08B88202B82
:2008A00001D1052305E08B88402B01D1062300E007231E00F6B2072E17D06E46737056699E
:2008C0000196019EF669A54F3740BC466E4676783702E026F6003E4067463E430296029E5B
:2008E000019FFE6101266F463E700E78002E01D0012600E006005769F86904403000C0B2D6
:20090000000105402543FD6168460078FEBD0000FFFCFFFFF3B581B0070000242600009433
:20092000786901258069010928000840C0B2002818D069463800FFF773FD06003000C0B2D6
:2009400000280FD078698069000A4007400F85402900412905D2009802F0C7F902990860AA
:2009600000E026003000C0B2FEBDFEB5020000206B4618706B46587053699E691024E4436F
:20098000264010256F467F783F012F4037439F618E88012E01D103001EE08B88022B01D1BD
:2009A000012319E08B88042B01D1022314E08B88082B01D103230FE08B88102B01D1042379
:2009C0000AE08B88202B01D1052305E08B88402B01D1062300E007231E00F6B2072E17D08B
:2009E0006E46737056690196019EB6695B4F3740BC466E4676783702E026F6003E40674627
:200A00003E430296029E019FBE6101266F463E700E78002E01D0012600E006005769B86961
:200A200004403000C0B2000105402543BD6168460078FEBDFFC7FFFFFFFBFFFFF3B581B08E
:200A40000700002426000094786901254069010928000840C0B2002818D069463800FFF728
:200A600065FD06003000C0B200280FD078694069000A4007400F85402900412905D2009874
:200A800002F033F90299086000E026003000C0B2FEBDFEB5020000206B4618706B4658704B
:200AA00053695E691024E443264010256F467F783F012F4037435F618E88012E01D103000E
:200AC0001EE08B88022B01D1012319E08B88042B01D1022314E08B88082B01D103230FE08F
:200AE0008B88102B01D104230AE08B88202B01D1052305E08B88402B01D1062300E0072305
:200B00001E00F6B2072E17D06E46737056690196019E7669114F3740BC466E4676783702D4
:200B2000E026F6003E4067463E430296029E019F7E6101266F463E700E78002E01D0012620
:200B400000E006005769786904403000C0B20001054025437D6168460078FEBDFFF8FFFFC6
:200B6000F3B581B00700002426000094786901250069010928000840C0B2002818D069469C
:200B80003800FFF7D3FC06003000C0B200280FD078690069000A4007400F85402900412967
:200BA00005D2009802F0A1F80299086000E026003000C0B2FEBDFEB5020000206B461870C7
:200BC0006B46587053691E691024E443264010256F467F783F012F4037431F618E88012EC9
:200BE00001D103001EE08B88022B01D1012319E08B88042B01D1022314E08B88082B01D1AE
:200C000003230FE08B88102B01D104230AE08B88202B01D1052305E08B88402B01D10623D8
:200C200000E007231E00F6B2072E17D06E46737056690196019E3669A14F3740BC466E4680
:200C400076783702E026F6003E4067463E430296029E019F3E6101266F463E700E78002E10
:200C600001D0012600E006005769386904403000C0B20001054025433D6168460078FEBD22
:200C8000F3B581B0070000242600009478690125406A010928000840C0B2002818D069463A
:200CA0003800FFF754FC06003000C0B200280FD07869406A000A4007400F85402900412984
:200CC00005D2009802F011F80299086000E026003000C0B2FEBDFEB5020000206B46187036
:200CE0006B46587053695E6A1024E443264010256F467F783F012F4037435F628E88012E26
:200D000001D103001EE08B88022B01D1012319E08B88042B01D1022314E08B88082B01D18C
:200D200003230FE08B88102B01D104230AE08B88202B01D1052305E08B88402B01D10623B7
:200D400000E007231E00F6B2072E17D06E46737056690196019E766A594F3740BC466E4666
:200D600076783702E026F6003E4067463E430296029E019F7E6201266F463E700E78002EAE
:200D800001D0012600E006005769786A04403000C0B20001054025437D6268460078FEBD7F
:200DA000F3B581B0070000242600009478690125006A010928000840C0B2002818D0694659
:200DC0003800FFF7C4FB06003000C0B200280FD07869006A000A4007400F85402900412934
:200DE00005D2009801F081FF0299086000E026003000C0B2FEBDFEB5020000206B4618709F
:200E00006B46587053691E6A1024E443264010256F467F783F012F4037431F628E88012E84
:200E200001D103001EE08B88022B01D1012319E08B88042B01D1022314E08B88082B01D16B
:200E400003230FE08B88102B01D104230AE08B88202B01D1052305E08B88402B01D1062396
:200E600000E007231E00F6B2072E17D06E46737056690196019E366A114F3740BC466E46CD
:200E800076783702E026F6003E4067463E430296029E019F3E6201266F463E700E78002ECD
:200EA00001D0012600E006005769386A04403000C0B20001054025433D6268460078FEBDDE
:200EC000FFF8FFFF70B504000E00002560690068000E8007800FC0B2002805D002280FD0F4
:200EE00008D3032812D017E031002000FFF71EFB050011E031002000FFF792FA05000BE0FA
:200F000031002000FFF723FB050005E031002000FFF70CFB0500FFE72800C0B270BDF0B5DD
:200F200002004878012801D100230AE04878002801D1012305E04878022801D1022300E063
:200F4000FF231800C0B2FF2801D1002017E01C0050690668934D35402600F6B23704C0264E
:200F6000B6023E402E43066050690068000E8007800F1C00C0B2E4B2A042F5D10120F0BD85
:200F8000F8B504000E00002569462000FFF79AFF07003800C0B2002801D100200BE0E06811
:200FA00000680107090F0098C9B2491C01F09DFE30603800C0B2F2BD30B50200888800289D
:200FC00010D0888811280DDA8C88641ED36818680F25A8432500EDB22D072D0F05431D6098
:200FE000012000E0002030BDF8B504000E00002569462000FFF7C4FF07003800C0B200289E
:2010000001D100200CE060690068000A0107090F0098C9B2491C01F068FE30603800C0B28E
:20102000F2BD70B502008888002812D0888811280FDA8C88641E53691D685B482840250087
:20104000EDB22E02F0252D01354005431D60012000E0002070BDF8B504000F0000252E00E3
:201060002069C8214058000C8007800FC0B2002805D002280FD008D3032812D017E069463E
:201080002000FFF753FA060011E069462000FFF7C7F906000BE069462000FFF758FA060063
:2010A00005E069462000FFF741FA0600FFE73000C0B2002801D1002019E02069C8214058A0
:2010C00001090800C007C00FC0B200280CD02069C8214058000A0107090F0098C9B2491C46
:2010E00001F003FE386000E02E003000C0B2F2BDFCB502004878012801D100230AE04878CC
:20110000002801D1012305E04878022801D1022300E0FF231800C0B2FF2801D100203FE027
:20112000888800283BD08888112838DA684603701069C82405591B4C2C406D462D782D04D1
:20114000C026B6022E4026430196019CC82544518C88641E1569C826AE59134F3740BC4680
:201160002600F6B23702F02636013E4067463E43C827EE510F78002F01D0012400E0002491
:201180001569C82028581026B0432600F6B2360110273E400643C8202E50012000E00020B6
:2011A000F6BD0000FFFFFCFFFFF0FFFFF8B504000F006069406801090800C007C00FC0B24B
:2011C000002801D100209BE0002005000090606907264068000C3040C0B2002843D1606934
:2011E0004068C00C3040C0B200280BD0022815D00ED304281ED017D3062827D020D307285B
:201200002AD02FE069462000FFF725FF050066E069462000FFF704F9050060E069462000BB
:20122000FFF784F905005AE069462000FFF78FF9050054E069462000FFF7A2FE05004EE0DE
:2012400069462000FFF7D0FE050048E069462000FFF7CDFA050042E069462000FFF7EEFB6D
:2012600005003CE03BE060694068000C3040C0B201280AD033D3032813D00CD305281CD0C4
:2012800015D3072825D01ED329E069462000FFF7F7FC050023E06946200000F038FA050092
:2012A0001DE06946200000F00BFA050017E06946200000F0DEF9050011E06946200000F026
:2012C00067FD05000BE069462000FFF72FF9050005E069462000FFF729F90500FFE72800E9
:2012E000C0B201280AD160694068000A064031000098C9B2491C01F0F8FC38602800C0B2F7
:20130000F2BDF2B582B0010001206A461070002002004B695C681025AC431500EDB22D0153
:201320001026354025435D60029C6478002C40D0012C5DD0022C7AD0032C00D1D4E0052C70
:2013400000D1F0E0072C00D10CE10A2C00D18DE00B2C00D1A9E00C2C0CD00F2C00D12BE1CA
:20136000102C00D11AE1112C00D109E11A2C00D130E13DE102004B695D68B94C2C40150026
:20138000EDB22D04E026F6022E4026430196019C5C6004004D696E68B24F3740BC46260088
:2013A000F6B2F704E026B6033E4067463E436E6021E102004B695D68A94C2C401500EDB2BF
:2013C0002D04E026F6022E4026430196019C5C6001244D696E68A34F3740BC462600F6B22D
:2013E000F704E026B6033E4067463E436E6002E102004B695D689A4C2C401500EDB22D0424
:20140000E026F6022E4026430196019C5C6002244D696E68934F3740BC462600F6B2F70431
:20142000E026B6033E4067463E436E60E3E002004B695D688A4C2C401500EDB22D04E02608
:20144000F6022E4026430196019C5C6003244D696E68844F3740BC462600F6B2F704E026FF
:20146000B6033E4067463E436E60C4E002004B695D687B4C2C401500EDB22D04E026F60204
:201480002E4026430196019C5C6004244D696E68744F3740BC462600F6B2F704E026B6030D
:2014A0003E4067463E436E60A5E002004B695D686B4C2C401500EDB22D04E026F6022E403E
:2014C00026430196019C5C6005244D696E68654F3740BC462600F6B2F704E026B6033E40CB
:2014E00067463E436E6086E002004B695D685C4C2C401500EDB22D04E026F6022E40264341
:201500000196019C5C6006244D696E68554F3740BC462600F6B2F704E026B6033E40674655
:201520003E436E6067E002004B695D684C4C2C401500EDB22D04E026F6022E402643019645
:20154000019C5C6007244D696E68464F3740BC462600F6B2F704E026B6033E4067463E4339
:201560006E6048E001224B695D683D4C2C401500EDB22E04E025ED02354025435D603AE056
:2015800002224B695D68364C2C401500EDB22E04E025ED02354025435D602CE003224B6967
:2015A0005D682F4C2C401500EDB22E04E025ED02354025435D601EE004224B695D68284CFA
:2015C0002C401500EDB22E04E025ED02354025435D6010E005224B695D68214C2C401500AD
:2015E000EDB22E04E025ED02354025435D6002E002006B461A706A461278002A1AD0029A83
:201600009288002A13D0029A9288092A0FDA029A9288521E4B695D687F4C2C401500EDB247
:201620002E02E025ED00354025435D6002E002006B461A70029A1278002A01D0012200E0AB
:2016400002004B6958681024A0431400E4B2240110252C4004435C6068460078FEBD0000A9
:20166000FFFFF8FFFFFFC7FF0200106A08600120704700B502005068806C03091800C007AF
:20168000C00FC0B2002804D0FA2080000860012000E0002000BD70B502000878002801D08D
:2016A000012400E000245368986C1025A8432500EDB22D011026354005439D64012070BDEE
:2016C00000B502005068406C03091800C007C00FC0B2002804D0FA20C0010860012000E083
:2016E000002000BD70B502000878002801D0012400E000245368586C1025A8432500EDB2E1
:201700002D011026354005435D64012070BD0200FA20400208600120704770B504000E00C4
:20172000002561680120496809090140C9B2002901D100201AE061684968090C0140C9B2BB
:20174000002905D131002000FFF71AFC05000BE061684968090C0840C0B2012804D13100C5
:20176000200000F02FF905002800C0B270BDF2B582B0010000206A46107005004C686668B4
:201780001022D243164010232F00FFB23F011F4037436760029E76780A2E11D16C4660708F
:2017A0004C6866681D4D35406E467678360480277F023E402E43666001256F463D7018E08F
:2017C000029C6478182C14D1012425004E680196019E7668114F3740BC462E00F6B2360469
:2017E00080277F023E4067463E43019F7E606F463C70029C2478002C01D0012400E00400F6
:201800004D68686802402000C0B20001034013436B6068460078FEBDFFF8FFFFFFFFFEFF39
:2018200070B504000E0000256068806801090800C007C00FC0B2002804D031002000FFF73F
:20184000D3FB05002800C0B270BD70B502000878002801D0012400E0002453689868102535
:20186000A8432500EDB22D011026354005439D60012070BD70B504000E0000256068C06801
:2018800001090800C007C00FC0B2002804D031002000FFF7A9FB05002800C0B270BD70B556
:2018A00002000878002801D0012400E000245368D8681025A8432500EDB22D0110263540CC
:2018C0000543DD60012070BD70B504000E0000256068006901090800C007C00FC0B2002866
:2018E00004D031002000FFF77FFB05002800C0B270BD70B502000878002801D0012400E0E2
:201900000024536818691025A8432500EDB22D011026354005431D61012070BD70B504006D
:201920000E0000256068406901090800C007C00FC0B2002804D031002000FFF755FB050051
:201940002800C0B270BD70B502000878002801D0012400E00024536858691025A843250036
:20196000EDB22D011026354005435D61012070BD70B504000E00002560688069010908007C
:20198000C007C00FC0B2002804D031002000FFF72BFB05002800C0B270BD70B50200087863
:2019A000002801D0012400E00024536898691025A8432500EDB22D011026354005439D6146
:2019C000012070BDF8B505000F000020040000906868C06901090800C007C00FC0B2002809
:2019E00001D1002054E068680726C069000C3040C0B200280BD0022815D00ED304281ED0A0
:201A000017D3062827D020D307282AD02FE069462800FFF713F8040029E069462800FEF7DB
:201A2000E6FE040023E069462800FFF729F904001DE069462800FFF76AFE040017E06946EC
:201A40002800FFF716FE040011E069462800FFF737FE04000BE069462800FFF705FE04009A
:201A600005E069462800FEF7E9FF0400FFE72000C0B200280AD06868C069000A06403100D5
:201A8000C9B2491C009801F030F938602000C0B2F2BDF3B50100012002006B461A700022B2
:201AA00014004D68EE6910239E4310232700FFB23F011F403743EF61019E7678032E1CD0D4
:201AC000052E0AD0072E28D00E2E66D00F2E44D0102E52D0112E30D06FE014004D68EE69FB
:201AE000AA4F3740BC462600F6B23704E026F6023E4067463E43EE6162E004004D68EE6920
:201B0000A24F3740BC462600F6B23704E026F6023E4067463E43EE6152E002244D68EE69F5
:201B20009A4F3740BC462600F6B23704E026F6023E4067463E43EE6142E003244D68EE69EC
:201B4000924F3740BC462600F6B23704E026F6023E4067463E43EE6132E004244D68EE69E3
:201B60008A4F3740BC462600F6B23704E026F6023E4067463E43EE6122E005244D68EE69DA
:201B8000824F3740BC462600F6B23704E026F6023E4067463E43EE6112E006244D68EE69D1
:201BA0007A4F3740BC462600F6B23704E026F6023E4067463E43EE6102E014006D462C709C
:201BC000019CA488002C15D0019CA488092C11DA019CA488641E4D68EE69C04F3740BC4663
:201BE0002600F6B23702E026F6003E4067463E43EE6102E014006D462C70019C2478002C3D
:201C000001D00200FFE74C68E0691025A8431500EDB22D012B400343E36168460078F6BD3E
:201C200070B504000E00002561680120096A09090140C9B2002901D1002026E06168096AC0
:201C4000090C8907890FC9B2002905D002290FD008D3032912D016E031002000FEF7EEFEB3
:201C6000050010E031002000FFF70AF805000AE031002000FEF7BBFD050004E0FA214902EA
:201C800031600500FFE72800C0B270BDF2B582B00100012002006B461A7000226B465A702C
:201CA0004D682E6A1023DB431E4010246F467F783F01274037432F62029E7678032E2AD0DD
:201CC000052E04D0072E13D0112E37D049E06D466A704D682E6AC94F3740BC466E46767869
:201CE0003704C026B6023E4067463E432E623AE005004E680196019E366AC04F3740BC469C
:201D00002E00F6B23704C026B6023E4067463E43019F3E6227E002254E680196019E366A6E
:201D2000B64F3740BC462E00F6B23704C026B6023E4067463E43019F3E6214E003254E68B8
:201D40000196019E366AAD4F3740BC462E00F6B23704C026B6023E4067463E43019F3E629D
:201D600001E06D462A70029D2D78002D01D00200FFE74D68286A03401000C0B200010440BA
:201D80001C432C6268460078FEBD0000FFFFF8FF70B504000E0000256068806A0109080060
:201DA000C007C00FC0B2002801D1002027E06068806A000C8007800FC0B2002805D002288D
:201DC0000FD008D3032812D017E031002000FFF777FC050011E031002000FFF745FC050008
:201DE0000BE031002000FFF744FC050005E031002000FFF73EFC0500FFE72800C0B270BD54
:201E0000F2B582B0010000206A46107005004C68A66A1022D243164010232F00FFB23F01DF
:201E20001F403743A762029E7678102E11D16C4660704C68A66A714D35406E4676783704BC
:201E4000C026B6023E402E43A66201256F463D7031E0029C64780E2C15D1012425004E68BA
:201E60000196019EB66A654F3740BC462E00F6B23704C026B6023E4067463E43019FBE62C4
:201E80006F463C7017E0029C64780F2C13D102244D68AE6A594F3740BC462600F6B2370434
:201EA000C026B6023E4067463E430196019EAE6201266F463E70029C2478002C01D00124AC
:201EC00000E004004D68A86A02402000C0B2000103401343AB6268460078FEBDFFF8FFFF06
:201EE00070B504000E00002561680120096B090C0140C9B2002905D131002000FFF774F8A5
:201F000005000BE06168096B090C0840C0B2012804D131002000FFF7FAFB05002800C0B2EC
:201F200070BDF0B50200002318004C780B2C0CD15468266B9D4D35401E00F6B23704802667
:201F4000760237402F4327630FE04B78112B0CD101235468266B954D35401E00F6B2370402
:201F60008026760237402F432763C0B2F0BD70B504000E00002561680120496B090C014061
:201F8000C9B2002905D131002000FFF72DF805000BE06168496B090C0840C0B2012804D121
:201FA00031002000FFF7B3FB05002800C0B270BDF0B50200002318004C780B2C0CD15468EA
:201FC000666B7A4D35401E00F6B237048026760237402F4367630FE04B78112B0CD1012333
:201FE0005468666B714D35401E00F6B237048026760237402F436763C0B2F0BDFFFFFCFF37
:2020000070B504000E00002561680120896B090C0140C9B2002905D131002000FEF7E4FF8D
:2020200005000BE06168896B090C0840C0B2012804D131002000FFF76AFB05002800C0B2DB
:2020400070BDF0B50200002318004C780B2C0CD15468A66B554D35401E00F6B2370480260E
:20206000760237402F43A7630FE04B78112B0CD101235468A66B4D4D35401E00F6B2370429
:202080008026760237402F43A763C0B2F0BD70B504000E00002561680120C96B090C014040
:2020A000C9B2002905D131002000FEF79DFF05000BE06168C96B090C0840C0B2012804D10A
:2020C00031002000FFF723FB05002800C0B270BDF0B50200002318004C780B2C0CD1546859
:2020E000E66B324D35401E00F6B237048026760237402F43E7630FE04B78112B0CD101235A
:202100005468E66B294D35401E00F6B237048026760237402F43E763C0B2F0BD70B504002D
:202120000E00002561680120096C090C0140C9B2002905D131002000FEF756FF05000BE0B2
:202140006168096C090C0840C0B2012804D131002000FFF7DCFA05002800C0B270BDF0B5E6
:202160000200002318004C780B2C0CD15468266C0E4D35401E00F6B2370480267602374096
:202180002F4327640FE04B78112B0CD101235468266C064D35401E00F6B23704802676021E
:2021A00037402F432764C0B2F0BD0000FFFFFEFF70B504000E00002521680120C968090948
:2021C0000140C9B2002905D131002000FEF70CFF05000AE02168C96809090140C9B2012952
:2021E00003D1FA214902316005002800C0B270BDF0B50200002318004C780B2C0DD1146811
:20220000E5681026B5431E00F6B2360110273E402E43E6600125280012E04B78112B0FD1BB
:2022200001231C001568EF681026B743BC462600F6B2360110273E4067463E43EE6018000A
:20224000C0B2F0BD38B505000C002869006801090800C007C00FC0B2002801D1002003E051
:2022600021002800FEF78CFE32BD70B502000878002801D0012400E00024136918681025AD
:20228000A8432500EDB22D011026354005431D60012070BD38B505000C0028694068010962
:2022A0000800C007C00FC0B2002801D1002003E021002800FEF798FE32BD70B502000878A7
:2022C000002801D0012400E00024136958681025A8432500EDB22D011026354005435D60DE
:2022E000012070BD38B505000C002869006901090800C007C00FC0B2002801D1002003E081
:2023000021002800FEF770FE32BD70B502000878002801D0012400E0002413691869102527
:20232000A8432500EDB22D011026354005431D61012070BD38B505000C00286940690109BF
:202340000800C007C00FC0B2002801D1002003E021002800FEF748FE32BD70B50200087856
:20236000002801D0012400E00024136958691025A8432500EDB22D011026354005435D613B
:20238000012070BD38B505000C002869806901090800C007C00FC0B2002801D1002003E060
:2023A00021002800FEF7ECFD32BD70B502000878002801D0012400E000241369986910258C
:2023C000A8432500EDB22D011026354005439D61012070BD38B505000C002869C06901091F
:2023E0000800C007C00FC0B2002801D1002003E021002800FEF7F8FD32BD70B50200087807
:20240000002801D0012400E000241369D8691025A8432500EDB22D01102635400543DD619A
:20242000012070BDF2B582B0060030690124006A010920000840C0B2002801D1002037E032
:202440002000694608710027009730690325006A000C2840C0B2002805D002280FD008D384
:20246000032812D017E069463000FEF75FF8070011E069463000FDF7D3FF07000BE06946EF
:202480003000FEF764F8070005E069463000FEF74DF80700FFE73069006A000A0540AC408B
:2024A0000098210000F021FC029908603800C0B2FEBDFEB5020000206B4618706B46587067
:2024C00013691E6A1024E443264010256F467F783F012F4037431F624E78012E01D10300E2
:2024E0000AE04B78002B01D1012305E04B78022B01D1022300E0FF231E00F6B2FF2E17D066
:202500006E46737016690196019E366A844F3740BC466E4676783704C026B6023E406746DD
:202520003E430296029E019F3E6201266F463E706E463678002E36D08E88012E01D1060065
:202540000FE08E88022E01D101260AE08E88042E01D1022605E08E88082E01D1032600E015
:20256000FF266F467E706E467678FF2E19D06E4676786F46BE7016690296029E376A694E47
:202580003E400196019FBC466E46B6783702C026B6003E4067463E430196019E029F3E62AA
:2025A00001E06E4630700E78002E01D0012600E006001769386A04403000C0B20001054006
:2025C00025433D6268460078FEBD38B505000C002869806A01090800C007C00FC0B2002858
:2025E00001D1002003E021002800FEF7FDFC32BD70B502000878002801D0012400E0002417
:202600001369986A1025A8432500EDB22D011026354005439D62012070BD70B505000C00B4
:2026200028690126006B00093040C0B2002801D1002023E02869006B000C8007800FC0B2DF
:20264000002805D002280DD007D303280FD013E021002800FEF7F2F90FE021002800FEF749
:20266000C6F80AE021002800FEF70AFB05E021002800FEF7E3F900E00020C0B270BDFEB51E
:20268000020000206B4618706B46587013691E6B1024E443264010256F467F783F012F4010
:2026A00037431F634E78052E01D103000AE04B78032B01D1012305E04B78072B01D10223AE
:2026C00000E0FF231E00F6B2FF2E17D06E46737016690196019E366B114F3740BC466E46A4
:2026E00076783704C026B6023E4067463E430296029E019F3E6301266F463E700E78002EB0
:2027000001D0012600E006001769386B04403000C0B20001054025433D6368460078FEBDA3
:20272000FFFFFCFFFFFCFFFF0200506A0860012070470200906A0860012070470200D06A33
:2027400008600120704770B505000C0001262869A0214058000C4007400FC0B200280BD0DB
:20276000022813D00DD304281AD014D3062821D01BD307281ED022E021002800FFF7D4FF31
:202780001EE021002800FFF7D4FF19E021002800FFF7D4FF14E021002800FEF7E1F90FE023
:2027A00021002800FEF7B6F80AE021002800FEF7F7FA05E021002800FEF7D2F900E0002026
:2027C000C0B270BDF0B50200012318004C78042C49D0062C37D0082C55D02A2C04D02B2C57
:2027E00012D02C2C1FD05EE000231469A0256659AD4D35401E00F6B23704E026F6023E4062
:202800002E43A025665150E01469A0256659A64D35401E00F6B23704E026F6023E402E4344
:20282000A025665141E002231469A02566599E4D35401E00F6B23704E026F6023E402E4387
:20284000A025665131E003231469A0256659964D35401E00F6B23704E026F6023E402E437E
:20286000A025665121E004231469A02566598E4D35401E00F6B23704E026F6023E402E4375
:20288000A025665111E005231469A0256659864D35401E00F6B23704E026F6023E402E436C
:2028A000A025665101E000231800C0B2F0BD70B505000C0001262869A4214058000C4007C3
:2028C000400FC0B200280BD0022813D00DD304281AD014D3062821D01BD307281ED022E01E
:2028E00021002800FFF720FF1EE021002800FFF720FF19E021002800FFF720FF14E02100B2
:202900002800FEF72DF90FE021002800FEF702F80AE021002800FEF743FA05E021002800BA
:20292000FEF71EF900E00020C0B270BDF0B50200012318004C78042C49D0062C37D0082C8F
:2029400055D02A2C04D02B2C12D02C2C1FD05EE000231469A4256659534D35401E00F6B267
:202960003704E026F6023E402E43A425665150E01469A42566594C4D35401E00F6B237046B
:20298000E026F6023E402E43A425665141E002231469A4256659444D35401E00F6B2370478
:2029A000E026F6023E402E43A425665131E003231469A42566593C4D35401E00F6B237046F
:2029C000E026F6023E402E43A425665121E004231469A4256659344D35401E00F6B2370466
:2029E000E026F6023E402E43A425665111E005231469A42566592C4D35401E00F6B237045D
:202A0000E026F6023E402E43A425665101E000231800C0B2F0BD70B505000C0001200600B1
:202A20002969C0228958090C0840C0B2002802D0012805D009E021002800FEF741FE05E02F
:202A400021002800FEF710FE00E00020C0B270BDF0B50200012318004C780E2C11D0102C8D
:202A60001ED100231469C02566598E4D35401E00F6B2360480277F023E402E43C025665120
:202A800010E01469C0256659864D35401E00F6B2360480277F023E402E43C025665101E049
:202AA00000231800C0B2F0BDFFFFF8FF70B505000C00012006002969C4228958090C0840B4
:202AC000C0B2002802D0012805D009E021002800FEF7F6FD05E021002800FEF7C5FD00E0AD
:202AE0000020C0B270BDF0B50200012318004C780E2C11D0102C1ED100231469C4256659E2
:202B0000684D35401E00F6B2360480277F023E402E43C425665110E01469C4256659614D11
:202B200035401E00F6B2360480277F023E402E43C425665101E000231800C0B2F0BD38B541
:202B400005000C002869CC21405801090800C007C00FC0B2002801D1002003E021002800EE
:202B6000FEF70EFA32BD70B502000878002801D0012300E000231469CC2020581025A843A1
:202B80001D00EDB22D01102635400543CC202550012070BDFEB50899099A0A9B0B9C009DC9
:202BA0000560019D4560029D8560C16002614361256885616568C561A568056200252E0094
:202BC0002E00F6B2032E0BD22E00F6B2B600A619F6682F00FFB2BF00C7197E626D1CEFE7AA
:202BE000F7BDF8B506000C0017002000C0B2322801DB002011E000252B4A2000C0B2C00086
:202C00001058002807D0390030002300DBB2DB00D258904705002800C0B2F2BDF4B588B029
:202C200004000F003800C0B2322801DB002037E000252E001C4A3800C0B2C0001018406877
:202C400000282BD01948079060680690079806998023C85016480590A06804900598049939
:202C600008661448039020680290039802998023C850089920003B00DBB2DB00D2185268E4
:202C800090470600019560680199802281500095A168009A0A6622688023D5503000C0B250
:202CA00009B0F0BDFFFFFEFF10A6000052455355202096194B4D4352F446002804D44942DD
:202CC00000F013F8404260474042002905D45FD000F00BF8404249426047494200F005F8FE
:202CE0004942604703460B43E6D40022030A8B420BD203098B4219D243088B422ED2411A41
:202D000000D20146524110467047FF2209023FD012068B4205D3121209028B4201D312120E
:202D2000090203098B4219D300E0090AC3098B4201D3CB01C01A524183098B4201D38B0171
:202D4000C01A524143098B4201D34B01C01A524103098B4201D30B01C01A5241C3088B42A2
:202D600001D3CB00C01A524183088B4201D38B00C01A524143088B4201D34B00C01A52417F
:202D8000884200D3401A5241CFD201461046704708B500F001F808BD7047FEE700B50100F7
:202DA00000200A00D2B2002A05D0022A09D005D3032A09D00AE01022100007E01822100026
:202DC00004E02822100001E048221000C0B200BDF8B505000C00286806008036002768464C
:202DE00007703800C0B2FFF7D9FF0100C9B289080800C0B2220092B2504380003018F2BDED
:202E000000B5010000200A00D2B2002A082A0ED9093A0ED0521E0FD0521E10D0521E11D0FA
:202E2000521E12D0521E13D0521E14D016E0080014E00C22100011E0102210000EE0142212
:202E400010000BE01822100008E02022100005E03022100002E040221000FFE7C0B200BD43
:202E6000F8B505000C0000206946487069460870210089B22800FFF7ABFF06003068000C18
:202E800007073F0F3800C0B2FFF7BAFFC0B2F2BD70B500231400E4B2002C0CD00468C02511
:202EA000ED03254305604468640F6407CD00ED08254345600BE00468BC4D25400560446826
:202EC000BB4E26408C04BB4D25403543456070BD10B40268B84B1340036002680B00DBB253
:202EE0001B04F02424031C401443046010BC704700B502685200520802600268AF4B1340FA
:202F000003600A00D2B2002A09D0026880231B061343036002688023DB051343036000BD73
:202F200000B50A00D2B2002A06D10268A44B13400360026802600CE00A00D2B2012A08D1F4
:202F400002689F4B1340036002688023DB041343036000BD30B50268803200231D001C00A8
:202F6000057EED01AC4205D2A500551929000B60641CF5E730BDF8B4924982688023D150F6
:202F800001234468256D2026B5431E00F6B2760120273E402E430096009D2565002586684E
:202FA0008027F551F1BC7047F8B4864982688023D15001234468256D1026B5431E00F6B241
:202FC000360110273E402E430096009D2565002586688027F551F1BC7047F2B40599069C8D
:202FE000079D089E37780776009F076042608360C16004614561F1BC704730B50022110028
:203000008260026142618261C260C26142628262C2620262012303701300C370130003712C
:203020000023DB4343638363C36303641400442544551400452544551400C8254455082443
:203040004625445514002100C9B2202906DA2100C9B2890041188B64641CF4E71100417009
:203060001100817011003023C1541100C923C1541100CA23C1541100CB23C1541100D52393
:20308000C1541100D423C1541100D623C1541100D723C1541100CC23C154D021425030BD3A
:2030A000F0B50024210002681368444D1D400B00DBB29B078026F60533402B4313600568B7
:2030C0002E68414F3740BC462600F6B2360780277F053E4067463E432E60016809680A0EEF
:2030E0001100C907C90FC9B20029F6D1F0BDF8B50400206801250068000D2840C0B2002829
:2031000014D0002021680A68520052080300DBB2DB0713430B6020680068000D2840C0B2FA
:20312000002803D02000FFF73FFFF4E7280021680B68264A1A400300DBB25B068026B60426
:20314000334013430B6020680068400E2840C0B20028F8D16846057020680168174A0A4073
:203160006946097889078023DB051940114301602A0023681E68144F3740BC461600F6B229
:20318000360780277F053E4067463E431E6020680068000E2840C0B20028F8D020680068E5
:2031A000C00E2840C0B20028F1D0F1BDFFFF9FFFFFFF03E00000FC1FFFFFF0FFFFFFFFBF8F
:2031C000FFFFFFF052455355FFFFFFEFFFFFFFFDF8B594B007000C0016003100C9B289B2DC
:2031E0003800FFF7F5FD0500227A61682800FFF74FFEA17A2800FFF76BFEE17A2800FFF7BF
:2032000077FE617A2800FFF78BFE207B002805D06846067101A9380000F009FD607A01281F
:203220000AD1206969460E7039686A46127892008A1888231B01D05015B0F0BDF0B58DB0B3
:2032400005000E000020694648700020694608702800FFF790FE012029680A685200520811
:203260000300DBB2DB0713430B6028680068010D0800C007C00FC0B20028F6D030786946C0
:2032800048712868029002984068CE4901406846407940038022920110400843059005980D
:2032A000029948602800FFF722FF0120694608712F683968C448084069460979C905802216
:2032C00012041140014304910498386001206946C8702C68616BBD4808406946C9780907C5
:2032E00080225205114001430391039860632800FFF730FE3020305CFFF750FD694688703C
:2033000068468078002809D08020800069468978FFF7EBFC297E484369464870684640785A
:203320006946087128680690069800687F218843694609794906490E01430C910C980699D3
:20334000086001206946C870286805900598006D400040086946C978C90701430B910B9803
:2033600005990865CE48B16809186A46D1812968049104990A6DCB4911406A46D2895205EF
:20338000C94B13400B430A930A99049A1165F16809186A46918129680B6DC44A1A406B46C6
:2033A0009B891B04F82464031C4014430994099A0A65326912186B465A812A68146DBC4B7A
:2033C00023406C466489A702FC2424023C401C430894089B136573691B186C4623812B6872
:2033E0001C6DB44F2740BC466C4624896701F824A4003C4067463C430794079C1C65B469CD
:2034000020186C46E0802868046D1F27BC436F46FF88FF06FF0E27430765F478002C6ED022
:2034200001206946887128680268A34911406A469279520780239B051A400A430692069957
:20344000016031796A46517129680B68CB4A1A406B465B79DB0380242402234013430593FE
:20346000059A0A60326C04922A680392049A039B9A644422B25C6B461A712A681468C04BE5
:2034800023406C4624792702C024A4003C401C430294029B13604523F35C6C46E3702B68F9
:2034A0005C6BB84F2740BC466C46E4782706F02424053C4067463C435C63C827F75D012F83
:2034C0003BD1002069460870684600784621715C884232D26846007880003018806C6946E8
:2034E00009782A680B00DBB29B00D3188824240118516B461B785B1C6C462370E4E7002076
:2035000029680B686C4A1A400300DBB25B078024A405234013430193019A0A6000222B6851
:203520001C68964F2740BC461400E4B2E40380273F023C4067463C431C60706B039028681E
:2035400003990161B16B02912968029A4A61F26B01922A68019B9361C823F35C6C46E37095
:203560002B681C68BC4F2740BC466C46E478240480277F023C4067463C431C60C927F75DFA
:20358000002F25D0002029680B68B44A1A400300DBB25B048024A402234013430193019A6A
:2035A0000A6001222B685C68AD4F2740BC461400E4B2240380277F013C4067463C435C6066
:2035C00024E000BFFFDFFFFFFFFF7FFFFFFFFFEF012029680B68A14A1A400300DBB25B048B
:2035E0008024A402234013430193019A0A6000222B685C689A4F2740BC461400E4B2240393
:2036000080277F013C4067463C435C60D420305C002853D0012001006A46917129680B687C
:20362000904A1A406B469B799B058024E403234013430593059A0A6002006B465A712A68FC
:203640001468894B23406C466479A4068027FF043C401C430494049B136003006C46237106
:203660002B681C68814F2740BC466C462479A4048027FF023C4067463C430394039C1C6001
:2036800004006F46FC706C690294029CA46C0127BC436F46FF7838402043029CA06453E0E9
:2036A000FFFF0000FFFF1F800000E07FFFFFE0FFFF03FFFF1FFCFFFFFFFFFFDF002001001D
:2036C0006A46517129680B68664A1A406B465B799B058024E403234013430593059A0A6060
:2036E00002006B461A712A6814685F4B23406C462479A4068027FF043C401C430494049BBC
:20370000136003006C46E3702B681C68574F2740BC466C46E478A4048027FF023C40674681
:203720003C430394039C1C606C690294029CA76C0124A743BC460700FFB23C00E407E40F59
:2037400067463C43029FBC64D520305C6946087128680268424911406A461279120380230A
:203760005B011A400A43049204990160D621715C6A46D17029684B68004A05E0FF7FFFFF0E
:20378000FFFCFFFFFFFFFFF01A406B46DB78DB0380242402234013430393039A4A60D722AE
:2037A000B25C2B685C68324F2740BC461400E4B2A4038027FF013C4067463C430294029CE6
:2037C0005C6000273800CC21715CC0B288422DD20020D02171583A00D2B214235A438C5A87
:2037E000220092B2D02030583900C9B214235943435AD020305884463900C9B21420414319
:20380000604640184088181882420DDA2200D2B2D02030583900C9B21423594341182800E1
:20382000FFF7D6FC641CDBE77F1CCBE7280000F082F92800FFF734FC002029680B680D4AD5
:203840001A400300DBB2DC0580231B041C4014430C600DB0F0BD0000FFFFFEFFFFFFFDFF5D
:20386000FFEFFFFFFFFFBFFFFFFFFFFBFFFFFBFFFFBFFFFFFFFF7FFF38B504000D002978D9
:2038800089B22000FFF7A4FA0168C02212050A43026031BDF1B50C00217889B20098FFF726
:2038A00097FA05000835217889B20098FFF7D8FA00210B000A001300DBB2834238D2032336
:2038C0001E00324209D129602B681600F6B2A619367A36061E432E6028E01600F6B21E40E4
:2038E000012E08D12B681600F6B2A619367A36041E432E601AE01600F6B21E40022E08D1B8
:203900002B681600F6B2A619367A36021E432E600CE01600F6B23340032B07D12B681600F4
:20392000F6B2A619367A1E432E602D1D521CC2E7F1BDF8B506000C00217889B23000FFF7B9
:2039400047FA05002868000C0007000FFFF758FA482160542868400D0100C907C90F6846D6
:203960000170281D69460978002904D00168C900C908616004E00168890C4905490D616059
:20398000051D217889B23000FFF76AFA00210A000A000300D2B2DBB29A422AD2032213004E
:2039A000194206D12A68120E0B00DBB2E3181A721DE00B00DBB21340012B06D12A68120C69
:2039C0000B00DBB2E3181A7211E00B00DBB21A40022A06D12A68120A0B00DBB2E3181A7215
:2039E00005E02A680B00DBB2E3181A722D1D491CCEE732689268F1BDF0B500252E000A7811
:203A0000D206D20E0124230093400F78402F12DB1C0002260568002E0AD0022E04D005D35B
:203A2000032E07D12C6705E06C6703E0EC6201E02C63FFE725E00E78202E11DB1D0006685B
:203A4000002C0AD0022C04D005D3032C07D1356705E0756703E0F56201E03563FFE710E099
:203A60001C000668002D0AD0022D04D005D3032D07D1346705E0746703E0F46201E03463C6
:203A8000FFE7F0BDF0B50300002215000878C406E40E01200600A6400F78402F16DB022062
:203AA0001D6800280DD0022805D007D303280BD12F6F3A0008E06F6F3A0005E0EF6A3A004C
:203AC00002E02F6B3A00FFE732402EE00D78202D15DB1D6800280DD0022805D007D303287A
:203AE0000BD12F6F3A0008E06F6F3A0005E0EF6A3A0002E02F6B3A00FFE7324015E0100087
:203B00001D6800280DD0022805D007D303280BD12F6F3A0008E06F6F3A0005E0EF6A3A00EB
:203B200002E02F6B3A00FFE73240002A01D0012000E00020F0BDF0B5017E032937D1002135
:203B4000C9430D0002270668002F0AD0022F04D005D3032F07D1356705E0756703E0F5622E
:203B600001E03563FFE70A0001230468002B0AD0022B04D005D3032B07D1226705E0626731
:203B800003E0E26201E02263FFE700260568002E0AD0022E04D005D3032E07D1296705E0BD
:203BA000696703E0E96201E02963FFE73EE0017E022925D10021C9430A0001250368002D01
:203BC0000AD0022D04D005D3032D07D11A6705E05A6703E0DA6201E01A63FFE7002604680C
:203BE000002E0AD0022E04D005D3032E07D1216705E0616703E0E16201E02163FFE715E03D
:203C0000017E012912D10021C94300230268002B0AD0022B04D005D3032B07D1116705E01D
:203C2000516703E0D16201E01163FFE7F0BDF0B500231E000A78D406E40E01221500A5407D
:203C40000F78402F1ADB2A0002230668002B10D0022B06D009D3032B0FD1B76E1743B76628
:203C60000BE0F76E1743F76607E0776A1743776203E0B76A1743B762FFE735E00E78202EFC
:203C800019DB2B000668002A10D0022A06D009D3032A0FD1B76E1F43B7660BE0F76E1F434C
:203CA000F76607E0776A1F43776203E0B76A1F43B762FFE718E02A000668002B10D0022B77
:203CC00006D009D3032B0FD1B76E1743B7660BE0F76E1743F76607E0776A1743776203E0A3
:203CE000B76A1743B762FFE7F0BDFFB591B00025012009900120089008200190032104919E
:203D00000222059214221092834A0F92FA2292050E921BAA1278002A0DD1804A0D925E220F
:203D200002920C911F2107910299079A8918491C0B910A900CE0794A0D92262202920C913B
:203D4000072107910299079A8918491C0B910A90139800F0EDF8040001260D98B04259DBB5
:203D6000129800F0E5F80500300000F0F1F80100280000F0F8F80500139800F0D9F8010043
:203D8000280000F0F0F800F041F900900098002803D000980A99884200DA3BE0009800F054
:203DA000D7F80100280000F0DEF80700139800F0BFF80100380000F07EF98021090400F0AE
:203DC000D3F908D8139800F0B3F80100380000F072F9020006E0139800F0AAF8390000F00F
:203DE0006AF902000B980099884211DB2000110000F0BAF90CD80996009801901400109830
:203E00000099884204DB10000F9900F0C1F901D3761CA2E714A8008800F08AF80E9900F0C2
:203E2000CAF9039001980299884201DA01980290029C0C98844225DB2000401C3849484398
:203E40000199FEF74FFF050014A80088281A012803DB14A800882F1A02E014A80088471BDE
:203E600014A8008885420DDB380000F071F8039900F08EF904D20494380000F069F8039021
:203E8000641ED6E701980499401A401E05902548039001250598A84221DB21486843019909
:203EA000FEF720FF07001AA80088381A012804DB1AA80088381A069003E01AA80088C01B09
:203EC0000690069800F044F8039900F061F904D20895069800F03CF803906D1CDAE70998E9
:203EE00011990860049800F0CFF90FA20CCA00F0D5F900F095FA11998860049811998968CF
:203F0000401A1199C86005981199086108981199486015B0F0BD0000CDCCCC3DFF030000BD
:203F20001027000000401C46333333333333E33F9D2102000AD002D4491E9218FCD5C90534
:203F4000100A1206524100D3012A4841704700009D210200EED55242F446FFF7EBFF01220A
:203F6000D2071043604730B405004D400122D20715404B180418240E25D01B0E2CD0FF2CB1
:203F800031D0FF2B34D0E41A000209021043114343084808D10D1B1A02D2641EDB181B1816
:203FA000DB18834200D31B1A4941F9D37F3423DDFF2C05DAE40548086041284330BC704746
:203FC000FF20C005F9E728001B0E03D0FF2BF5D14902F3D0D043F1E7FF2C01D14002F9D107
:203FE000FF20C005E9E74002F4D1FF2BF8D1F1E728004902E2D0EDE70B0200202442DCD102
:204000005B129B1CD9D9D805D7E7FEE70122D2070118090E7F3910D449421F310FD40018AC
:2040200005D2C0011043C84000D5D0437047C0011043C84005D440427047002070470042A7
:20404000F3D5100070470122D20703004B402ED4431A01D2C01AC91830B44B180418240EC5
:204060001B0E22D0FF2C20D0E31A182B1DDC09021143C40D641E0002104394461925ED1AAB
:204080000A00AA40D940451801D36D08A41CE405D209280A2D062A436546AA4160410318C5
:2040A0001B0EFF2B01D3C00DC00530BC7047514006E05140CCE70122D20703004B40F8D493
:2040C000431A03D2C01AC9185040514030B44B18090211430418240E1B0E40D0FF2C3AD070
:2040E00025009D410BD31ED8C50D4002401A0BD3ED050100400AC90591416841D5E7C50D89
:2041000040024918401AD0D001214008491C0018FCD58C4204D36D1A000AED054019C4E71E
:20412000E8051040C1E7182DBFDCAC1C0D00E140E5414D40012D4941C40D00021043451AD4
:2041400001D46D199543641EE405280A2D069541604130BC7047FF2BA7D1D843A5E7244293
:20416000A3D10020A1E7FEE70CB4012212060318DA4207D84B18DA4204D802000A439218D9
:2041800002D281420CBC7047FCD088420CBC70470CB4012212060318DA4207D84B18DA4264
:2041A00004D802000A43921802D288420CBC7047FCD08142FAE730B405004D400122D2072B
:2041C00015404B180418240E2ED01B0E32D0FF2C34D0FF2B3AD0E41800020902104311439D
:2041E000000A090A9446C2B24A43000AC3B24B43000A4843110A5B181A43D2B2190A091872
:2042000001D44918641E080A7F3C23DBFE2C08DAE40509061143634699416041284330BC48
:204220007047FF20C005F9E728001B0EFF2BF6D1D043F4E72800FF2CF1D1F9E74002F7D1D4
:20424000FF2B01D14902F3D1E005E7E7D8054902E4D0EDE743020020641CDFD15B129B1C37
:20426000DCD9D805DAE7FEE7010042221201D21E004207D002D4521E0018FCD5C10A400546
:2042800012058918704700000100EED54042F446FFF7EBFF0122D20711436047F0B50E00A5
:2042A0005E400125ED072E40B446AE0ADF184C18F44208D2F7420ED2640D01D07F0D12D1F1
:2042C00000206146F0BD05D1F74201D87F0D05D10020C143F0BDFBD1640DF9D00020C14325
:2042E000490549088FE0E419C902DB0229432B43DB0A460DC00231438E4630B487B295B28B
:204300007D432E0CADB2140C7C43A419260C240425439CB27C43A419190C7943270CC91926
:20432000A4B20F043C43090C000C97B247432E0CBE193543ADB2170C4743360CBF19A6B29A
:20434000BF193E043543240C3E0C36199FB24743BF19BCB23E0C89191F0C47437F183E0467
:204360003443390C704680B297B247432E0CBE193543ADB2170C4743360CBF19A6B2BF19E7
:204380003E043543240C3E0C36199FB24743BF19BCB23E0C89191F0C47437F183E04344388
:2043A000390C77463F0C90B278432E0C80190604ADB22E43050CA0B22D18120C7A4350191A
:2043C000020C80B2240CA4189AB27A43121914042043120C89181B0C7B43C91830BCEF0A98
:2043E000394203D1B61940414941641E6F12BF0DE41B0BDBFF19BC4211DA24050027420845
:20440000AE417841614166463143F0BD641C05D1401C6141CF0201D34908F4E750E75DE7E5
:204420004A1812D2400DC90208430121C9070843520D40210901521A521C06D452421F3233
:2044400001D4D0407047C017704700207047000000B5010008000200D2B2802A01DB7F22F0
:204460001000C0B200BD00B501000800C0B2F12805DB0800C0B2FA2801DA012006E008004E
:20448000C0B2802801DA080000E00020C0B200BDFEB582B0070000252C006E463F20307000
:2044A00030786946097AF0220A43024032706846007B70706846007CFFF7CAFFB07038781D
:2044C000002810D0032004002000C0B2082804DA2000C0B23554641CF6E708226946F8685C
:2044E000BB6D984704E003226946F868BB6D984740B205B0F0BDFEB5060000200500010063
:204500006A460F2313701378F48AF02727431F40177004002100C9B2F38A89B2994209D2B8
:2045200031692300DBB2C95C2300DBB2D3185970641CEFE73178002916D005002800C0B2FB
:204540000721F38AC91A884208DA2800C0B2F18A40181018CC2141706D1CEFE708226946BC
:20456000F068B36D984706E0F28A521CD2B26946F068B36D984740B2FEBD3EB50500684637
:204580001F2101700178EA8A92B2120AF02313430B400370E98A417000242100C9B2E4B27C
:2045A0002100C9B2062909DA29692200D2B2895C2200D2B282189170641CF1E708226946BE
:2045C000E868AB6D9847010049B2002904D1298B891D29830121A97640B23EBDFEB50600AD
:2045E00000273900C9B201A82F2202700278B37EF0241C4314400470F28A338BD21A6B46B7
:204600001A806A461288082A02DB07226B461A803C00E4B22100C9B26A46128889B291426D
:204620000BD23169328B2300DBB2D218895C2200D2B282185170641CECE7317800291BD0B6
:204640003900C9B23D00EDB22A00D2B207216B461B88C91A8A4209DA2900C9B26A46128820
:2046600089184118CC224A706D1CEDE7082201A9F068B36D984707E068460288521CD2B2FF
:2046800001A9F068B36D9847010049B200290BD1318B6A46128889183183B17E491CB17602
:2046A000B17E102900DBB77640B2FEBDF8B504000D00160000210F000F202B7802001342B0
:2046C00006D03200D2B2521E2B7803409A4208DA606D002802D0A248616D88470620C043C3
:2046E00015E02A7810404222A0520800C0B24222A25A80B2904209D20800C0B22818407852
:20470000E26B0B00DBB2D054491CEEE70020F2BDF8B504000D001700002108006A46107059
:204720003800C0B2082808D0606D002802D08D48616D88470620C04339E028780002F02298
:204740001201024068781618300080B2082808DA606D002802D08448616D88470620C04329
:2047600025E04020205A320092B2904208D2606D002802D07D48616D88470220C04316E0F4
:20478000422026520800C0B2062809DA0800C0B228188078E26B0B00DBB2D054491CF1E7BC
:2047A00006204422A05201204622A0540020F2BDF4B505000C00002217004620285C2178B9
:2047C0000907090F884202D00320C04340E04220285A4421695A461A300080B2082801DBF5
:2047E0000720060068460078401E310089B2884208DA686D002802D05D48696D88470620B1
:20480000C04325E011000800C0B2330080B29BB298420CD2E86B0B00DBB24427EF5BDB1907
:204820000F00FFB2E7197F78C754491CEBE74420285A80194423E8524620285C401C4623A0
:20484000E8544620285C102801DB46202A540020F2BD70B504000D0016003000C0B2032852
:2048600008DA606D002802D04248616D88470620C04300E0002070BD70B504000E001500C6
:204880002B009BB23200E168200000F001F870BDFEB5040000263700002C02D10020C043B9
:2048A0005CE0A08A69460989884208D2606D002802D03148616D88470220C0434EE0342029
:2048C000205C012808D1606D002802D0CA48616D88470120C04341E068460089E0823000D6
:2048E000208335002800C0B26946098980B2884209D201982900C9B2405C21692A00D2B21D
:2049000088546D1CEEE7E08A082804DA2000FFF7F2FD070020E02000FFF72FFE0700380057
:2049200040B2002818D13000A0833000A0773000E077E06D80472200203203C2083AE06D77
:2049400080470022643051412200283203C2083A2663012034216054380040B2FEBD00002D
:20496000F4B0000020B10000ECAF000024B000004CB100006CB100005CB00000FFB583B046
:2049800004006846007E022803DB6846007E092800DB2FE100252900C9B22800C0B2010033
:2049A0006A46127EC9B2914209D205990200D2B2895C01AA0300DBB2D154401CEFE72F00C4
:2049C000FFB23800C0B208216A46127E891A884208DA01A83900C9B26A46127E89184554ED
:2049E0007F1CEEE701AE3078C0B20009002806D0022865D021D3032800D1B3E0FAE051204A
:204A0000205C012804D10520C0435021605401E0502025546846027E01A92000FFF746FED3
:204A200069460870694600200856002804D10498A063022051216054DCE05120205C01286C
:204A400004D10520C0435021605401E0502025546846027E01A92000FFF75AFE69460870FD
:204A60006946002008560221C94388420CD10720C043502160545120255400230022022192
:204A80002000FFF705FDB5E0694600200856002815D10498A0630120512160546078472108
:204AA000605401234720225C00212000FFF7F0FCE06D8047002264305141A064E16499E0F8
:204AC0005120205C012804D00520C0435021605490E00498A16B884200D08BE06846027E54
:204AE00001A92000FFF764FE694608700326F643694600200856B04207D101A800F0A6FBDA
:204B0000502026545120255474E0694600200856002826D1E06D8047002264305141A064C1
:204B2000E1644420205A4221615A884203D302205121605415E06078002812D04720205C92
:204B4000401E472160544720205C002809D160784721605401234720225C00212000FFF7C2
:204B600097FC47E03420205C012843D16846027E01A92000FFF76DFE69460870694600201F
:204B80000856002835D1E06D80470022643051412200283203C2083A0F2031780140022966
:204BA00006D10720C043206302203421605420E03178014001290CD1E07F401CE077E07FE4
:204BC000022816DB0620C04320630220342160540FE0317801420CD17078002802D184487C
:204BE000A08301E07078A083B078FFF73CFCA077E577FFE707B0F0BD90B00000FEB501009F
:204C0000089A0020030051240C5D022C02D00420C04328E08C6B8D68AC4201D1012400E011
:204C20000400009D2C7042240C5B6D462D892600B6B2B54202D26D462D892C0005002B00E3
:204C400026009BB2B6B2B34209D2CB6B2E00B6B29B5D019E2F00BFB2F3556D1CEFE714806B
:204C60005123C8540020FEBD70B402000B0018781070587850705868506098689060D86858
:204C8000D06018691061988A908200242000D08220001083200090762000908320009077F5
:204CA0002000D077002000211500203503C5083D1500283503C5083D146325003426955576
:204CC0009D69D5639D8B402695532500422695532500442695532500462695552500472627
:204CE00095559064D16420005021505451201454186A5065586A9065986AD06570BC70478B
:204D000070B504003420205C01285AD1384DA08BA84202D0A08B002841D0A07F002810D04F
:204D2000A07F00283BD0E06D804702000B002000203003C8801A9941002930DC01DB002818
:204D40002DD22000FFF74AFC0600300040B2002822D1A08BA84202D0A08B4019A083E06DDA
:204D600080470022643051412200283203C2083AE06D804702000B00A07F0021801859410E
:204D80002200203203C2083A208BE18A884206D300203421605402E0022034216054E06D5C
:204DA0008047220028320CCA121A8B41002B08DC01DB002A05D20120C043206302203421D8
:204DC00060545120205C012811D1E06D8047A26CE36C121A8B41002B09DC01DB002A06D2D0
:204DE0000220C0435021605400205121605470BDFFFF000008B4024B9C4608BC6047C0469C
:204E000039020020F0B5020052B2002A17D41822B74B040064B2A408A4001C59FF25C60072
:204E20001640B540AC438D01EDB2C600324095402543020052B2920892009D501BE00F224B
:204E4000AC4B182405006DB21540083DAD08AE0005006DB22A40083A920892009A58FF25EC
:204E6000C7002740BD40AA438D01EDB2C7003C40A54015439D51F0BD10B50400601E8021EA
:204E80004904884201D301200EE0601E9A49086003210020C043FFF7B5FF002097490860F6
:204EA0000720BD490860002010BD002202604160012303724272704700B5017A00290FD00F
:204EC000417A00290CD101684268914208D20168491C016001684268914201D10121417295
:204EE00000BD70B504000E001500AC48215AD6482018FFF7DAFF7820205C012806D02A00D8
:204F000092B2310020001830FFF7B6FC70BDFEB505000E001400082100226F46380000F0DD
:204F200095FA2000C0B2782805D09C48295AC6482818FFF7BAFF7920285C002814D020002E
:204F4000C0B211280FD02000C0B212280BD02000C0B2312807D02000C0B27E2803D0200033
:204F6000C0B27F2800D10AE068467F210170467084700322694628001830FFF77DFCF7BD8D
:204F800010B5040088200001201803C80022401C514188221201A21803C2083A8920000164
:204FA0002018FFF789FFB5482018FFF785FFA6482018FFF781FF10BDB14803C8704780B573
:204FC000B0480168491C0160AD4A03CA083A0023401C594103C2083AAB48FFF7D1FF01BD0D
:204FE000F8B596B0002000216A461170A74C68460078CC21615C884251D2684600786946C7
:205000000873A34D03A92868FEF73CFD002840D0D020205869460978142251434018407A0F
:20502000012832D103A92868FEF7E6FC03A92868FEF77FFC03AC4820205C029003A808307D
:205040000190944D982040012E1830784C2148432818071D029A0199380000F039FA04986E
:2050600031784C225143685030784C214843281844214822A25C42543078401C307030783E
:20508000202806D30020307003E003A92868FEF7B3FC68460078401C69460870A6E717B06F
:2050A000F0BDF1B582B000246846047079487A49451898214901415C2A78914215D04C26D8
:2050C00029784C22514340180190029F32000199380000F0FDF92878401C2870287820283D
:2050E00000D32C7001206946087068460078FEBD00E400E01CED00E014E000E018E000E0BF
:20510000F3B595B0170000242600F6B22000C0B2E4B25E482100CC22825CC9B291420ED2B0
:205120001599D02282582300DBB214256B43D2185268914201D1260001E0641CE9E7D030BE
:2051400002A902683300DBB214256B43D25A0A7048228F5400683100C9B21422514340186A
:20516000406803903800C0B201901698009002A805000835019A0099280000F0A9F9444D10
:2051800002A92868FEF786FB02A92868FEF774FB002017B0F0BD000010E000E08C080000C7
:2051A000FEB5002402943A4F934E3000803038603500D03505220021280000F09AF905224C
:2051C0000121280000F095F9304D2800FDF715FF0420CC2168548948D021685001200100F1
:2051E0002970210069702100A9702100E97030216C54C821685402AA0B2130000830FDF77E
:20520000F0FC687801280BD101200190FA20C00000907B4B7B4A029928001C30FEF765FDB0
:205220000020019078480090754B784A029928000830FEF75AFD29003868FDF7FFFF0920C0
:2052400000F0F4F9F7BD0000A808000010B5040000200100C9B2082908DA0100C9B2615C5C
:205260006B4A0300DBB2D154401CF2E7082268498D208000FFF744FF10BD00009C080000DD
:2052800000200020A032002008200020D04F0020A8500020CC3C002001130000F8B59CB008
:2052A00000F0E6FA5B49002000F03EFD00F0B4F9514C200000F048FDC0204000201800F058
:2052C000E1FD5548039000260296544D029A0399280000F0BBF8D82001900096504D009A08
:2052E0000199280000F0B2F8012004A902000A70888004AA132120000830FDF78FFC04AA99
:20530000142120000830FDF789FC04AA152120000830FDF783FC04AA162120000830FDF7A7
:205320007DFC04AA172120000830FDF777FC2500D83501220921280000F0DBF80122092198
:20534000280000F031F900220921280000F03BF9FFF726FF334D3449280000F0BDFD334B0B
:20536000334A29002000603001F033F8314F3A00092120000830FDF734FC3868FA21890017
:20538000FDF7B3FCFFF778FD2B4800F04FF920006030FFF72FFD00F031F928480168002966
:2053A00013D0066026480168491C016001680168FA229200914200D30660012001F00CF964
:2053C000280001F0D9F901F0F1F809A8FFF769FE0128E2D109981B49884203D009981A4978
:2053E0008842DAD109A84421435C021D099928001830FFF7C3FAD0E71C3100209CAF000030
:205400004C1D000080841E00C409000020A10700EC0600200CB2000004130000CC3C00205D
:20542000D04F002008200020B80600200F4F0000E34E0000A8320020FFFF0000A03200208E
:20544000A432002031070000DF0700001206130A1A43130C1A4300BF094205D0830705D0EC
:205460000270401C491EF9D1704700001300103906D330B41400150010393CC0FCD230BC35
:20548000490700D30CC000D504C0890002D30280801C002900D502707047000070B4103A73
:2054A00003D378C9103A78C0FBD2530701D318C918C001D508C908C0D20704D30B8803806A
:2054C000891C801C002A01D50B78037070BC70478B0701D18307E1D0124205D00B78491C02
:2054E0000370401C521EF9D170470000016042607047F5B582B06846007B002828D168465E
:20550000007B6A4610700800029A12688300D458244B23406C4624782402E025ED00254076
:205520001D430195019B8400135101230C00029D2D68A600AF590426B743BC461E00F6B2F3
:20554000B60004273E4067463E43A700EE5127E000200A00029B1B6894001C590425AC4366
:205560000500EDB2AD000426354025430195019C95005C516C46247B6D462C700C00029D13
:205580002D68A600AE59074F3740BC466E4636783702E026F6003E4067463E43A700EE51D1
:2055A000FFBD0000FFF8FFFF30B443685B6901248C40A3431400E4B28C401C43230045686B
:2055C0006B6130BC704730B443681B6801248C40A3431400E4B28C401C43230045682B6043
:2055E00030BC704700B5010049B2002905D40121C206D20E91400B4A116000BD00B50A4830
:205600000168012906DB0168491E01600068012800DA62B600BD000072B603480168491C64
:205620000160704700E100E01831002010B50400200040B2FFF7D6FF10BD000010B55B4C49
:205640000320206160615A48A0615A49E1618021C90021620021A1626162E1622066564822
:2056600060661020A0662167E166616753A1E01D01F0FCF85249200001F0F8F82020A071D4
:2056800010BDF1B586B00C001500002001900698C7680698006900900098874203D200985D
:2056A000C01B401E05E006988068C01B00994018401E06998968C91B884202D30698806883
:2056C000C01BA84201D2060000E02E0006984068C01903900596049403980290059A0499D0
:2056E0000298FFF7F5FE0298019880190190A419AD1BBF1906988068874201D10020070025
:205700000698C760002DC4D1019807B0F0BDF8B588B004000D001600E0680390A06803997A
:20572000401A0290029886420FD2606803994018009005960495009F059A04993800FFF7B1
:20574000C7FE03988019E06020E0029801906068039940180090019807900695009F079A8E
:2057600006993800FFF7B4FE0298301A01906068009001980590029828180490009F059A03
:2057800004993800FFF7A4FE0198E06009B0F0BD00B501000A69CB68934204D38868401E07
:2057A000C01A801801E0D01A401E00BDAC50002034B2000054510020545500205254540007
:2057C00040B20000F1B582B00F0015000197274802991822514340180600183670690028BE
:2057E00003D0022821D010D326E03000FFF7D0FF00900098A84201D2002405E02C002A0099
:2058000001993000FFF783FF17E03000FFF7C0FF00900098A84201D2009C00E02C002200BB
:2058200001993000FFF773FF07E02A0001993000FFF727FF040000E000242000FEBDF1B5B6
:205840000F001600094D2878002801D1FFF7F6FEEFF31084012080F31088320039000098A4
:20586000FFF7B0FF84F31088F2BD0000AC50002080B5FFF7E3FE01BD70B504000E00A5689B
:2058800061682800401C814207D3206846552800401CA060E068401CE060A06861688842F8
:2058A0000DD1A26821682069FFF7C9FFA168884203D00020C043E06001E00020A06070BDF9
:2058C000F7B584B01F000C9D059802900124012602980699884206D302980699FDF705FA9D
:2058E0000290761CF4E7BE4200D23E000D98C0071BD4002D19D00D98800705D5002F03D11F
:2059000030206946087002E0202069460870002D0BD0AE4209D26D1E684601780498FFF7B0
:20592000ABFF0498C0680028F1D50498C06800283CD4022F01D37F1E08E005982100FDF7D3
:20594000D4F9019001980699884202D306984443EFE705982100FDF7C8F9019005980199DC
:205960006143401A059012480199415C0498FFF783FF0498C068002806D420000699FDF776
:20598000B4F90400002CE4D10D98C0070ED5002D0CD0002D0AD0AE4208D26D1E20210498E4
:2059A000FFF76AFF0498C0680028F2D507B0F0BD24B20000FEB582B007000A9C0298002847
:2059C00002D50298454200E0029D01260398854206DB28000399FDF785F90500761CF5E73D
:2059E0000498864201D204980600002C06D00298002802D40B98400700D5641E0B988007C9
:205A000002D50498002810D00B98C0070DD4002C0BD0002C09D0A64207D2641E20213800F8
:205A2000FFF72AFFF8680028F3D5F868002836D40298002807D50298414202912D21380091
:205A4000FFF71AFF06E00B98400703D52B213800FFF712FFF868002821D40B988007800FCE
:205A6000022810D1049800280DD1002C0BD0002C09D0A64207D2641E30213800FFF7FCFEB1
:205A8000F8680028F3D5F868002808D40B9801900094049B039A02993800FFF711FF05B0C0
:205AA000F0BDF5B59BB00C000AA8059040200690002007901B9809900020089020780700A1
:205AC000641C3800C0B2002800D11BE13800C0B2252800D00DE1002005000121029122787E
:205AE00017003A00D2B2232A13D02B2A0CD02D2A02D0302A03D011E00D43641C0FE02A0040
:205B000002251543641C0AE02A0004251543641C05E02A0008251543641C00E00290029A4F
:205B2000002ADCD1039021780F003900C9B2302903DB3900C9B23A2906DB04902078010043
:205B4000C9B22E2920D109E0641C03990A2251433A00D2B2891830390391E4E7641C21787D
:205B600008000100C9B2302903DB0100C9B23A2900DB09E0641C04990A2251430200D2B264
:205B8000891830390491EAE727783800C0B26C2803D03800C0B2682803D1641C20780700B8
:205BA000F3E73800C0B2252800D19BE058284ED063280AD064281CD070287BD073285DD0A2
:205BC00075282DD0782842D091E01C9800681C9908601C98006800681C990968091D1C9A49
:205BE00011600290029E3100C9B205A8FFF744FE7DE01C9800681C9908601C980068006857
:205C00001C990968091D1C9A11600290019503980090049B0A22029905A8FFF7CBFE66E0A6
:205C20001C9800681C9908601C98006800681C990968091D1C9A11600290019503980090E1
:205C4000049B0A22029905A8FFF73AFE4FE01C9800681C9908601C98006800681C990968F1
:205C6000091D1C9A11600290019503980090049B1022029905A8FFF723FE38E01C98006820
:205C80001C9908601C98006806681C980068001D1C99086030780700761C3800C0B20028F4
:205CA00007D03900C9B205A8FFF7E6FD08980028F0D51CE01C9800681C9908601C980068F5
:205CC00000681C990968091D1C9A11600290002001900820009008231022029905A8FFF753
:205CE000EFFD04E0252105A8FFF7C6FDFFE7641C04E03900C9B205A8FFF7BEFD0898002804
:205D000000D4DBE6089801280BDB0798002804D0079A0AA91B98FFF792FD08980799401880
:205D2000089008981DB0F0BD0CB438B505000C0004A800906A4621002800FFF7B2FE01B067
:205D4000029930BC03B00847F0B58BB0040035480590069000200790089009900A90324D2D
:205D6000324F334E05A8039002960197314800902B00314A314920000830FCF70BFF2A0009
:205D80002F492000603000F0ABFD02206946087404A803902B48029001960095264B3A00DB
:205DA000294920008030FDF718F9284A28492000C830FFF79BFB274A27492000D030FFF71E
:205DC00095FB264A26492000D830FFF78FFB254A25492000E030FFF789FB244A244920002A
:205DE000E830FFF783FB0095124B320021492000F03000F0ABFE104B3A00104988204000DA
:205E0000201800F0B5FE1C49B2204000201801F04BFB1A49C0204000201800F031F80BB032
:205E2000F0BD00BF00127A0000E0064000F8064000E8064000E4064000F0064000F0074041
:205E40000000024000F00540008003400050034000000640405003400010064080500340F3
:205E600000200640C050034000300640005103400040064000D0074000C0024000A00740D9
:205E80000160704710B502680121126852090A401300DBB2012B19D10D4B046863600368D2
:205EA0001B688024A343046823600A4B0468A36003681B68DB0A0B40DBB2002BF8D1036818
:205EC0001B685B0A0B40DBB2002BF8D010BD000020C528D9FFFF000038B505000C0021003F
:205EE000280000F010FC0548A8600548E8600F206860044828610620A88231BDCCAE000010
:205F0000C4B000005C080020F3B581B01400C0252600F6B2281D0090029F32000099380070
:205F2000FFF7D6FAF7BD43780B707047F3B581B01400C0252600F6B2280028300090029FA9
:205F4000320000993800FFF7C3FAF7BDF5B583B00C00C0250C200290280018300190260024
:205F6000029A01993000FFF7B3FA082628000C30009027000C37320000993800FFF7A8FAF1
:205F80002020E07205B0F0BDF3B581B01400C0252600F6B20095029F320000993800FFF73E
:205FA00097FAF7BD30B500231C001500E4B2EDB2AC4205D220241D00EDB24C555B1CF3E777
:205FC00030BD000008B4024B9C4608BC6047C0464D02002008B4024B9C4608BC6047C046AD
:205FE0004D04002038B50124A34D0C21280000F0C7FD002813D10121280000F0C1FD0128F8
:206000000AD19E4801689E4A914202D00020040007E00021016004E00020040001E0002033
:2060200004002000C0B232BD802000017047F0B50400200000252E00954209D2914E4F5D2A
:206040004740FFB2BF00F659000A70406D1CF3E71E00F6B2012E02D10026F643301AF0BDBF
:20606000FEB5002701970097FFF7D6FA8648FDF73EF885242401854D3A0021002800FFF740
:20608000E5F9802040020568814806688148066081490D600A6882F30988096881F3088849
:2060A00080214902B94A116000688047F7BD70B585252D010024754E220029003000FFF748
:2060C000C5F9FFF7A9FA23216B4800F019FE70BDE0B56846762101706C4B3421595C417081
:2060E0000222694658689B68984707BD80B56748417C002916D184210901415C012903D06D
:20610000B249415C01290AD10021A14A81500121AE4A8154022141744068417002E00420DF
:2061200000F082F901BDF8B5584C607C002802D0607C012832D1E06900282FD0206AE169C3
:2061400088422BD200252E006769C048205C032814D0FFF761FA01216069FFF733FF060058
:206160003000C0B2002807D1E169491E8020C0003818FFF727FF0600FFF740FA3000C0B228
:20618000002805D102206074E561A561256205E0E561A5612562032000F046F9F1BDF8B5D3
:2061A000A0480078012864D1384C607C002802D0607C01285DD1B248205C012859D1E06A81
:2061C000A16A884255D200263700A048205C03282BD03000694608703000694648700220CC
:2061E00069460870FFF718FA3500280069460978C0B2884217D28022D2002800C0B280022E
:20620000201801003531606AE36AC0182B00DBB29B02C018FFF7DEFE07003800C0B2002818
:2062200001D16D1CE1E7FFF7E9F93800C0B2002813D1E06A802109014018E062E06AA16AC9
:20624000884205D330008F4960540220607401E001206074FFF73CFF07E030008949605446
:20626000A662E662032000F0DFF83000844960542663F1BD000000002C320020F06300200B
:2062800055AAAA55D88700009C310020C0280020040001001431002010310020F8B5A34C45
:2062A000607C002802D0607C01286DD12600113601253570654820180178012902D00178BA
:2062C000002957D18D4801F021F900284AD18C4801F01CF9002845D188480068894988425E
:2062E00007D03A482554022030700020B74960544AE08F480768824800688E4940180090D5
:206300000098A021890288420ED200988A4988420AD30123009A802149020020C043FFF71A
:2063200086FE8649605002E000208449605083482058874207D02548255402203070002030
:20634000A249605420E0A1482554204820180178002903D1052000F067F815E00570022026
:20636000307011E0194825540220307000209749605409E00178022906D00078032803D162
:206380009248255402203070F1BD000008ED00E04808000080B56548417C002902D0417CBE
:2063A000012912D18A4941580A290CD30749415C002908D195490020FFF7B6FCFFF72CF9A2
:2063C000FFF74EFE01E00121417401BD430800007047FEB582B006008520000101900025BC
:2063E0000095524C2700009A01993800FFF72EF82660029860600398A0600498E0604F48CD
:2064000025503000FEF7F6FCFFF7ECFD012807D16F48255001204A496054022061684870D9
:2064200005B0F0BDFD3000200021404A0B0053741074774BD15070477648007C7047754864
:20644000407C704774480078704700004408000010B560493A4A8A181378002B07D18423C9
:206460001B01C85400236A4C0B510123137002224A7410BD574A694BD054694BD154704750
:206480003E0800003D08000038B505000C0051488461456100210A00624BC254624A8154E0
:2064A000802149028D420CD1A02189028C4208D101215E4A815481695D4A8918890AC161CB
:2064C00017E0002D0AD1082C08D10221574A81548169574A8918890AC1610AE055498D42DF
:2064E00007D155498C4204D20321504A81540221C1610120FFF798FF31BD0000C00001004D
:20650000F87F0300DDCCBBAA38B505000C0031480121454A815400210A00424BC254456281
:206520008462C1620220FFF77FFF31BDC0280020FC7F03000000FFFF0140000038080000C9
:2065400043080000F4B503000022140010000C00A4B2A24208D21F4C256BAD186419352547
:206560009E5C6655521CF2E71A4C256B0E00B6B2AD1925636D462D783426A555256B802683
:206580003601B54204D301252E00264FE6552800C0B2F2BD00200F4902004A7404220A74CD
:2065A00002000A4BCA54254A8850704780B50948017C062909DA2249027C92008A58002ACC
:2065C00003D0007C80000858804701BD3C08000048080000C028002010B504000D48017CD0
:2065E000002902D0017C052906D1094941180A682300DBB2D2180A600849401801780129B1
:2066000003D100210170FFF752FD10BDF4B1000048080000C0280020FC3000204108000070
:20662000420800003E0800003D08000044080000FF030000F05B0020010800003808000083
:20664000A00600200021016041600A00027241727047002202604160012303724272704740
:20666000407A7047FEB505000E001400082100226F463800FEF7EAFE2000C0B2782805D0B3
:206680007448295A74482818FFF7E3FF7920285C002814D02000C0B211280FD02000C0B282
:2066A00012280BD02000C0B2312807D02000C0B27E2803D02000C0B27F2800D10AE0684656
:2066C0007F210170467084700322694628001830FEF7D2F8F7BD10B502000023180018002E
:2066E00080B25468A0420CD290681C00A4B2E400005D0C00E4B2A04201D1012002E05B1C71
:20670000EDE7002010BD70B505000C00210028001830FEF7A9FA0120687000263000A870F2
:206720003000782168540020002188221201AA1803C2083AA08D49496852E08D48496852DC
:20674000208E44496852892000012818FFF77AFF44482818FFF776FF3F482818FFF772FF86
:20676000310030004049884205D231002A187B23D154401CF6E770BDFEB5040000263000E5
:206780006946C8803000694608713700350020001830FEF7B5FA01A8801C0090324B2200BE
:2067A0007B322100793120001830FEF727FA6946087169460420085600283CD17B20205C3E
:2067C00007003900C9B22000FFF785FF00282CD03500606885422ED2A068E900405C3900B6
:2067E000C9B288421FD1A068E90040188078002806D07C20205CC0B2C0097821605402E0A3
:2068000030007821605428007A2160546846C28821007B3120000400A368E80018184368CD
:206820002000984707E06D1CD3E711223900C9B22000FFF717FF08482018FFF711FF012865
:2068400006D101206070A67003482018FFF7FAFEF7BD00008C080000A80800008808000061
:206860008A0800009C0800000208000031B48B0707D00B780370002B20D0401C491C8B0726
:20688000F7D1164CE501830722D104C9131B93432B4205D104C004C9131B93432B42F9D08C
:2068A000FF231A42027009D0120A1A42427005D0120A1A42827001D0120AC27031BC7047E3
:2068C0000270120A4270120A8270120AC270001D04C9131B93432B42F2D0E1E70101010133
:2068E000F8B504000F001500276065600026A660E0208002E0608020400520618020000281
:206900006061200000F002F92076E661207E002800D06661200000F001F8F1BDF1B489B0DC
:20692000012069460871099909680791002106916A461279520002231A400692069A079BC5
:206940001A606A46D070099A126805916B46DB781B01102423400593059B13606B469870FF
:20696000099B1B6804916C46A478640120252C400494049C1C606C466070099C246803917C
:206980006D466D78AD01402635400395039D25606D462870099D2D6802916E463678F600A8
:2069A00008273E400296029E2E60099E366808910100C9B289000427394031600AB0F0BCE6
:2069C0007047F0B5010000252800012213000C681E00F6B2F60180273E4026600B681B6805
:2069E000DB091340DBB2002BF8D00B681B685B091340DBB2002B0CD10B681B681B09134031
:206A0000DBB2002B05D10B681B681340DBB2002B00D01000C0B2F0BDFFB587B000242700B2
:206A2000250009A80078402801DB012007000A98002801D1012007003800C0B200284DD1E8
:206A40000798006801260068C10930000840C0B2002802D10220070040E00798FFF75EFFB6
:206A600008206946C8702000694648700798006805900294FF20049005996A4652788918E2
:206A8000097F049A91436A46D378049A1A400A430292029A05996B465B78C9180A7709A956
:206AA00009786A46917069460E7007990E6801940390684600783018007F03998843694636
:206AC0008978039A0A4002430192019869460978711808770798FFF774FF07003800C0B26C
:206AE00000280FD12500082D0CD22800C01D0799096822000300DBB2CB181B7F0A9E7355A1
:206B00006D1CF0E73800C0B20BB0F0BD7CB5050008220021684600F0D7FD00263400FF2097
:206B2000694608706B46002200212800FFF774FF01000800C0B2002805D168460078800783
:206B400001D4012004002000C0B276BD10B4019C016042608360C46010BC704700B5BFF321
:206B60004F8F054805490860BFF34F8F00BFFDE701604260836070470400FA050CED00E088
:206B800030B50200002318000C00E4B20D2C01DBC0B2B4E00C00E4B2002C14D0022C29D03D
:206BA0001CD3042C3ED031D3062C53D046D3082C68D05BD30A2C7DD070D30C2C00D191E05C
:206BC00000D283E09AE0156801242D682540EDB2012D01D1200000E018008FE015680124A2
:206BE0002D686D082540EDB2012D01D1200000E0180083E0156801242D68AD082540EDB21C
:206C0000012D01D1200000E0180077E0156801242D68ED082540EDB2012D01D1200000E0D5
:206C200018006BE0156801242D682D092540EDB2012D01D1200000E018005FE01568012487
:206C40002D686D092540EDB2012D01D1200000E0180053E0156801242D68ED092540EDB2A9
:206C6000012D01D1200000E0180047E0156801242D682D0A2540EDB2012D01D1200000E063
:206C800018003BE0156801242D686D0A2540EDB2012D01D1200000E018002FE01568012446
:206CA0002D68AD0A2540EDB2012D01D1200000E0180023E0156801242D68ED0A2540EDB237
:206CC000012D01D1200000E0180017E0156801242D682D0B2540EDB2012D01D1200000E032
:206CE00018000BE0156801242D686D0B2540EDB2012D01D1200000E01800FFE7C0B230BD81
:206D0000F3B581B0304801998968802288506A46127A002A5AD0022A00D187E06ED3042ABA
:206D200000D1B3E000D299E0062A00D1DEE000D2C4E0082A00D109E100D2EFE00A2A00D1DC
:206D400034E100D21AE10C2A00D15FE100D245E10E2A00D18AE100D270E1102A00D1B5E1DA
:206D600000D29BE1122A00D1E0E100D2C6E1142A00D10BE200D2F1E1162A00D136E200D2E3
:206D80001CE2182A00D161E200D247E21A2A00D18CE200D272E21C2A00D1B7E200D29DE2FA
:206DA0001E2A00D1EAE200D2CCE2202A00D11DE300D2FFE2222A00D150E300D232E3232A1C
:206DC00000D167E369E300BF5245535501200100019A9268546801239C430B00DBB20340FD
:206DE000234353600024019DAD686E680127BE432700FFB23840304368604EE301200100C6
:206E0000019A9268946801239C430B00DBB20340234393600024019DAD68AE680127BE4394
:206E20002700FFB238403043A86036E301200100019A9268D46801239C430B00DBB203409D
:206E40002343D3600024019DAD68EE680127BE432700FFB238403043E8601EE30120010015
:206E6000019A9268146901239C430B00DBB20340234313610024019DAD682E690127BE43B1
:206E80002700FFB238403043286106E301200100019A9268546901239C430B00DBB203406B
:206EA000234353610024019DAD686E690127BE432700FFB2384030436861EEE20120010063
:206EC000019A9268946901239C430B00DBB20340234393610024019DAD68AE690127BE43D1
:206EE0002700FFB238403043A861D6E201200100019A9268D46901239C430B00DBB203403C
:206F00002343D3610024019DAD68EE690127BE432700FFB238403043E861BEE201200100B2
:206F2000019A9268146A01239C430B00DBB20340234313620024019DAD682E6A0127BE43ED
:206F40002700FFB2384030432862A6E201200100019A9268D46A01239C430B00DBB2034089
:206F60002343D3620024019DAD68EE6A0127BE432700FFB238403043E8628EE2012001007F
:206F8000019A5268146801239C430B00DBB20340234313600024019D6D682E680127BE4313
:206FA0002700FFB238403043286076E201200100019A5268546801239C430B00DBB203401D
:206FC000234353600024019D6D686E680127BE432700FFB23840304368605EE20120010015
:206FE000019A5268146901239C430B00DBB20340234313610024019D6D682E690127BE43B0
:207000002700FFB238403043286146E201200100019A5268546901239C430B00DBB20340EA
:20702000234353610024019D6D686E690127BE432700FFB23840304368612EE201200100E1
:20704000019A5268946901239C430B00DBB20340234393610024019D6D68AE690127BE43CF
:207060002700FFB238403043A86116E201200100019A5268D46901239C430B00DBB20340BA
:207080002343D3610024019D6D68EE690127BE432700FFB238403043E861FEE10120010032
:2070A000019A5268146A01239C430B00DBB20340234313620024019D6D682E6A0127BE43EC
:2070C0002700FFB2384030432862E6E101200100019A5268946A01239C430B00DBB2034049
:2070E000234393620024019D6D68AE6A0127BE432700FFB238403043A862CEE101200100BF
:20710000019A5268146B01239C430B00DBB20340234313630024019D6D682E6B0127BE4388
:207120002700FFB2384030432863B6E101200100019A5268546B01239C430B00DBB2034056
:20714000234353630024019D6D686E6B0127BE432700FFB23840304368639EE1012001004B
:20716000019A5268146C01239C430B00DBB20340234313640024019D6D682E6C0127BE4325
:207180002700FFB238403043286486E101200100019A5268546C01239C430B00DBB2034024
:2071A000234353640024019D6D686E6C0127BE432700FFB23840304368646EE10120010018
:2071C000019A5268946C01239C430B00DBB20340234393640024019D6D68AE6C0127BE4345
:2071E0002700FFB238403043A86456E101200100019A5268146D01239C430B00DBB20340B3
:20720000234313650024019D6D682E6D0127BE432700FFB23840304328653EE101200100A4
:20722000019A5268146E01239C430B00DBB20340234313660024019D6D682E6E0127BE435E
:207240002700FFB238403043286626E101200100019A5268546E01239C430B00DBB20340BF
:20726000234353660024019D6D686E6E0127BE432700FFB23840304368660EE101200100B1
:20728000019A5268946E01239C430B00DBB20340234393660024019D6D68AE6E0127BE437E
:2072A0002700FFB238403043A866F6E001200100019A5268D46E01239C430B00DBB2034090
:2072C0002343D3660024019D6D68EE6E0127BE432700FFB238403043E866DEE00120010002
:2072E000019A5268146F01239C430B00DBB20340234313670024019D6D682E6F0127BE439B
:207300002700FFB2384030432867C6E001200100019A52688023D45801239C430B00DBB294
:2073200003402343802413510024019D6D688026AE590127BE432700FFB2384030438026C6
:20734000A851AAE001200100019A52688423D45801239C430B00DBB2034023438424135110
:207360000024019D6D688426AE590127BE432700FFB2384030438426A8518EE001200100A6
:20738000019A52689023D45801239C430B00DBB203402343902413510024019D6D68902610
:2073A000AE590127BE432700FFB2384030439026A85172E001200100019A52689C23D45877
:2073C00001239C430B00DBB2034023439C2413510024019D6D689C26AE590127BE43270095
:2073E000FFB2384030439C26A85156E001200100019A52689423D45801239C430B00DBB20B
:2074000003402343942413510024019D6D689426AE590127BE432700FFB2384030439426A9
:20742000A8513AE001200100019A5268C823D45801239C430B00DBB203402343C824135117
:207440000024019D6D68C826AE590127BE432700FFB238403043C826A8511EE001200100AD
:20746000019A5268CC23D45801239C430B00DBB203402343CC2413510024019D6D68CC267B
:20748000AE590127BE432700FFB238403043CC26A85102E0FFF762FBFFE700200199896848
:2074A00080228850F7BD0000F2B482B00299016001680A690192019A80235B0013430B6100
:2074C000026813690093009B8024A4001C43146101230468256902262E43266100BF00BFC0
:2074E00000BF002607683E61F7BC704708B4024B9C4608BC6047C0460100002008B4024BA9
:207500009C4608BC6047C046A7000020F0B595B00400002528006946C8736007400F00284E
:2075200001D00120CAE06748006802900298006801260068C0093040C0B2002801D10920A7
:20754000BCE00298FFF7D2FF684686732800694608710298006814900995FF201390149984
:207560006A4612798918097F139A91436A46927B139B13400B4309930999149A6B461B79E9
:20758000D218117721006A4651736946CE700299096812910895119012996A46D2788918C4
:2075A000097F119A91436A46527B119B13400B4308930899129A6B46DB78D2181177210A71
:2075C0006A46117302216A46917002990968109107950F9010996A4692788918097F0F9A86
:2075E00091436A46127B0F9B13400B4307930799109A6B469B78D21811772100090C6A462F
:20760000D17103216A465170029909680E9106950D900E996A4652788918097F0D9A9143EB
:207620006A46D2790D9B13400B43069306990E9A6B465B78D2181177210E6A46917104212A
:207640006A461170029909680C9105950B900C996A4612788918097F0B9A91436A469279DF
:207660000B9B13400B43059305990C9A6B461B78D218117729006A465171052702990E6859
:2076800004950A903800C0B23018007F0A998843694649790A9A0A400243049204983900C9
:2076A000C9B2711808770298FFF728FF01000800C0B2002801D10B2000E02800C0B215B0B1
:2076C000F0BD0000F05B002010B504000800110002002000FDF7BAFE200010BDF1B489B017
:2076E000012069460871099909680791002106916A461279520002231A400692069A079BF8
:207700001A606A46D070099A126805916B46DB781B01102423400593059B13606B46987031
:20772000099B1B6804916C46A478640120252C400494049C1C606C466070099C24680391AE
:207740006D466D78AD01402635400395039D25606D462870099D2D6802916E463678F600DA
:2077600008273E400296029E2E60099E366808910100C9B289000427394031600AB0F0BC18
:207780007047F0B5010000252800012213000C681E00F6B2F60180273E4026600B681B6837
:2077A000DB091340DBB2002BF8D00B681B685B091340DBB2002B0CD10B681B681B09134063
:2077C000DBB2002B05D10B681B681A40D2B2002A01D007221000C0B2F0BDF2B584B0040015
:2077E0000025280069468870280069464870206801260068C10A30000840C0B200280ED133
:207800006846007C01280AD160680068010D30000840C0B2012802D13000694648702068F7
:207820000068C10930000840C0B2002801D109206DE02000FFF752FF0D20694608702900D8
:2078400022680195FF2002900B00DBB2D3181F7F029B9F43BC466B461F78029B3B406746A8
:207860003B430193019B0F00FFB2D7193B776B461B7C002B01D0370000E02F0031006A468D
:20788000117021680391019502900398694609784018007F029988433900C9B2029A0A4080
:2078A00002430192019803996A461278891808772000FFF766FF6946097C002909D0216827
:2078C0000968CA0A31001140C9B2002901D1052108006946097C002909D1216809680A0BF7
:2078E00031001140C9B2002901D1052108000100C9B200290BD169464978002907D02168E8
:207900003200D2B2520380239B011A400A60C0B205B0F0BD10B50400824804602000FFF778
:20792000DDFE0020E06110BDF3B595B000273800694608707B48046815988005800D0028B5
:2079400003D0012069460870E7E038003D001698854200D3E1E0206801260068C1093000B6
:207960000840C0B2002803D1092069460870D4E02000FFF7B3FE05216846017338006A4656
:207980009071206814900997FF201390149A6B469B79D218137F139A93439C466A46137BC6
:2079A000139A1A4063461A430992099B9C46149B6A4692799A1863461377159A6B46DA729E
:2079C00032006B465A712268129208971190129A6B465B79D218137F119A93439C466A46CB
:2079E000D37A119A1A4063461A430892089B9C46129B6A4652799A1863461377159AAB02A7
:207A0000D218120A6B469A7202226B461A712268109207970F90109A6B461B79D218137F6F
:207A20000F9A93439C466A46937A0F9A1A4063461A430792079B9C46109B6A4612799A186A
:207A400063461377159AAB02D218120C6B465A7203226B46DA7022680E9206970D900E9AE6
:207A60006B46DB78D218137F0D9A93439C466A46537A0D9A1A4063461A430692069B9C4688
:207A80000E9B6A46D2789A1863461377159AAB02D218120E6B461A7204226B469A70226850
:207AA0000C9205970B900C9A6B469B78D218137F0B9A93439C466A46137A0B9A1A406346C9
:207AC0001A430592059B9C460C9B6A4692789A18634613776A46D6716A4651702668049759
:207AE0000A90684640783018007F0A9988436946C9790A9A0A40024304920498694649788B
:207B0000711808772000FFF73CFE6946087068460078002801D16D1C19E76846007817B050
:207B2000F0BD0000F05B0020F7B598B00025280069464874874800680190072018990140A0
:207B4000002901D0012501E11A990840002801D00325FBE028006946087002950B9501980D
:207B6000006801270068C10A38000840C0B2012802D138006946087068460078002803D0D4
:207B800000210198FFF729FE18988005800D0B900B98A021490544182E001A98864205D224
:207BA0001998805D2070641C761CF6E7019800680068C10938000840C0B2002801D109256B
:207BC000BCE00198FFF78AFD0620694608742800694688720198006816900A95FF201590C7
:207BE00016996A46927A8918097F159A91436A46137C159A1A400A430A920A9A16996B4639
:207C00009B7AC9180A7718996A46D17369464F720199096814910995139014996A46527ABE
:207C20008918097F139A91436A46D27B139B13400B4309930999149A6B465B7AD21811776A
:207C40001899090A6A46917302216A4611720199096812910895119012996A46127A8918E2
:207C6000097F119A91436A46927B119B13400B4308930899129A6B461B7AD21811771899A2
:207C8000090C6A46517303216A46D17001990968109107950F9010996A46D2788918097F93
:207CA0000F9A91436A46527B0F9B13400B4307930799109A6B46DB78D21811771899090E5D
:207CC0006A46117304216A469170019909680E9106950D900E996A4692788918097F0D9A87
:207CE00091436A46127B0D9B13400B43069306990E9A6B469B78D21811771A99C908491E29
:207D00006A46D17205216A46517001990F6805950C90684640783818007F0C99884369463E
:207D2000C97A0C9A0A4002430592059869464978791808770198FFF724FD0500684600783C
:207D4000002803D001210198FFF747FD2800C0B21BB0F0BDF05B002000220260416001236D
:207D600003724272704770B504000E0015009E48215A9E482018FFF7EFFF7820205C012837
:207D800006D02A0092B2310020001830FCF774FD70BDFEB505000E001400082100226F469B
:207DA0003800FDF753FB2000C0B2782805D08E48295A8E482818FFF7CFFF7920285C0028CA
:207DC00014D02000C0B211280FD02000C0B212280BD02000C0B2312807D02000C0B27E2874
:207DE00003D02000C0B27F2800D10AE068467F210170467084700322694628001830FCF71C
:207E00003BFDF7BD30B5002003000421020013000C00DBB2E4B2A34208D2754B1400E4B2DC
:207E200014256C431B191871521CF0E730BDFFB581B0070000252E002C00280069460870B1
:207E400029002A00002F02D10A98058032E03878C0B200096B46187038780007000F6B46B9
:207E60005870280001006A461278C9B291420BD20100C9B2791849780322121AD2009140EA
:207E800031430E00401CEDE7280069464978C0B288420BD22800C0B2381840790321491B54
:207EA000C9008840204304006D1CEDE721003000FEF7EAFA05B0F0BD7047FBB5040017005F
:207EC000089D2E88FEF7B8FA012814D1FEF7B7FA0100C9B2022908D10121320092B2B954C7
:207EE000761C0021424A11710DE00221320092B2B954761C07E00320310089B27854761CC8
:207F000000203B4908712E80F7BDF8B504000F0015001E00FEF73EFBF1BD7047FBB50400A8
:207F20001700089D2E88FEF787FA042822D1FEF786FA012805D10220310089B27854761CDA
:207F400018E0FEF77CFA022814D1FEF77BFA012808D10120310089B27854761C00202549CA
:207F6000087007E00320310089B27854761C0020204908702E80F7BDF8B504000F0015007D
:207F80001E00FEF707FBF1BD7047FBB504001700089D2E88FEF750FA042822D1FEF74FFAA5
:207FA000012805D10220310089B27854761C18E0FEF745FA022814D1FEF744FA012808D166
:207FC0000120310089B27854761C00200849087607E00320310089B27854761C0020044986
:207FE00008762E80F7BD00008C080000A80800000C08002038080020704770477047F7B5F8
:20800000FFB087B0002604963000694608733000694648813400300069460870042069465A
:208020004873802080000190320005AD01992800FDF70CFA30006946088188A800888699F5
:208040008968869A7A23D25CD2008918497889B2884205D2132231218698FFF79AFE2BE1F5
:208060007F27879840783840694608738798807800028799C97840186946C88188A800885F
:20808000001F6946488168464089002802D08798001D0490350028006946497BC0B28842FC
:2080A00034D287482900C9B214225143415A6A46D289914228D1869949782A00D2B2142346
:2080C0005A4382189278914218D12900C9B2142251434118C97800290FD02900C9B21422B9
:2080E00051434018C07886998978884205D0332231218698FFF74DFEDEE007E0222231215C
:208100008698FFF746FED7E06D1CC4E728006946497BC0B2884205D3312231218698FFF7B4
:2081200038FEC9E0802080000190009605AC009A01992000FDF78AF905AC712020708798AC
:208140004078607087988078A0708798C078E0700420694608816846007B012805D000D274
:2081600081E003285BD02CD37DE055482900C9B21422514340180079012808D12770312026
:2081800060702420A07003206946088118E04C4E02A8009080239B0005AA68464189049893
:2081A00084462F00FFB214204743F01987686046B84701202900C9B2142251437118087129
:2081C0005AE03F482900C9B2142251434018007900281BD002A8009080239B0005AA6846B7
:2081E000418904980190364884462F00FFB2142047436046C019C7680198B84730482900BB
:20820000C9B2142251434018067107E02770312060702420A0700320694608812CE0284E7A
:208220002800C0B21421484330180079002811D002A8009080239B0005AA684641890498DF
:20824000B4462F00FFB2142677436646F6193669B04707E02770312060702420A0700320E9
:208260006946088108E02770312060701220A0700320694608811FE068460089042809DB43
:208280002078712806D16846028905A98698FFF76AFD11E068460089032808D120787F2809
:2082A00005D1A27831218698FFF773FD04E0242231218698FFF76DFD7FB00AB0F0BD000068
:2082C0000C080020002202604160012303724272704770B504000E0015009648215A9648BE
:2082E0002018FFF7EFFF7820205C012806D02A0092B2310020001830FCF7BEFA70BDFEB5BD
:2083000005000E001400082100226F463800FDF79DF82000C0B2782805D08648295A86484F
:208320002818FFF7CFFF7920285C002814D02000C0B211280FD02000C0B212280BD020009F
:20834000C0B2312807D02000C0B27E2803D02000C0B27F2800D10AE068467F210170467007
:2083600084700322694628001830FCF785FAF7BDFAB583B00400150001A870490A6802606E
:2083800088200001201803C8009001A8009901700099090A41700099090CC9B24278072384
:2083A0005A43891881700099090EC9B2027803235A438918C1706846007C042819D30420EE
:2083C00001000A9A11806946097BA278914208D1029000262F00320002993800FDF736F860
:2083E00007E0029001AE2F00029A31003800FDF76FF805B0F0BDFEB504002000C0B20128F2
:2084000002D0092846D093E04D4D68460E782F78774007704E786F78774047708E78AF78E5
:2084200077408770CE78ED787540C57001ADC678F02737402F70C678B700BC263E404778CC
:20844000BF07BF0F37436F7046783700FFB2BF08BC460778C0263E4067463E43AE70067813
:20846000360180780007000F3043E87028781E78B0420BD168785E78B04207D1A8789E7832
:20848000B04203D1E878DD78A84201D0002050E001204EE02A4D68460E782F787740077087
:2084A0004E786F78774047708E78AF7877408770CE78ED787540C57001AD4678B700BC460C
:2084C0008778F0263E4067463E432E700678F6B2B6083B273740BC4647787E263E406746F0
:2084E0003E436E70C6783700FFB23F09BC4607782C263E4067463E43AE7086783601C078A5
:208500007D2707403743EF7028781E78B0420BD168785E78B04207D1A8789E78B04203D117
:20852000E878DD78A84201D0002002E0012000E00020FEBD8C080000A808000048B20000AF
:208540004CB20000F7B586B000206946887208210020009003AC009A2000FCF777FF0020A7
:208560006946C8800020694608810020694648716846008C06998968069A7A23D25CD2001D
:208580008918497889B2884205D2132227210698FFF7B5FE14E106984078012805D122224B
:2085A00027210698FFF7ABFE0AE1079840784006400E6946087103AF672038706846007930
:2085C000787068460079C00700D47FE0002630007C49087034002000C0B2022837DA7A4D37
:2085E000684600792100C9B20901695C88422CD12000C0B20001281880782100C9B20901B1
:208600006918497888421FD206988821090140180CC808382000C0B200012818083003C8CA
:20862000121A8B41694800218B4208DC01DB824205D2362227210698FFF761FEC0E02000F5
:20864000C0B200012818467001E0641CC3E72000C0B2022805DB312227210698FFF74FFE8E
:20866000AEE006206946088101A8801C009068460389DBB2BA1C684601790698FFF778FE6A
:208680006846C08800281BD06846C288921C92B203A90698FFF71DFE68460079494908705B
:2086A0006846C0884A4908806846C088009003A8851C484E009A29003000FCF709FF7FE0F4
:2086C000312227210698FFF71AFE79E03D4D684600792978491C884205D024222721069878
:2086E000FFF70DFE6CE06846008C801E80B200900798831C3648028836492878FFF77BFEBF
:208700006946487168464079012822D1022203A90698FFF7DEFD0020010029706946097944
:20872000491E069A917004002100C9B2022947DA25496A4612792300DBB21B01CB5C9A42CD
:2087400005D102002300DBB21B01C9184A70641CEAE7352227210698FFF7D1FD0024200044
:20876000C0B202282CDA184A28782100C9B20901515C884222D12000C0B2000110184078D2
:20878000401C2100C9B20901511848702000C0B20001101880782100C9B209015118497833
:2087A00088420BD2069888210901401803C82300DBB21B01D218083203C2083A641CCEE772
:2087C00009B0F0BDB75500208006002010270000B4550020645500200000000096300777E4
:2087E0002C610EEEBA51099919C46D078FF46A7035A563E9A395649E3288DB0EA4B8DC79E1
:208800001EE9D5E088D9D2972B4CB609BD7CB17E072DB8E7911DBF906410B71DF220B06AF0
:208820004871B9F3DE41BE847DD4DA1AEBE4DD6D51B5D4F4C785D38356986C13C0A86B6400
:208840007AF962FDECC9658A4F5C0114D96C0663633D0FFAF50D088DC8206E3B5E10694C40
:20886000E44160D5727167A2D1E4033C47D4044BFD850DD26BB50AA5FAA8B5356C98B242A0
:20888000D6C9BBDB40F9BCACE36CD832755CDF45CF0DD6DC593DD1ABAC30D9263A00DE51D0
:2088A0008051D7C81661D0BFB5F4B42123C4B3569995BACF0FA5BDB89EB802280888055F80
:2088C000B2D90CC624E90BB1877C6F2F114C6858AB1D61C13D2D66B69041DC760671DB01CE
:2088E000BC20D2982A10D5EF8985B1711FB5B606A5E4BF9F33D4B8E8A2C9077834F9000FC0
:208900008EA8099618980EE1BB0D6A7F2D3D6D08976C6491015C63E6F4516B6B62616C1C4F
:20892000D83065854E0062F2ED95066C7BA5011BC1F4088257C40FF5C6D9B06550E9B7125F
:20894000EAB8BE8B7C88B9FCDF1DDD62492DDA15F37CD38C654CD4FB5861B24DCE51B53ABF
:208960007400BCA3E230BBD441A5DF4AD795D83D6DC4D1A4FBF4D6D36AE96943FCD96E343F
:20898000468867ADD0B860DA732D0444E51D03335F4C0AAAC97C0DDD3C710550AA4102276F
:2089A00010100BBE86200CC925B56857B3856F2009D466B99FE461CE0EF9DE5E98C9D9299F
:2089C0002298D0B0B4A8D7C7173DB359810DB42E3B5CBDB7AD6CBAC02083B8EDB6B3BF9AEB
:2089E0000CE2B6039AD2B1743947D5EAAF77D29D1526DB048316DC73120B63E3843B64944F
:208A00003E6A6D0DA85A6A7A0BCF0EE49DFF099327AE000AB19E077D44930FF0D2A30887BE
:208A200068F2011EFEC206695D5762F7CB67658071366C19E7066B6E761BD4FEE02BD389AE
:208A40005A7ADA10CC4ADD676FDFB9F9F9EFBE8E43BEB717D58EB060E8A3D6D67E93D1A1CE
:208A6000C4C2D83852F2DF4FF167BBD16757BCA6DD06B53F4B36B248DA2B0DD84C1B0AAF8E
:208A8000F64A0336607A0441C3EF60DF55DF67A8EF8E6E3179BE69468CB361CB1A8366BCDE
:208AA000A0D26F2536E2685295770CCC03470BBBB91602222F260555BE3BBAC5280BBDB22E
:208AC000925AB42B046AB35CA7FFD7C231CFD0B58B9ED92C1DAEDE5BB0C2649B26F263EC80
:208AE0009CA36A750A936D02A906099C3F360EEB8567077213570005824ABF95147AB8E26E
:208B0000AE2BB17B381BB60C9B8ED2920DBED5E5B7EFDC7C21DFDB0BD4D2D38642E2D4F15D
:208B2000F8B3DD686E83DA1FCD16BE815B26B9F6E177B06F7747B718E65A0888706A0FFF4D
:208B4000CA3B06665C0B0111FF9E658F69AE62F8D3FF6B6145CF6C1678E20AA0EED20DD74D
:208B60005483044EC2B30339612667A7F71660D04D476949DB776E3E4A6AD1AEDC5AD6D9ED
:208B8000660BDF40F03BD83753AEBCA9C59EBBDE7FCFB247E9FFB5301CF2BDBD8AC2BACA3D
:208BA0003093B353A6A3B4240536D0BA9306D7CD2957DE54BF67D9232E7A66B3B84A61C40D
:208BC000021B685D942B6F2A37BE0BB4A18E0CC31BDF055A8DEF022DF0B590B0012001009E
:208BE0006A469170DA4A04920499C96A0423DB4319406C46A478A40004252C400C430B94A7
:208C00000B99049CE16201006C46617003920399C96A0124A1436C46647804400C430A941D
:208C20000A99039CE16200210C006D462C700292029AD26A13406A4612789200042422401E
:208C40001A430992099A029BDA62CB4A0892CB4A0792089B079C23660300C94C0194019C2A
:208C600024680F25AC431D00EDB22D072D0F25430695069C019D2C60C24CC34D0595059DF0
:208C80008026AC51C14D2D682D0EAD07AD0FEDB2022D2AD10B006C462370BD4B5D68BD4CF4
:208CA0002C406D462D782D02F02636012E4026430296029C5C600C00B44D0195019E3668CB
:208CC000B54F3740BC462600F6B23704C026B6023E4067463E43019F3E602B001B681B0EAF
:208CE0009B079B0FDBB2002BF7D103000092009CE4680C25AC431D00EDB2AD000C262E4002
:208D000026430196019C009DEC6004001500EE680127BE432700FFB207403743EF6013003A
:208D20001B6A9C0803002340DBB2002BF7D00B006C4663710892089B5B690124A3436C46D6
:208D4000647904401C430F940F9B089C63610B006C4623710792079B9B691024A3436C4682
:208D60002479240110252C401C430E940E9B079CA3610B006C46E3700692069B5C69874B5F
:208D800023406C46E4782402C025AD0025401D430D950D9B069C636150236C46A370059266
:208DA000059B5B69FE24A3436C46A4786400FE2525401D430C950C9B059C63610B006C46C3
:208DC00063700492049B5C69754B23406C466478A4028025ED002C401C430B940B9B049C2D
:208DE000636104231C006D462C700392039C65696C4C2C406D462D78ED02E026B6012E4085
:208E000026430A960A9C039D6C6104000292029D6D690126B5432600F6B206402E430996E6
:208E2000099D029E7561FA256D015F4E35605F4D29605F4E05273760346880277F02BC42E0
:208E4000FAD33360584B1960296013001C6A03002340DBB2002BF8D002246B461C71554B8A
:208E60000693069DC826AE594B4D35406E4636793704C026B6023E402E430896089D069EA2
:208E8000C827F55109256E46F5700593059DC826AD59404E2E400296029D6E46F67837029A
:208EA000F02636013E402E430296029D059EC827F55105006E46B5700493049BC8255B59B2
:208EC0001025AB436D46AD782D01102635401D430795079B049DC826AB516B4658702C4DA3
:208EE0006B682C4818406B465B781E02F0231B01334003436B606846047024480390039CBC
:208F00002668254C34406E4636783704C026B6023E402643039C266003001B681B0E9B0746
:208F20009B0FDBB2022BF7D10B00154C0094009C24680F25AC431D00EDB22D072D0F254326
:208F40000295029C009D2C600C000568114E01E000F005402E402500EDB22F02F0252D011F
:208F60003D40354305600191019E1666064E8027F15110B0F0BD00BF2020961900E006406C
:208F800000E406405245535500F0064000E8064000000240FFF0FFFFFFFFFCFFFFFCFFFFE3
:208FA000FFFBFFFFFFC7FFFF14E000E018E000E010E000E000F806400022026041600123F2
:208FC00003724272704770B504000E001500B848215AB8482018FFF7EFFF7820205C012891
:208FE00006D02A0092B2310020001830FBF744FC70BDFEB505000E001400082100226F465B
:209000003800FCF723FA2000C0B2782805D0A848295AA8482818FFF7CFFF7920285C002855
:2090200014D02000C0B211280FD02000C0B212280BD02000C0B2312807D02000C0B27E2801
:2090400003D02000C0B27F2800D10AE068467F210170467084700322694628001830FBF7AA
:209060000BFCF7BDF7B5FFB085B0050000206946488000206946C8800026002069468880F5
:209080000024002069460870802189000020029004AF029A3800FCF7D9F986A80088A96876
:2090A0007A22AA5CD2008918497889B2884205D2132222212800FFF79CFFF6E086A8008841
:2090C000401EC00705D5132222212800FFF791FFEBE086A8008840086946488068464088B5
:2090E000002805D1132222212800FFF782FFDCE0622004A9320092B28854761C012738002C
:2091000086A9098880B2884200D3BEE08598390089B2405C000285993A0092B289184978F5
:2091200008436946C880002001006A46117004002000A98A80B2884200D3A0E02869210043
:2091400089B214224A43805A6946C988884200D093E0A8782969220092B214235343C91864
:209160000979884205D0332222212800FFF741FF9BE0300080B22969220092B21423534336
:20918000C91889894018801C4B49884205DB142222212800FFF72DFF87E02869210089B293
:2091A00014224A4380188078052809D068782969220092B214235343C918C978884205D2EE
:2091C000222222212800FFF714FF6EE02869210089B214224A4380188289D2B22869210000
:2091E00089B214234B43C0188168280005002B699C4623009BB21420584363461818036987
:209200002800984701206946087004A885993A0092B2895C320092B28154761C85993A009D
:2092200092B289184978320092B28154761C684686802869210089B214224A4380188089A6
:2092400003902869210089B214224A4380188068029004A8694689884618039A0299300087
:20926000FCF736F9684680882969220092B214235343C9188989461801E0641C58E76846B2
:209280000078002801D0BF1C39E768460078002806D0320092B204A92800FFF794FE04E087
:2092A000312222212800FFF7A4FE7FB008B0F0BD8C080000A80800000102000000220260F9
:2092C0004160012303724272704770B504000E0015009D48215A9D482018FFF7EFFF7820A4
:2092E000205C012806D02A0092B2310020001830FBF7C2FA70BDFEB505000E00140008210E
:2093000000226F463800FCF7A1F82000C0B2782805D08D48295A8D482818FFF7CFFF7920E1
:20932000285C002814D02000C0B211280FD02000C0B212280BD02000C0B2312807D020006A
:20934000C0B27E2803D02000C0B27F2800D10AE068467F21017046708470032269462800C9
:209360001830FBF789FAF7BD7047704770477047F4B5FFB085B005000E00002738006946F2
:209380004880380069460870380069460871022069464870802189003A0004AC2000FCF796
:2093A00055F884A80088A9687A22AA5CD2008918497889B2884205D213222F212800FFF746
:2093C0009AFFBDE06878012805D122222F212800FFF791FFB4E070780002B1784018694688
:2093E0004880F078694608703C00200069464978C0B2884223D256482100C9B21422514315
:20940000415A6A465288914217D12100C9B2142251434118897800290ED02100C9B21422D3
:20942000514340188078A978884205D033222F212800FFF760FF83E001E0641CD5E72000C6
:2094400069464978C0B2884205D331222F212800FFF751FF74E004A86F21017071784170DC
:20946000B1788170F178C17068460078002802D003281CD05FE036482100C9B214225143DE
:209480004118CF722100C9B2142251434118096900290BD02100C9B21422514340180069D6
:2094A0008047042204A92800FFF70FFF48E0284F84A800882100C9B2142251437918097A19
:2094C000091D884205DA22222F212800FFF713FF36E001202100C9B2142251437918C87291
:2094E0002000C0B2142148433818007A0390301D02902000C0B21421484338184068019003
:20950000039A02990198FBF7E3FF01982000C0B2142148433818C06800280BD02000C0B2AE
:20952000142148433818C0688047042204A92800FFF7CBFE04E031222F212800FFF7DBFEF4
:209540007FB006B0F0BD00008C080000A8080000E4070020002202604160012303724272B8
:20956000704770B504000E0015002548215A25482018FFF7EFFF7820205C012806D02A003A
:2095800092B2310020001830FBF776F970BDFEB505000E001400082100226F463800FBF75C
:2095A00055FF2000C0B2782805D01548295A15482818FFF7CFFF7920285C002814D02000C6
:2095C000C0B211280FD02000C0B212280BD02000C0B2312807D02000C0B27E2803D020006D
:2095E000C0B27F2800D10AE068467F210170467084700322694628001830FBF73DF9F7BD0E
:209600008C080000A808000010B50024FCF70CFD801C10BD10B50100002003000122130099
:20962000DBB2052B0CDA04239B1ADB000C00DC40002C03D005239B1A180001E0521CEEE790
:20964000C0B210BDF7B586B00020050001006A4611700400070001006A4651700290010082
:209660006A46D170060006994978012905D1222234210698FFF78BFFA4E069460B8C069973
:209680008A689446069A7A21515CC90062465118497889B28B4205D2132234210698FFF77E
:2096A00076FF8FE0079989780907090F6A46117007998978C9B209096A46917069460978BD
:2096C00000290BD069460978052907D269468978002903D069468978052905D33122342145
:2096E0000698FFF754FF6DE001000A006B461B78D2B29A4208D22A02079B0D00EDB25B19BF
:20970000DB78D518491CF0E70700380069468978C0B288420BD2210207986A4612783B008E
:20972000DBB2D2188018C0780C187F1CEDE7002C05D1222234210698FFF729FF42E000F0E6
:2097400083F8280000F08EF8200000F08EF8012000F091F8FFF758FF02900298FFF75AFFF8
:209760006946487003A87421320092B28154761C694649780901320092B28154761C69465F
:209780008E800126694649783200D2B291420FD302996A465278921BD200D1406A4692884A
:2097A000815469468988491C6A469180761CE9E721002800FCF7A8FE6846828803A90698A8
:2097C000FFF7CFFE09B0F0BD0022026041600123037242727047FEB505000E001400082134
:2097E00000226F463800FBF731FE2000C0B2782805D06348295A63482818FFF7E5FF7920A6
:20980000285C002814D02000C0B211280FD02000C0B212280BD02000C0B2312807D0200085
:20982000C0B27E2803D02000C0B27F2800D10AE068467F21017046708470032269462800E4
:209840001830FBF719F8F7BD002001004E4A117001004E4A11704E4908604E4908604E4920
:20986000086070474B49086070474B490860704749480068704749490870704747480078EB
:209880007047434800687047F6B583B005000A2100226C462000FBF7D9FD6878012805D1BE
:2098A000222236212800FFF796FF66E06846008AA9687A22AA5CD2008918497889B28842F0
:2098C00005D2132236212800FFF785FF55E033480078012802D0022844D049E02A4C0398E8
:2098E00040782070294E2078317888420BD020783178491CC9B2884205D0732236212800EF
:20990000FFF769FF39E0224F2348006839686A46128A8918891E884205D2712236212800A4
:20992000FFF759FF29E020783178491CC9B2884217D122786846018A891E89B20398801C11
:20994000FCF700FE012805D138686946098A4018801E386020783070684676210170217820
:2099600041700AE0312236212800FFF734FF04E0242236212800FFF72EFF05B0F0BD000023
:209980008C080000A8080000BA550020BB550020785500207055002074550020B95500203B
:2099A00091490870704730B5010089B2142928DA00218E4A0B000400A4B20C25654354199A
:2099C000237103009BB20C245C4313191B1D1C78102525431D7003009BB20C245C43131967
:2099E0001B1D1C78402525431D7003009BB20C245C431319D98003009BB20C245C43121953
:209A0000117230BD70B5010000231C001A0018001C00A4B2142C10DA744C1D00ADB20C2635
:209A20006E43A41924796406640E22001400E4B20C4200D0401C5B1CEAE780B270BDF2B5AB
:209A4000010000242500230020002500ADB2142D39DA664D2600B6B20C277743EE193679BD
:209A600033001E00F6B216422BD06E4636880700BFB23F1DBE4223DB2600B6B20C277743DB
:209A8000EE59360C0700BFB2CE55401C2600B6B20C277743EE59360A0700BFB2CE55401C4D
:209AA0002600B6B20C277743ED590600B6B28D55401C5D066D0E0600B6B28D55401C00E0CF
:209AC00001E0641CC1E780B2F2BDF0B5020000242500230020002500ADB2142D33DA434D07
:209AE0002600B6B20C277743EE19367933000E00B6B20700BFB23F1DBE4224DB2600B6B22B
:209B00000C277743EE59360C0700BFB2D655401C2600B6B20C277743EE59360A0700BFB256
:209B2000D655401C2600B6B20C277743ED590600B6B29555401C5D066D0E0600B6B29555F3
:209B4000401C641CC7E780B2F0BD38B50400002005002100264A891A04D09D3918D02F3958
:209B600035D03FE00500280080B214280FDA1F48290089B20C224A43805880214903884228
:209B800003D2280080B2FFF70EFF6D1CEBE729E00500280080B2142818DA1448290089B2E2
:209BA0000C224A4381588022D20391420CD3290089B20C224A43805880210904884203D2A4
:209BC000280080B2FFF7EFFE6D1CE2E70AE00500280080B2142805DA280080B2FFF7E3FE61
:209BE0006D1CF5E731BD0000B6550020F406002033FFFF0001000500000000000000000096
:209C00000000000009000500000000000000000000000000ED600000276100009F61000061
:209C2000D16300009D620000956300000100000031070000DF070000B1070000AC32002024
:209C400000020000AC340020200800000000000001510000B94F00003200F40188130000BE
:209C600001020304050607081A62040050000000000000001B63040050000000000000001E
:209C80001603F00050000000000000001703F00050000000000000008873C0005000000006
:209CA000000000000100C10050000000000000000101C10050000000000000000121C1009C
:209CC00050000000000000000127C10050000000000000000128C1005000000000000000C1
:209CE0000129C10050000000000000000131C10050000000000000000041C1005000000094
:209D0000000000000151C10050000000000000000063C10050000000000000000069C10042
:209D200050000000000000000181C10050000000000000000136C2005000000000000000F7
:209D40000064C10050000000000000000067C100500000000000000092F000006C550020B3
:209D600002000000699300006B93000020F000006E550020020000006D9300006F930000F0
:209D800001FD0209000000002F7E0000B97E0000BB7E000002FD020900000000797F00009B
:209DA000897F00008B7F000003FD0209000000000B7F00001B7F00001D7F000004FD0209BA
:209DC00000000000F97F0000FB7F0000FD7F000086F10601000000007C55002001000000A5
:209DE000275F000087F10601000000007D550020080000002D5F000080F106010000000060
:209E00008555002008000000095F000091F10601000000008D550020180000004D5F000089
:209E200093F1060100000000A555002004000000895F000095F1060100000000A9550020E6
:209E400008000000A55F0000002202604160012303724272704770B504000E0015007E48BB
:209E6000215A7E482018FFF7EFFF7820205C012806D02A0092B2310020001830FAF7FCFC82
:209E800070BDFEB505000E001400082100226F463800FBF7DBFA2000C0B2782805D06E48FF
:209EA000295A6E482818FFF7CFFF7920285C002814D02000C0B211280FD02000C0B21228C6
:209EC0000BD02000C0B2312807D02000C0B27E2803D02000C0B27F2800D10AE068467F2198
:209EE0000170467084700322694628001830FAF7C3FCF7BDF6B583B004000E00082100275F
:209F00003A0001AD2800FBF7A1FA3800694648706846008AA1687A22A25CD20089184978F6
:209F200089B2884205D2132228212000FFF7A9FF8EE06078012805D1222228212000FFF721
:209F4000A0FF85E070784006400E69460870B57801A8682101706946097841706846007883
:209F6000002805D0022838D01CD3032850D06AE02800C0B2012807D02800C0B2022803D0FD
:209F80002800C0B2032807D135480770022201A92000FFF760FF04E0312228212000FFF757
:209FA00070FF55E02800C0B2012807D02800C0B2022803D02800C0B2032808D1012028499C
:209FC0000870022201A92000FFF745FF04E0312228212000FFF755FF3AE02800C0B201281A
:209FE00007D02800C0B2022803D02800C0B2032808D102201A490870022201A92000FFF774
:20A000002AFF04E0312228212000FFF73AFF1FE02800C0B2012807D02800C0B2022803D018
:20A020002800C0B2032808D103200D490870022201A92000FFF70FFF04E0312228212000FF
:20A04000FFF71FFF04E0122228212000FFF719FF05B0F0BD000000008C080000A8080000B7
:20A06000B8550020002202604160012303724272704770B504000E0015002548215A2548E9
:20A080002018FFF7EFFF7820205C012806D02A0092B2310020001830FAF7EEFB70BDFEB5D0
:20A0A00005000E001400082100226F463800FBF7CDF92000C0B2782805D01548295A154845
:20A0C0002818FFF7CFFF7920285C002814D02000C0B211280FD02000C0B212280BD02000E2
:20A0E000C0B2312807D02000C0B27E2803D02000C0B27F2800D10AE068467F21017046704A
:20A1000084700322694628001830FAF7B5FBF7BD8C080000A8080000F6B585B005000E007B
:20A1200000242000694608802000694648800821220003AF3800FBF789F96846008BA9681A
:20A140007A22AA5CD2008918497889B2884205D213222E212800FFF7A2FF82E070780002BE
:20A16000B17808436946088003A86E21017071784170B17881702000A98A80B288426BD249
:20A180002869210089B214224A43805A6946098888425FD12869210089B214224A438018B3
:20A1A000007900280FD0A8782969220092B214235343C9180979884205D033222221280078
:20A1C000FFF76DFF4DE06846008BC01E2969220092B214235343C9188989884205D013224D
:20A1E0002E212800FFF75BFF3BE02869210089B214224A4380188078032809D068782969C7
:20A20000220092B214235343C918C978884205D222222E212800FFF742FF22E028692100A2
:20A2200089B214224A43801880890290F01C01902869210089B214224A4380188768029A7D
:20A2400001993800FBF744F9032203A92800FFF710FF06E0641C8EE731222E212800FFF764
:20A260001EFF07B0F0BD0000002202604160012303724272704770B504000E00150025487B
:20A28000215A25482018FFF7EFFF7820205C012806D02A0092B2310020001830FAF7ECFAC9
:20A2A00070BDFEB505000E001400082100226F463800FBF7CBF82000C0B2782805D0154846
:20A2C000295A15482818FFF7CFFF7920285C002814D02000C0B211280FD02000C0B21228FB
:20A2E0000BD02000C0B2312807D02000C0B27E2803D02000C0B27F2800D10AE068467F2174
:20A300000170467084700322694628001830FAF7B3FAF7BD8C080000A8080000F6B5FFB0EE
:20A3200082B00700002210006946487010006946087010006946488015008021890001ACA1
:20A340002000FBF783F882A80088B9687A22BA5CD2008918497889B2884205D2132219216C
:20A360003800FFF79EFF75E07F268198407830406946487001AC5920207068464078607084
:20A3800068464078012804D0022827D00A2844D05BE082A80088032805D01322192138005F
:20A3A000FFF77FFF56E0819880786946087068460078FFF727FB69464880A6700120E0707F
:20A3C0006846408880B2000A2071684640886071062201A93800FFF74EFF3BE082A80088D9
:20A3E000032805D0132219213800FFF75AFF31E08198807869460870A67068460278FF21C0
:20A40000FE31E01CFFF71BFB05002A00D21C92B201A93800FFF72FFF1CE082A800880228C6
:20A4200005D0132219213800FFF73BFF12E0FF21FE31E01CFFF749FB05002A00D21C92B298
:20A4400001A93800FFF717FF04E0122219213800FFF727FF7FB004B0F0BD00000022026054
:20A460004160012303724272704770B504000E0015006348215A63482018FFF7EFFF782066
:20A48000205C012806D02A0092B2310020001830FAF7F2F970BDFEB505000E00140008212E
:20A4A00000226F463800FAF7D1FF2000C0B2782805D05348295A53482818FFF7CFFF79206F
:20A4C000285C002814D02000C0B211280FD02000C0B212280BD02000C0B2312807D02000B9
:20A4E000C0B27E2803D02000C0B27F2800D10AE068467F2101704670847003226946280018
:20A500001830FAF7B9F9F7BDF2B582B0050017000821002422006E463000FAF797FF380095
:20A52000A9687A22AA5CD2008918497880B289B2884205D0132210212800FFF7ACFF5EE0BB
:20A54000029840784606760E68465021017046702D49695A89B2090A81702B49695AC170B3
:20A560002A49695A89B2090A01712849695A4171FDF748FC3000C0B2012806D03AD30328EE
:20A580000BD018D3042827D034E0AC706E70062269462800FFF769FF31E0AC706E70062234
:20A5A00069462800FFF761FF1548295A15482818FFF754FF23E0AC706E70062269462800AC
:20A5C000FFF753FF0E48295A0E482818FFF746FF0120FBF73DFF12E0AC706E700622694677
:20A5E0002800FFF742FF0648295A06482818FFF735FF04E0122210212800FFF74CFFF7BD0D
:20A600008C080000A8080000880800008A080000210400004D0400002D050000000000002C
:20A620004F05000045060000EF07000045080000150900006B0900003D0A0000930A0000C2
:20A64000610B0000B70B0000810C0000D70C0000A10D0000F70D0000C50E00001F0F0000A9
:20A66000810F0000B90F0000E90F00002310000057100000F1100000AD110000031300001B
:20A6800069160000000000007316000097160000C1160000E51600000F170000000000000D
:20A6A0001B1700006F170000211800004B180000751800009F180000C9180000F318000016
:20A6C0001D19000047190000711900009B190000C5190000931A0000211C00008D1C000035
:20A6E000911D0000011E0000E11E0000231F00006F1F0000B11F000001200000432000006A
:20A700008F200000D12000001D2100005F210000B1210000F1210000452200006B22000003
:20A7200095220000BB220000E52200000B230000352300005B23000085230000AB23000004
:20A74000D5230000FB23000025240000B3240000CB250000F12500001B2600007F260000D7
:20A76000292700000000000033270000000000003D2700000000000047270000C527000071
:20A78000AF2800002D290000172A0000512A0000AD2A0000E72A00003F2B0000672B0000EC
:20A7A000002202604160012303724272704770B504000E0015002548215A25482018FFF7A1
:20A7C000EFFF7820205C012806D02A0092B2310020001830FAF750F870BDFEB505000E0045
:20A7E0001400082100226F463800FAF72FFE2000C0B2782805D01548295A15482818FFF775
:20A80000CFFF7920285C002814D02000C0B211280FD02000C0B212280BD02000C0B2312805
:20A8200007D02000C0B27E2803D02000C0B27F2800D10AE068467F210170467084700322B4
:20A84000694628001830FAF717F8F7BD8C080000A8080000F2B582B00400160000221500B7
:20A8600008216F463800FAF7F1FD6078012805D1222237212000FFF7B0FF40E03000A16852
:20A880007A22A25CD2008918497880B289B2884205D2132237212000FFF79FFF2FE07720F5
:20A8A00069462A0092B288546D1C2F00FEF7E6FF012802D0022814D019E0FEF7E2FF050030
:20A8C000FEF7D6FF854205D0132237212000FFF784FF11E03A0092B269462000FFF767FF52
:20A8E0000AE0312237212000FFF777FF04E0242237212000FFF771FF0020FEF7BCFFF7BDAB
:20A90000002202604160012303724272704770B504000E0015002548215A25482018FFF73F
:20A92000EFFF7820205C012806D02A0092B2310020001830F9F7A0FF70BDFEB505000E008D
:20A940001400082100226F463800FAF77FFD2000C0B2782805D01548295A15482818FFF7C4
:20A96000CFFF7920285C002814D02000C0B211280FD02000C0B212280BD02000C0B23128A4
:20A9800007D02000C0B27E2803D02000C0B27F2800D10AE068467F21017046708470032253
:20A9A000694628001830F9F767FFF7BD8C080000A8080000FEB504000F0016000821002203
:20A9C00001AD2800FAF742FDFF253100A0687A22A25CD2008018407889B280B2814205D053
:20A9E000132211212000FFF7A8FF37E078784006400E6946087001A85121017069460978B5
:20AA00004170857068460078012804D021D3032815D00AD31DE0022201A92000FFF777FF35
:20AA200001210120FBF726FD18E0022201A92000FFF76DFF02210120FBF71CFD0EE0022215
:20AA400001A92000FFF763FF03210120FBF712FD04E0122211212000FFF76FFFF7BD00000C
:20AA6000002202604160012303724272704770B504000E0015002548215A25482018FFF7DE
:20AA8000EFFF7820205C012806D02A0092B2310020001830F9F7F0FE70BDFEB505000E00DD
:20AAA0001400082100226F463800FAF7CFFC2000C0B2782805D01548295A15482818FFF714
:20AAC000CFFF7920285C002814D02000C0B211280FD02000C0B212280BD02000C0B2312843
:20AAE00007D02000C0B27E2803D02000C0B27F2800D10AE068467F210170467084700322F2
:20AB0000694628001830F9F7B7FEF7BD8C080000A8080000FEB504000E0015000821002254
:20AB20006F463800FAF792FC2800A1687A22A25CD2008918497880B289B2884205D2132267
:20AB400085212000FFF7A9FF2DE06078012805D1222285212000FFF7A0FF24E070784706D5
:20AB60007F0E6846C521017047703800C0B2012802D0022809D011E00120FEF711FF0222A9
:20AB800069462000FFF773FF0DE00020FEF708FF022269462000FFF76AFF04E01222852165
:20ABA0002000FFF77AFFF7BD002202604160012303724272704770B504000E001500444851
:20ABC000215A44482018FFF7EFFF7820205C012806D02A0092B2310020001830F9F74CFEFE
:20ABE00070BDFEB505000E001400082100226F463800FAF72BFC2000C0B2782805D034487B
:20AC0000295A34482818FFF7CFFF7920285C002814D02000C0B211280FD02000C0B2122892
:20AC20000BD02000C0B2312807D02000C0B27E2803D02000C0B27F2800D10AE068467F212A
:20AC40000170467084700322694628001830F9F713FEF7BDF7B504000D00002216000821C2
:20AC60006F463800FAF7F2FB68460089A1687A22A25CD2008918497889B2884205D01322EC
:20AC800014212000FFF7ADFF20E0687800043043A97809020143EE780E43542069460870A4
:20ACA00030000D49401A03D09D3801D02F3808D13000FEF74AFF012269462000FFF77BFF2B
:20ACC00004E0312214212000FFF78BFFF7BD00008C080000A808000033FFFF0000220260BB
:20ACE0004160012303724272704770B504000E0015002548215A25482018FFF7EFFF78205A
:20AD0000205C012806D02A0092B2310020001830F9F7B2FD70BDFEB505000E0014000821E2
:20AD200000226F463800FAF791FB2000C0B2782805D01548295A15482818FFF7CFFF7920A6
:20AD4000285C002814D02000C0B211280FD02000C0B212280BD02000C0B2312807D0200030
:20AD6000C0B27E2803D02000C0B27F2800D10AE068467F210170467084700322694628008F
:20AD80001830F9F779FDF7BD8C080000A8080000FEB504000E001500082100226F463800FB
:20ADA000FAF754FB2800A1687A22A25CD2008918497880B289B2884205D013223E21200094
:20ADC000FFF7A9FF15E0707847067F0E3800C0B2002809D168467E2101704770022269462A
:20ADE0002000FFF782FF04E012223E212000FFF792FFF7BDF0B587B0254802902548264933
:20AE00000691264901912649264A0592264A274B0493274B0093274B274C0394069C8442C2
:20AE200007D00478029D2C70029C641C0294401CF4E7059C8C4207D00C78019D2C70019CF8
:20AE4000641C0194491CF4E7049C944203D000241470521CF8E7039C9C4207D01C78009DDA
:20AE60002C705B1C009C641C0094F4E70024134DAD08AC4207D2124DA600AD59114EA70023
:20AE8000F551641CF3E70F4D0F4E356007B0F0BD80060020F49B0000489E00000000002025
:20AEA000DC760000587D000000200020BC55002000000000000000000000000000000000FA
:20AEC000000000000000000008ED00E01002010009A5000011020100B5A900002702010040
:20AEE0004585000028030100F59E00003E02010091AD00008502010015AB000022030000DD
:20AF0000659000002E04000019A100001404000055AC0000190301001DA300002F03000028
:20AF20007193000031040100FF7F00003405000045960000360200008998000037010000B4
:20AF400055A8000072B60021002200230024002500260027B846B946BA46BB46BC460A497D
:20AF60000A4A521A013A05DD0020042308601944043AFBDA06488546064880470648804792
:20AF800062B6FAF78BF9FEE700000020EF5B0020F05B0020D98B0000F5AD00000000010043
:20AFA000310700000001080001000000FFFFFFFF01000100DF070000000108000100000061
:20AFC000FFFFFFFF02000100B10700000000080000000000FFFFFFFF03000100340200007C
:20AFE0000000080000000000FFFFFFFF4669727374206672616D652073686F756C64206EDD
:20B000006F7420757365206D756C7469706C65206672616D65207472616E736D69737369BC
:20B020006F6E2E004D756C74692D6672616D6520726573706F6E736520746F6F206C617262
:20B04000676520666F7220726563656976696E67206275666665722E000000004D65737381
:20B060006167652073697A6520746F6F206C617267652E205365742061206C617267657293
:20B080002073656E64206275666665720A00000041626F72742070726576696F7573206D20
:20B0A0006573736167652C207472616E736D697373696F6E20696E2070726F677265737316
:20B0C0002E0A00000000000000000000000000000000000000000000000000000000000038
:20B0E000000000000000000000000000000000000000000053696E676C652D6672616D65B6
:20B10000206C656E67746820746F6F20736D616C6C206F7220746F6F206C617267652E0016
:20B120004669727374206672616D652073686F756C64206265203820627974657320696EB0
:20B14000206C656E6774682E00000000436F6E7365637574697665206672616D6520746F69
:20B160006F2073686F72742E00000000466C6F7720636F6E74726F6C206672616D6520746A
:20B180006F6F2073686F72742E00000000F00DF8002801D000BF00BF00BF00BF002000BF8A
:20B1A00000BFFAF77BF800F002F80120704780B500F002F801BD00000746384600F002F818
:20B1C000FBE7000080B500BF00BF024A11001820ABBEFBE7260002000548014603B46846D9
:20B1E00080F3098800BF00BF00BF00BFFFF7CEFFA5EDF5FE2D2D2D2D2D4A756D70546F4186
:20B2000070702D2D2D2D2D0A000000002D2D2D2D2D494E544F20424F4F542D2D2D2D2D0A09
:20B2200000000000303132333435363738394142434445465465726D696E616C0000000030
:20B240005345474745520000010203044D535751FFFFFFFFFFFFFFFFFFFFFFFFFFFFFFFFEF
:20B26000FFFFFFFFFFFFFFFFFFFFFFFFFFFFFFFFFFFFFFFFFFFFFFFFFFFFFFFFFFFFFFFFEE
:20B28000FFFFFFFFFFFFFFFFFFFFFFFFFFFFFFFFFFFFFFFFFFFFFFFFFFFFFFFFFFFFFFFFCE
:20B2A000FFFFFFFFFFFFFFFFFFFFFFFFFFFFFFFFFFFFFFFFFFFFFFFFFFFFFFFFFFFFFFFFAE
:20B2C000FFFFFFFFFFFFFFFFFFFFFFFFFFFFFFFFFFFFFFFFFFFFFFFFFFFFFFFFFFFFFFFF8E
:020000021000EC
:20000000F05F002069A901002B4201007B4201000000000000000000000000000000000032
:200020000000000000000000000000006743010000000000000000004F45010037A30100A5
:20004000C0AC0100C0AC0100C0AC0100C0AC0100C0AC0100C0AC0100C0AC0100C0AC010038
:20006000C0AC010051640100C0AC0100C0AC0100C0AC0100C0AC0100C0AC0100C0AC0100CF
:20008000C0AC0100C0AC0100C0AC0100C0AC0100C0AC0100C0AC0100C0AC0100C0AC0100F8
:2000A000C0AC0100C0AC0100C0AC0100C0AC0100C0AC0100C0AC0100C0AC0100C0AC0100D8
:2000C000DDCCBBAA31343A30393A34340000000046656220203520323032350000000000FD
:2000E0005357303130315F32303235303230340000000000000000000000000000000000A6
:2001000000B583680122DB681340DBB2002B0AD083681B6A9B081A40D2B2002A03D0C069DD
:200120000860012000E0002000BD70B500231C008568EE68012296430122E4B21440344352
:20014000EC600978002943D0C169224CA14201D11D0012E0C169BA4CA14201D215000CE053
:20016000C169B84CA14201D2022506E0C169B64CA14201D2032500E004252900C9B20429AA
:2001800001D1002025E08168CC680C26B443EDB2AE000C2535402543CD608168CC68102548
:2001A000AC43DBB21B0110252B402343CB6011008368DC680125AC43C9B211402143D960B8
:2001C0008168096A8B0811001940C9B20029F7D0012070BD00093D0000B58268126A530851
:2001E0001A00D207D20FD2B2002A03D080690860012000E0002000BD7CB504000D00002019
:20020000A16801264A6931001140C9B200295BD0A1680A6A31001140C9B2002954D0A168DA
:2002200089690A0931001140C9B2002902D0012905D009E069462000FFF762FF04E0694620
:200240002000FFF7C9FFFFE7C0B2002801D100203BE03100A0684069000A8007800FC0B2BF
:20026000002805D0022807D004D3032806D007E0310005E0022103E0042101E00821FFE790
:20028000A0684069400843065B0EDBB2002B01D18023FFE7A0684069C00A4207520FD2B2F7
:2002A000002A01D10822FFE7A0684069800A34000440E4B2641C00985843604351434900B6
:2002C00002F0DFFC28603000C0B276BDF1B500242000009A9268556901239D430123C0B21E
:2002E00018402843506118004A78002A02D0012A0DD019E02600009A9568AA691027BA43AF
:20030000F6B2360110273E401643AE610DE01E00009A9568AA691027BA43F6B236011027E2
:200320003E401643AE6100E020000200D2B2002A01D1002081E0CA68012A01D126000FE090
:20034000CA68022A01D11E000AE0CA68042A01D1022605E0CA68082A01D1032600E0FF26C2
:200360003200D2B2FF2A01D1002066E0009A92685769BD4D3D40F6B23702C026B6003E4090
:200380002E4356614A88002A18D04A88812A15DA4A88802A01D1220000E04A88009DAD6811
:2003A0006E69FE27BE43D2B25700FE223A4032436A610A69002A03D100203EE000203CE0A0
:2003C0000A69092AF8D20A69082A00D00C69009A92685669A54D3540E4B2E602E024A401E2
:2003E00034402C4354618A68012A02D08A68022A24D18D686D1E009A926856699C4C344034
:20040000EDB2AD028026F6003540254355610978002911D01900009A926854690125AC4355
:20042000C9B2194021435161009989680A6A19001140C9B20029F7D0C0B2F2BD0020FCE7DB
:2004400001127A0001366E01015A6202F8B504000E0000270020009060690125C0690109F2
:2004600028000840C0B2002817D069462000FFF747FE07003800C0B200280ED06069C069D8
:20048000000A4007400F85402900412904D2009802F0F7FB306000E000273800C0B2F2BD22
:2004A000FCB500226B461A7016004569EF691023DB431F401024F6B2360126403E43EE6119
:2004C0008D88012D01D115001EE08D88022D01D1012519E08D88042D01D1022514E08D8877
:2004E000082D01D103250FE08D88102D01D104250AE08D88202D01D1052505E08D88402DE2
:2005000001D1062500E007252E00F6B2072E14D06E4635704569EF699A4E3E400196019FE7
:20052000BC466E4636783702E026F6003E4067463E43EE6101256E4635700978002901D02D
:200540000122FFE74069C1690B40D2B211010C401C43C46168460078F6BDF8B504000E0076
:20056000002700200090606901258069010928000840C0B2002817D069462000FFF7C0FD4F
:2005800007003800C0B200280ED060698069000A4007400F85402900412904D2009802F09A
:2005A00070FB306000E000273800C0B2F2BDFCB500226B461A7016004569AF691023DB43A5
:2005C0001F401024F6B2360126403E43AE618D88012D01D115001EE08D88022D01D101254F
:2005E00019E08D88042D01D1022514E08D88082D01D103250FE08D88102D01D104250AE065
:200600008D88202D01D1052505E08D88402D01D1062500E007252E00F6B2072E14D06E4669
:2006200035704569AF69574E3E400196019FBC466E4636783702E026F6003E4067463E43B0
:20064000AE6101256E4635700978002901D00122FFE7406981690B40D2B211010C401C4369
:20066000846168460078F6BDFFFCFFFFFFC7FFFFFFFBFFFFF8B504000E0000270020009071
:20068000606901254069010928000840C0B2002817D069462000FFF79FFD07003800C0B2B5
:2006A00000280ED060694069000A4007400F85402900412904D2009802F0E3FA306000E01D
:2006C00000273800C0B2F2BDFCB500226B461A70160045696F691023DB431F401024F6B264
:2006E000360126403E436E618D88012D01D115001EE08D88022D01D1012519E08D88042D6A
:2007000001D1022514E08D88082D01D103250FE08D88102D01D104250AE08D88202D01D14E
:20072000052505E08D88402D01D1062500E007252E00F6B2072E14D06E46357045696F6951
:20074000104E3E400196019FBC466E4636783702E026F6003E4067463E436E6101256E4698
:2007600035700978002901D00122FFE7406941690B40D2B211010C401C43446168460078A6
:20078000F6BD0000FFF8FFFFF8B504000E0000270020009060690125006901092800084049
:2007A000C0B2002817D069462000FFF715FD07003800C0B200280ED060690069000A4007A7
:2007C000400F85402900412904D2009802F059FA306000E000273800C0B2F2BDFCB50022FC
:2007E0006B461A70160045692F691023DB431F401024F6B2360126403E432E618D88012DE6
:2008000001D115001EE08D88022D01D1012519E08D88042D01D1022514E08D88082D01D16F
:2008200003250FE08D88102D01D104250AE08D88202D01D1052505E08D88402D01D10625A8
:2008400000E007252E00F6B2072E14D06E46357045692F69974E3E400196019FBC466E46AE
:2008600036783702E026F6003E4067463E432E6101256E4635700978002901D00122FFE757
:20088000406901690B40D2B211010C401C43046168460078F6BDF8B504000E000027002075
:2008A000009060690125406A010928000840C0B2002817D069462000FFF79EFC0700380076
:2008C000C0B200280ED06069406A000A4007400F85402900412904D2009802F0D2F930607A
:2008E00000E000273800C0B2F2BDFCB500226B461A70160045696F6A1023DB431F40102409
:20090000F6B2360126403E436E628D88012D01D115001EE08D88022D01D1012519E08D88CF
:20092000042D01D1022514E08D88082D01D103250FE08D88102D01D104250AE08D88202DCD
:2009400001D1052505E08D88402D01D1062500E007252E00F6B2072E14D06E463570456935
:200960006F6A544E3E400196019FBC466E4636783702E026F6003E4067463E436E6201250C
:200980006E4635700978002901D00122FFE74069416A0B40D2B211010C401C434462684646
:2009A0000078F6BDF8B504000E0000270020009060690125006A010928000840C0B2002809
:2009C00017D069462000FFF717FC07003800C0B200280ED06069006A000A4007400F854009
:2009E0002900412904D2009802F04BF9306000E000273800C0B2F2BDFCB500226B461A70C2
:200A0000160045692F6A1023DB431F401024F6B2360126403E432E628D88012D01D1150015
:200A20001EE08D88022D01D1012519E08D88042D01D1022514E08D88082D01D103250FE01D
:200A40008D88102D01D104250AE08D88202D01D1052505E08D88402D01D1062500E0072591
:200A60002E00F6B2072E14D06E46357045692F6A104E3E400196019FBC466E463678370237
:200A8000E026F6003E4067463E432E6201256E4635700978002901D00122FFE74069016A07
:200AA0000B40D2B211010C401C43046268460078F6BD0000FFF8FFFF80B50A00002143696A
:200AC0001B681B0E9B079B0FDBB2002B05D0022B0DD007D3032B0FD013E01100FFF77CFB2F
:200AE00001000EE01100FFF70BFB010009E01100FFF782FB010004E01100FFF76DFB010037
:200B0000FFE70800C0B202BD30B54A78012A01D100210AE04A78002A01D1012105E0497881
:200B2000022901D1022100E0FF210A00D2B2FF2A01D1002016E00A0043691C688B4D25407F
:200B4000D2B21404C022920222402A431A6042691268120E9207920F0B00D2B2DBB29A42C3
:200B6000F5D1012030BD7CB504000D00002069462000FFF7A1FF06003000C0B2002801D138
:200B800000200BE0E06800680107090F0098C9B2491C02F076F828603000C0B276BD00B590
:200BA0008A88002A0FD08A88112A0CDA8988491EC06802680F239A43C9B20907090F1143D7
:200BC0000160012000E0002000BD7CB504000D00002069462000FFF7C6FF06003000C0B242
:200BE000002801D100200CE060690068000A0107090F0098C9B2491C02F043F82860300037
:200C0000C0B276BD00B58A88002A11D08A88112A0EDA8988491E40690268554B1340C9B22F
:200C20000A02F0210901114019430160012000E0002000BDF8B504000D00002637002069FD
:200C4000C8214058000C8007800FC0B2002805D002280FD008D3032812D017E069462000CB
:200C6000FFF7BAFA070011E069462000FFF748FA07000BE069462000FFF7BEFA070005E070
:200C800069462000FFF7A8FA0700FFE73800C0B2002801D1002019E02069C821405801092F
:200CA0000800C007C00FC0B200280CD02069C8214058000A0107090F0098C9B2491C01F083
:200CC000E0FF286000E037003800C0B2F2BD30B54A78012A01D100220AE04A78002A01D1CF
:200CE000012205E04A78022A01D1022200E0FF221300DBB2FF2B01D1002036E08B88002BF7
:200D000032D08B88112B2FDA0369C8241C59174D2540D2B21404C022920222402A43C82416
:200D20001A518B885B1E0269C8241459104D2540DBB21C02F0231B0123402B43C82413513B
:200D40000978002901D0012100E000210069C822825810239A43C9B2090110231940114353
:200D6000C8228150012000E0002030BDFFFFFCFFFFF0FFFFF8B504000D006069406801098B
:200D80000800C007C00FC0B2002801D100209BE0002007000090606907264068000C3040DD
:200DA000C0B2002843D160694068C00C3040C0B200280BD0022815D00ED304281ED017D36F
:200DC000062827D020D307282AD02FE069462000FFF730FF070066E069462000FFF790F934
:200DE000070060E069462000FFF7F6F907005AE069462000FFF700FA070054E069462000EE
:200E0000FFF7B1FE07004EE069462000FFF7DDFE070048E069462000FFF718FB070042E028
:200E200069462000FFF726FC07003CE03BE060694068000C3040C0B201280AD033D30328FA
:200E400013D00CD305281CD015D3072825D01ED329E069462000FFF71EFD070023E0694618
:200E6000200000F0EFF907001DE06946200000F0C5F9070017E06946200000F09BF90700A1
:200E800011E06946200000F0ABFC07000BE069462000FFF7A1F9070005E069462000FFF7F9
:200EA0009BF90700FFE73800C0B201280AD160694068000A064031000098C9B2491C01F0A8
:200EC000E0FE28603800C0B2F2BDF2B5012319000024260045696A681027BA43F6B2360192
:200EE00010273E4016436E60009A5278002A39D0012A50D0022A67D0032A00D1AFE0052A15
:200F000000D1C5E0072A00D1DBE00A2A75D00B2A00D18BE00C2A0CD00F2A00D1F8E0102A86
:200F200000D1E8E0112A00D1D8E01A2A00D1FCE008E12600426957689A4D3D40F6B23704A3
:200F4000E026F6023E402E435660260042695768954D3D40F6B2F704E026B6033E402E43AE
:200F60005660F0E02600426957688E4D3D40F6B23704E026F6023E402E4356601E004269B4
:200F80005768894D3D40F6B2F704E026B6033E402E435660D7E0260042695768814D3D40A6
:200FA000F6B23704E026F6023E402E4356600226426957687C4D3D40F6B2F704E026B60371
:200FC0003E402E435660BEE0260042695768754D3D40F6B23704E026F6023E402E43566079
:200FE000032642695768704D3D40F6B2F704E026B6033E402E435660A5E026004269576808
:20100000684D3D40F6B23704E026F6023E402E435660042642695768634D3D40F6B2F704B4
:20102000E026B6033E402E4356608CE02600426957685C4D3D40F6B23704E026F6023E40CB
:201040002E435660052642695768574D3D40F6B2F704E026B6033E402E43566073E0260033
:20106000426957684F4D3D40F6B23704E026F6023E402E4356600626426957684A4D3D40BD
:20108000F6B2F704E026B6033E402E4356605AE0260042695768434D3D40F6B23704E02689
:2010A000F6023E402E4356600726426957683E4D3D40F6B2F704E026B6033E402E435660ED
:2010C00041E01E0042695768364D3D40F6B23704E026F6023E402E43566034E002264269FA
:2010E0005768304D3D40F6B23704E026F6023E402E43566027E0032642695768294D3D4024
:20110000F6B23704E026F6023E402E4356601AE0042642695768234D3D40F6B23704E026E5
:20112000F6023E402E4356600DE00526426957681C4D3D40F6B23704E026F6023E402E43DA
:20114000566000E021000A00D2B2002A17D0009A9288002A12D0009A9288092A0EDA009A10
:201160009688761E426957686D4D3D40F6B23702E026F6003E402E43566000E02100009AFF
:201180001278002A00D12300406942681024A243DBB21B0110242340134343600800C0B288
:2011A000F2BD0000FFFFF8FFFFFFC7FF006A08600120704700B54068806C02091000C007F2
:2011C000C00FC0B2002804D0FA2080000860012000E0002000BD00B50978002901D00121A0
:2011E00000E000214068826C10239A43C9B209011023194011438164012000BD00B54068C3
:20120000406C02091000C007C00FC0B2002804D0FA20C0010860012000E0002000BD00B52D
:201220000978002901D0012100E000214068426C10239A43C9B209011023194011434164A0
:20124000012000BDFA20400208600120704710B50200002054680123646824091C40E4B262
:20126000002C01D1002015E054686468240C1C40E4B2002C03D11000FFF775FC09E0546895
:201280006468240C2340DBB2012B02D1100000F009F9C0B210BDF3B5002211001600436886
:2012A0005F681024E44327401025F6B236012E403E435E60019B5B780A2B0DD116004368A1
:2012C0005F6818493940F6B2360480277F023E400E435E60012112E0019B5B78182B0ED131
:2012E000012143685F680F4E3E400096009EC9B2090480277F023940314359600121019B37
:201300001B78002B01D00122FFE7406843681C40D2B212011540254345600800C0B2F6BD60
:20132000FFF8FFFFFFFFFEFF10B50A00002143689B681C092300DB07DB0FDBB2002B03D080
:201340001100FFF742FC01000800C0B210BD00B50978002901D0012100E00021406882681B
:2013600010239A43C9B209011023194011438160012000BD10B50A0000214368DB681C0936
:201380002300DB07DB0FDBB2002B03D01100FFF71CFC01000800C0B210BD00B5097800290D
:2013A00001D0012100E000214068C26810239A43C9B20901102319401143C160012000BDF3
:2013C00010B50A00002143681B691C092300DB07DB0FDBB2002B03D01100FFF7F6FB010056
:2013E0000800C0B210BD00B50978002901D0012100E000214068026910239A43C9B20901AB
:201400001023194011430161012000BD10B50A00002143685B691C092300DB07DB0FDBB2AC
:20142000002B03D01100FFF7D0FB01000800C0B210BD00B50978002901D0012100E0002141
:201440004068426910239A43C9B209011023194011434161012000BD10B50A0000214368A9
:201460009B691C092300DB07DB0FDBB2002B03D01100FFF7AAFB01000800C0B210BD00B520
:201480000978002901D0012100E000214068826910239A43C9B209011023194011438161C4
:2014A000012000BDF8B504000D000020070000906068C06901090800C007C00FC0B20028A6
:2014C00001D1002054E060680726C069000C3040C0B200280BD0022815D00ED304281ED0CD
:2014E00017D3062827D020D307282AD02FE069462000FFF7BFF8070029E069462000FEF762
:20150000A5FF070023E069462000FFF7C4F907001DE069462000FFF795FE070017E0694692
:201520002000FFF747FE070011E069462000FFF765FE07000BE069462000FFF737FE07003D
:2015400005E069462000FFF795F80700FFE73800C0B200280AD06068C069000A0640310049
:20156000C9B2491C009801F08CFB28603800C0B2F2BDF2B501231900002426004568EA696C
:201580001027BA43F6B2360110273E401643EE61009A5278032A19D0052A0AD0072A22D035
:2015A0000E2A54D00F2A38D0102A43D0112A27D05AE026004268D769CC4D3D40F6B237044C
:2015C000E026F6023E402E43D6614EE01E004268D769C64D3D40F6B23704E026F6023E40C2
:2015E0002E43D66141E002264268D769BF4D3D40F6B23704E026F6023E402E43D66134E06C
:2016000003264268D769B94D3D40F6B23704E026F6023E402E43D66127E004264268D76912
:20162000B24D3D40F6B23704E026F6023E402E43D6611AE005264268D769AC4D3D40F6B2FA
:201640003704E026F6023E402E43D6610DE006264268D769A54D3D40F6B23704E026F602D8
:201660003E402E43D66100E02100009A9288002A12D0009A9288092A0EDA009A9688761E68
:201680004268D769BA4D3D40F6B23702E026F6003E402E43D66100E02100009A1278002A8A
:2016A00000D123004068C2691024A243DBB21B01102423401343C3610800C0B2F2BD10B5A2
:2016C0000200002054680123246A24091C40E4B2002C01D100201FE05468246A240CA40719
:2016E000A40FE4B2002C05D0022C0BD006D3032C0CD010E01000FEF7BDFF0CE01000FFF710
:20170000CAF808E01000FEF7A1FE04E0FA20400208601800FFE7C0B210BDF3B501210A00C2
:201720006B461A70002216004468256A10239D431023F6B236011E402E432662019C647806
:20174000032C20D0052C04D0072C0FD0112C27D033E016004468276AC54D3D40F6B2370447
:20176000C026B6023E402E43266228E00E004468276ABF4D3D40F6B23704C026B6023E4079
:201780002E4326621BE002264468276AB84D3D40F6B23704C026B6023E402E4326620EE088
:2017A00003264468276AB24D3D40F6B23704C026B6023E402E43266201E06C462270019C8D
:2017C0002478002C00D111004068026A1024A243C9B209010B401343036268460078F6BDCE
:2017E00010B50200002053689B6A1C092300DB07DB0FDBB2002B01D100201EE053689B6AC6
:201800001B0C9B079B0FDBB2002B05D0022B0BD006D3032B0CD00FE01000FFF7EFFC0BE012
:201820001000FFF7C3FC07E01000FFF7C3FC03E01000FFF7BFFCFFE7C0B210BDF3B50022A4
:201840001100160043689F6A1024E44327401025F6B236012E403E439E62019B5B78102B3E
:201860000DD1160041688F6A814B3B40F6B23704C026B6023E401E438E62012124E0019B79
:201880005B780E2B0FD1012143689F6A784E3E400096009EC9B20F04C02189023940314327
:2018A0009962012110E0019B5B780F2B0CD1022641688F6A6E4B3B40F6B23704C026B60216
:2018C0003E401E438E620121019B1B78002B01D00122FFE74068836A1C40D2B21201154006
:2018E000254385620800C0B2F6BD0000FFFFF8FF10B50200002054680123246B240C1C4095
:20190000E4B2002C03D11000FFF75FF909E05468246B240C2340DBB2012B02D11000FFF77A
:2019200091FCC0B210BD10B50200002318004C780B2C0BD151680A6B8D4C1440DBB21A04FC
:2019400080235B021A4022430A630EE0497811290BD101215268136B854C1C40C9B2090487
:2019600080235B02194021431163C0B210BD0000FFF8FFFF10B50200002054680123646B6C
:20198000240C1C40E4B2002C03D11000FFF71DF909E05468646B240C2340DBB2012B02D176
:2019A0001000FFF74FFCC0B210BD10B50200002318004C780B2C0BD151684A6B6C4C144044
:2019C000DBB21A0480235B021A4022434A630EE0497811290BD101215268536B644C1C4085
:2019E000C9B2090480235B02194021435163C0B210BD10B50200002054680123A46B240CA9
:201A00001C40E4B2002C03D11000FFF7DEF809E05468A46B240C2340DBB2012B02D1100015
:201A2000FFF710FCC0B210BD10B50200002318004C780B2C0BD151688A6B4D4C1440DBB264
:201A40001A0480235B021A4022438A630EE0497811290BD101215268936B454C1C40C9B2B5
:201A6000090480235B02194021439163C0B210BDFFFFFCFF10B50200002054680123E46B5A
:201A8000240C1C40E4B2002C03D11000FFF79DF809E05468E46B240C2340DBB2012B02D176
:201AA0001000FFF7CFFBC0B210BD10B50200002318004C780B2C0BD15168CA6B2C4C144084
:201AC000DBB21A0480235B021A402243CA630EE0497811290BD101215268D36B244C1C40C4
:201AE000C9B2090480235B0219402143D163C0B210BD10B50200002054680123246C240CA7
:201B00001C40E4B2002C03D11000FFF75EF809E05468246C240C2340DBB2012B02D1100013
:201B2000FFF790FBC0B210BD10B50200002318004C780B2C0BD151680A6C0D4C1440DBB2A3
:201B40001A0480235B021A4022430A640EE0497811290BD101215268136C054C1C40C9B2F2
:201B6000090480235B02194021431164C0B210BDFFFFFEFF10B50200002014680123E46819
:201B800024091C40E4B2002C03D11000FFF71DF80AE01268D26812091A40D2B2012A03D175
:201BA000FA20400208601800C0B210BD10B50200002318004C780B2C0BD11068C16810225E
:201BC0009143DBB21A0110231A400A43C26001200EE0497811290BD1012001001268D368D0
:201BE0001024A343C9B20901102421401943D160C0B210BD80B50269126813091A00D207BC
:201C0000D20FD2B2002A01D1002001E0FEF7ABFF02BD00B50978002901D0012100E00021B1
:201C20000069026810239A43C9B209011023194011430160012000BD80B5026952681309A7
:201C40001A00D207D20FD2B2002A01D1002001E0FEF7BBFF02BD00B50978002901D001216F
:201C600000E000210069426810239A43C9B209011023194011434160012000BD80B50269BC
:201C8000126913091A00D207D20FD2B2002A01D1002001E0FEF799FF02BD00B509780029AD
:201CA00001D0012100E000210069026910239A43C9B209011023194011430161012000BDA7
:201CC00080B50269526913091A00D207D20FD2B2002A01D1002001E0FEF777FF02BD00B559
:201CE0000978002901D0012100E000210069426910239A43C9B2090110231940114341611B
:201D0000012000BD80B50269926913091A00D207D20FD2B2002A01D1002001E0FEF723FFC2
:201D200002BD00B50978002901D0012100E000210069826910239A43C9B20901102319401C
:201D400011438161012000BD80B50269D26913091A00D207D20FD2B2002A01D1002001E023
:201D6000FEF733FF02BD00B50978002901D0012100E000210069C26910239A43C9B2090101
:201D8000102319401143C161012000BDF8B504000E0020690125006A010928000840C0B29F
:201DA000002801D1002035E02800002700972069006A000C8007800FC0B2002805D0022860
:201DC0000FD008D3032812D017E069462000FEF703FA070011E069462000FEF791F9070037
:201DE0000BE069462000FEF707FA070005E069462000FEF7F1F90700FFE72069006A000AAF
:201E00008007800F85402900009800F03AFF30603800C0B2F2BDFCB500231A001F00066998
:201E2000356A1024A5431024FFB23F0127402F4337624D78012D01D11D000AE04D78002D92
:201E400001D1012505E04D78022D01D1022500E0FF252E00F6B2FF2E0BD00269176AA24EFA
:201E60003E40EDB22F04C025AD023D403543156201221500EDB2002D2CD08D88012D01D1FD
:201E80001D000FE08D88022D01D101250AE08D88042D01D1022505E08D88082D01D10325A8
:201EA00000E0FF252E00F6B2FF2E12D06E46357005692F6A8D4E3E400196019FBC466E4693
:201EC00036783702C026B6003E4067463E432E6200E01A000978002901D00123FFE700695B
:201EE000016A1025A943DBB21B011C400C4304621000C0B2F6BD80B50269926A13091A0095
:201F0000D207D20FD2B2002A01D1002001E0FEF75CFE02BD00B50978002901D0012100E046
:201F200000210069826A10239A43C9B209011023194011438162012000BD80B50369012231
:201F40001B6B1B091340DBB2002B01D100201BE00269126B120C9207920FD2B2002A05D01C
:201F6000022A09D005D3032A09D00BE0FEF782FB09E0FEF76BFA06E0FEF78DFC03E0FEF7A2
:201F800079FB00E00020C0B202BDF2B500221100160003691F6B1024E44327401025F6B217
:201FA00036012E403E431E63009B5B78052B01D113000CE0009B5B78032B01D1012306E093
:201FC000009B5B78072B01D1022300E0FF231E00F6B2FF2E0BD001690F6B434E3E40DBB21A
:201FE0001F04C0239B023B4033430B630121009B1B78002B01D00122FFE70069036B1C4057
:20200000D2B212011540254305630800C0B2F2BD80B5036901225B6B1B091340DBB2002B22
:2020200001D100201BE00269526B120C9207920FD2B2002A05D0022A09D005D3032A09D0CD
:202040000BE0FEF717FB09E0FEF700FA06E0FEF722FC03E0FEF70EFB00E00020C0B202BDAB
:20206000F2B500221100160003695F6B1024E44327401025F6B236012E403E435E63009B19
:202080005B78052B01D113000CE0009B5B78032B01D1012306E0009B5B78072B01D102235D
:2020A00000E0FF231E00F6B2FF2E0BD001694F6B0D4E3E40DBB21F04C0239B023B40334332
:2020C0004B630121009B1B78002B01D00122FFE70069436B1C40D2B212011540254345638E
:2020E0000800C0B2F2BD0000FFFFFCFFFFFCFFFF80B5036901221B6C1B091340DBB2002B4B
:2021000001D100201BE00269126C120C9207920FD2B2002A05D0022A09D005D3032A09D02B
:202120000BE0FEF7A7FA09E0FEF790F906E0FEF7B2FB03E0FEF79EFA00E00020C0B202BD8E
:20214000F2B500221100160003691F6C1024E44327401025F6B236012E403E431E64009BB6
:202160005B78052B01D113000CE0009B5B78032B01D1012306E0009B5B78072B01D102237C
:2021800000E0FF231E00F6B2FF2E0BD001690F6CAD4E3E40DBB21F04C0239B023B403343F0
:2021A0000B640121009B1B78002B01D00122FFE70069036C1C40D2B212011540254305646A
:2021C0000800C0B2F2BD80B5036901225B6C1B091340DBB2002B01D100201BE00269526C06
:2021E000120C9207920FD2B2002A05D0022A09D005D3032A09D00BE0FEF73CFA09E0FEF72D
:2022000025F906E0FEF747FB03E0FEF733FA00E00020C0B202BDF2B50022110016000369F1
:202220005F6C1024E44327401025F6B236012E403E435E64009B5B78052B01D113000CE0DD
:20224000009B5B78032B01D1012306E0009B5B78072B01D1022300E0FF231E00F6B2FF2E7A
:202260000BD001694F6C784E3E40DBB21F04C0239B023B4033434B640121009B1B78002BCF
:2022800001D00122FFE70069436C1C40D2B212011540254345640800C0B2F2BD80B5036929
:2022A00001229B6C1B091340DBB2002B01D100201BE00269926C120C9207920FD2B2002A69
:2022C00005D0022A09D005D3032A09D00BE0FEF7D1F909E0FEF7BAF806E0FEF7DCFA03E078
:2022E000FEF7C8F900E00020C0B202BDF2B500221100160003699F6C1024E4432740102599
:20230000F6B236012E403E439E64009B5B78052B01D113000CE0009B5B78032B01D10123EC
:2023200006E0009B5B78072B01D1022300E0FF231E00F6B2FF2E0BD001698F6C974E3E4088
:20234000DBB21F04C0239B023B4033438B640121009B1B78002B01D00122FFE70069836CC0
:202360001C40D2B212011540254385640800C0B2F2BD80B5036901221B6E1B091340DBB24A
:20238000002B01D100201BE00269126E120C9207920FD2B2002A05D0022A09D005D3032A55
:2023A00009D00BE0FEF766F909E0FEF74FF806E0FEF771FA03E0FEF75DF900E00020C0B2FA
:2023C00002BDF2B500221100160003691F6E1024E44327401025F6B236012E403E431E660C
:2023E000009B5B78052B01D113000CE0009B5B78032B01D1012306E0009B5B78072B01D184
:20240000022300E0FF231E00F6B2FF2E0BD001690F6E624E3E40DBB21F04C0239B023B4007
:2024200033430B660121009B1B78002B01D00122FFE70069036E1C40D2B2120115402543D6
:2024400005660800C0B2F2BDFFFFFCFF7CB505000C0029690120496E0A0901001140C9B263
:20246000002901D1002037E0002600962869406E000C8007800FC0B2002805D002280FD095
:2024800008D3032812D017E069462800FDF7A4FE060011E069462800FDF732FE06000BE00D
:2024A00069462800FDF7A8FE060005E069462800FDF792FE0600FFE72869406E000A8106A9
:2024C000890EC9B2491C022900D20221009800F0D8FB20603000C0B276BDF3B501000022EA
:2024E000100016000C69656E10239D431023F6B236011E402E436666019C6478012C01D136
:2025000014000CE0019C6478002C01D1012406E0019C6478022C01D1022400E0FF24250072
:20252000EDB2FF2D0BD00869466E1C4D3540E4B22604C024A40234402C43446601200400F6
:20254000E4B2002C18D0019CA488A41E3F2C12D2019CA5886D1E0C69666E0096009F104EC6
:202560003E400096009EEDB22F02FC25AD013D403543656600E01000019C2478002C01D024
:202580000122FFE709694C6E1025AC43D2B21201134023434B66C0B2F6BD0000FFFFFCFFC3
:2025A000FFC0FFFF0020704700B50978002901D0012100E000210069826E10239A43C9B250
:2025C00009011023194011438166012000BD80B50269D26E13091A00D207D20FD2B2002ACE
:2025E00001D1002001E0FEF7F0FA02BD00B50978002901D0012100E000210069C26E10234B
:202600009A43C9B20901102319401143C166012000BD80B50269126F13091A00D207D20F62
:20262000D2B2002A01D1002001E0FEF7CEFA02BD00B50978002901D0012100E000210069E1
:20264000026F10239A43C9B209011023194011430167012000BD80B502698023D2581309C5
:202660001A00D207D20FD2B2002A01D1002001E0FEF779FA02BD00B50978002901D001218C
:2026800000E0002100698022825810239A43C9B2090110231940114380228150012000BD8E
:2026A00080B502698423D25813091A00D207D20FD2B2002A01D1002001E0FEF754FA02BD36
:2026C00000B50978002901D0012100E0002100698422825810239A43C9B20901102319409D
:2026E000114384228150012000BD80B502699423D25813091A00D207D20FD2B2002A01D140
:20270000002001E0FDF7FCFC02BD00B50978002901D0012100E0002100699422825810238E
:202720009A43C9B2090110231940114394228150012000BD80B502699C23D25813091A0033
:20274000D207D20FD2B2002A01D1002001E0FDF753FD02BD00B50978002901D0012100E009
:20276000002100699C22825810239A43C9B209011023194011439C228150012000BD406AAB
:20278000086001207047806A086001207047C06A08600120704780B501220269A023D258B5
:2027A000120C5207520FD2B2002A0BD0022A0FD00BD3042A12D00ED3062A15D011D3072AB4
:2027C00012D014E0FFF7DBFF12E0FFF7DCFF0FE0FFF7DDFF0CE0FDF7D7FF09E0FDF7BDFE81
:2027E00006E0FEF7DFF803E0FDF7CEFF00E00020C0B202BD10B50200012318004978042961
:2028000045D0062934D0082950D0372904D0382911D039291DD058E000231169A0228A58E1
:20282000BA4C1440DBB21B04E022D2021A402243A023CA504AE01169A0228A58B34C144085
:20284000DBB21B04E022D2021A402243A023CA503CE002231169A0228A58AC4C1440DBB222
:202860001B04E022D2021A402243A023CA502DE003231169A0228A58A44C1440DBB21B0486
:20288000E022D2021A402243A023CA501EE004231169A0228A589D4C1440DBB21B04E02298
:2028A000D2021A402243A023CA500FE005231169A0228A58954C1440DBB21B04E022D202BC
:2028C0001A402243A023CA5000E00020C0B210BD80B501220269A423D258120C5207520F91
:2028E000D2B2002A0BD0022A0FD00BD3042A12D00ED3062A15D011D3072A12D014E0FFF77F
:202900003EFF12E0FFF73FFF0FE0FFF740FF0CE0FDF73AFF09E0FDF720FE06E0FEF742F807
:2029200003E0FDF731FF00E00020C0B202BD10B50200012318004978042945D0062934D026
:20294000082950D0372904D0382911D039291DD058E000231169A4228A586C4C1440DBB24B
:202960001B04E022D2021A402243A423CA504AE01169A4228A58654C1440DBB21B04E022C3
:20298000D2021A402243A423CA503CE002231169A4228A585D4C1440DBB21B04E022D202E1
:2029A0001A402243A423CA502DE003231169A4228A58564C1440DBB21B04E022D2021A4050
:2029C0002243A423CA501EE004231169A4228A584E4C1440DBB21B04E022D2021A4022433B
:2029E000A423CA500FE005231169A4228A58474C1440DBB21B04E022D2021A402243A423CE
:202A0000CA5000E00020C0B210BD10B501231A000269C0241259120C1340DBB2002B02D0A5
:202A2000012B03D005E0FEF7E9FB03E0FEF7BEFB00E00020C0B210BD10B502000123180006
:202A400049780E2910D010291CD100231169C0228A587A4C1440DBB21A0480235B021A40F8
:202A60002243C023CA500EE01169C0228A58734C1440DBB21A0480235B021A402243C02368
:202A8000CA5000E00020C0B210BD10B501231A000269C4241259120C1340DBB2002B02D021
:202AA000012B03D005E0FEF7A9FB03E0FEF77EFB00E00020C0B210BD10B502000123180006
:202AC00049780E2910D010291CD100231169C4228A585A4C1440DBB21A0480235B021A4094
:202AE0002243C423CA500EE01169C4228A58534C1440DBB21A0480235B021A402243C423FC
:202B0000CA5000E00020C0B210BD0000FFFFF8FF80B50269CC23D25813091A00D207D20FBE
:202B2000D2B2002A01D1002001E0FEF71CF802BD00B50978002901D0012100E00021006990
:202B4000CC22825810239A43C9B20901102319401143CC228150012000BDF0B5059D069EB0
:202B6000079F089C016042608360C56006614761216881616168C161A168016200210A0004
:202B80000AE00A00D2B29200A218D2680B00DBB29B00C3185A62491C0A00D2B2032AF0D38A
:202BA000F0BD38B503000C0011002000C0B23F2801DB00200DE00020214A2500EDB2ED003D
:202BC0005559002D04D01800E4B2E300D2589047C0B232BDF8B50B0015001900C9B23F298A
:202BE00001DB002029E000242100154A1E00F6B2F60096197668002E1DD029000500114841
:202C00006F688026B8511048AE6830660F482F688026B8512800DBB2DB00D2185268904782
:202C2000010020006A688023D0502000AA6810662868802284500800C0B2F2BDFFFFFEFF0C
:202C40002C97010052455355202096194B4D4352F446002804D4494200F013F8404260476C
:202C60004042002905D45FD000F00BF8404249426047494200F005F84942604703460B43B9
:202C8000E6D40022030A8B420BD203098B4219D243088B422ED2411A00D201465241104668
:202CA0007047FF2209023FD012068B4205D3121209028B4201D31212090203098B4219D3A1
:202CC00000E0090AC3098B4201D3CB01C01A524183098B4201D38B01C01A524143098B421C
:202CE00001D34B01C01A524103098B4201D30B01C01A5241C3088B4201D3CB00C01A52417D
:202D000083088B4201D38B00C01A524143088B4201D34B00C01A5241884200D3401A524161
:202D2000CFD201461046704708B500F001F808BD7047010000B501000020C9B2002905D02C
:202D4000022907D004D3032906D006E0102004E0182002E0282000E04820C0B200BD70B5A0
:202D60000E0001680C0080340025290029000068C9B2002919D0022909D00FD303291BD1B2
:202D8000C02109014058400E8507AD0F14E0C02109014058800D8507AD0F0DE0C0210901F6
:202DA0004058C00C8507AD0F06E0C02109014058000C8507AD0FFFE72800C0B2FFF7BAFF7B
:202DC0000100C9B2890830002A00D2B2002A05D1C9B280B241438800201832E02A00D2B257
:202DE000012A0ED1C9B2020092B251430D0080B21521FFF743FF4000290008188000201886
:202E00001FE0EDB2022D0ED1C9B2020092B251430D0080B20C21FFF731FFC0002900081816
:202E2000800020180DE0C9B2020092B251430D0080B20721FFF722FF400029000818800011
:202E4000201870BD00B5010000200A00D2B2002A082A0ED9093A0ED0521E0ED0521E0ED0A9
:202E6000521E0ED0521E0ED0521E0ED0521E0ED00FE008000DE00C200BE0102009E01420D2
:202E800007E0182005E0202003E0302001E04020FFE7C0B200BD80B500231A0089B2FFF7C2
:202EA0005EFF0068000C0007000FC0B2FFF7CAFFC0B202BD00B50023D2B2002A0CD00268FD
:202EC000C023DB03134303604268520F5207C900C908114341600BE00268B14B134003607E
:202EE0004268B04B13408A04AF4911401943416000BD0268AD4B134003600268C9B209043F
:202F0000F0231B030B4013430360704700B502685200520802600268A54B13400360C9B20D
:202F2000002909D00168802212060A43026001688022D2050A43026000BD00B50A00D2B22C
:202F4000002A06D101689B4A0A400260016801600BE0C9B2012908D10168964A0A4002604E
:202F600001688022D2040A43026000BD10B50168803100221300140003E0A300CB181A60F9
:202F8000641C037EDB019C42F7D310BD10B48A4982688023D15001214268136D2024A34324
:202FA000C9B249012024214019431165002180688022815010BC704710B47F4982688023BD
:202FC000D15001214268136D1024A343C9B209011024214019431165002180688022815002
:202FE00010BC7047F0B4049C059D069E079F3F780776016042608360C46005614661F0BC27
:20300000704710B500210A008160016141618161C160C16141628162C1620162012202705E
:203020000A00C2700A0002710022D24342638263C26302640B00442403550B0045240355F4
:203040000B00C82403550823462403550B0005E01C00E4B2A4000419A2645B1C1C00E4B2A2
:20306000202CF5DB0A0042700A0082700A003023C2540A00C923C2540A00CA23C2540A00E6
:20308000CB23C2540A00D523C2540A00D423C2540A00D623C2540A00D723C2540A00CC23D1
:2030A000C254D022815010BD30B500210A0003681C683F4D2540D2B292078024E40522406E
:2030C0002A431A60026813683C4C1C40C9B2090780235B05194021431160016809680A0E92
:2030E0001100C907C90FC9B20029F6D130BD38B50400206801250068000D2840C0B20028A9
:2031000013D0002021680A6852005208C0B2C0071043086002E02000FFF74EFF20680068DC
:20312000000D2840C0B20028F5D1280021680A68234B1340C0B2400680229204104018433B
:20314000086020680068400E2840C0B20028F8D1280021680A68164B1340C0B2800780228C
:20316000D205104018430860280021680A68134B1340C0B20007802252051040184308600C
:2031800020680068000E2840C0B20028F8D020680068C00E2840C0B20028F1D031BD0000F8
:2031A000FFFF9FFFFFFF03E00000FC1FFFFFF0FFFFFFFFBFFFFFFFF052455355FFFFFFEFB6
:2031C000FFFFFFFDF0B593B007000C0015002900C9B289B23800FFF7C2FD0600227A6168AE
:2031E0003000FFF767FEA17A3000FFF782FEE17A3000FFF78BFE617A3000FFF79EFE207B41
:20320000002805D0684605706946380000F0A8FD607A012807D120693968EDB2AA00891823
:2032200088221201885013B0F0BD0000F8B504000E00002500202000FFF7A8FE0127390068
:203240002068026852005208C9B2C9071143016020680068010D38000840C0B20028F7D0F1
:20326000327821684B686D481840D2B2520380239B011A4002434A602000FFF738FF3A0073
:2032800021680B6866481840D2B2D20580231B041A4002430A603A0021684B6B614818408C
:2032A000D2B2120780235B051A4002434A632000FFF75CFE3020305CFFF73CFD010008009E
:2032C000C0B2002807D080208000C9B2FFF7D9FC0500207E4543206801687F229143EDB2E7
:2032E0006A06520E0A430260380021680A6D52005208C0B2C007104308654B49B06843186B
:203300002068056D494A2A409BB25D05484B2B4013430365F06843182068056D454A2A40A5
:203320001D04F8235B032B4013430365306943182068056D404A2A409BB29D02FC231B02C0
:203340002B4013430365706943182068056D3B4A2A409BB25D01F8239B002B40134303659D
:20336000B06943182068026D1F25AA439BB2DB06DB0E13430365F078002861D03B00226856
:203380001568D7482840DBB25B078025AD052B4003431360337922681568D2482840DBB2FD
:2033A000DB0380252D022B4003431360306C226890644420335C20680568CB4A2A40DBB229
:2033C0001D02C0239B002B40134303604520335C2068456BC54A2A40DBB21D06F0231B05A4
:2033E0002B4013434363C820305C012840D1002210004623F35CC0B2984239D21000C0B2F5
:2034000080003018836C15002068EDB2AD004519882000012B50521CEAE700BFFFDFFFFFB0
:20342000FFFF7FFFFFFFFFEFFFFF0000FFFF1F800000E07FFFFFE0FFFF03FFFF1FFCFFFF34
:20344000002322681568A6482840DBB25B078025AD052B4003431360002322681568A1486F
:203460002840DBB2DB0380252D022B40034313607078002800D16CE1737822681568CE484B
:203480002840DBB2DB0280252D012B40034313603A002068C0231B01C3585B005B08D2B245
:2034A000D2071A43C0231B01C250F06943182268C2481558C24828409BB21D05C14B2B40B8
:2034C0000343BE481350306A43182268BB481558BD4828401D04E023DB022B400343B74830
:2034E0001350736A2268B5481558B84828409BB29D02F823DB012B400343B0481350B06A27
:2035000042182068AD4BC358E025AB4392B25501E0222A401A43A94BC250F06A411820681F
:20352000A64A825807239A4389B24907490F1143A24A81503020315C00232068C022120149
:203540008258DBB2002B1FD0022B0BD013D3032B23D1C44B1340C9B24906C022D2040A40AC
:203560001A431AE0C04B1340C9B28905C02212040A401A4311E0BD4B1340C9B2C904C02278
:2035800052030A401A4308E0B94B1340C9B20904C02292020A401A43FFE7C02109014250E8
:2035A0003020315C3B002068C02212018258DBB2002B1FD0022B0BD013D3032B23D1A94BF1
:2035C0001340C9B24906C022D2040A401A431AE0A54B1340C9B28905C02212040A401A438A
:2035E00011E0A24B1340C9B2C904C02252030A401A4308E09E4B1340C9B20904C022920252
:203600000A401A43FFE7C021090142503020315C02232068C02212018258DBB2002B1FD0A0
:20362000022B0BD013D3032B23D18E4B1340C9B24906C022D2040A401A431AE08A4B134003
:20364000C9B28905C02212040A401A4311E0874B1340C9B2C904C02252030A401A4308E09E
:20366000834B1340C9B20904C02292020A401A43FFE7C021090142503020315C0323206896
:20368000C02212018258DBB2002B1FD0022B0BD013D3032B2CD1734B1340C9B24906C022DE
:2036A000D2040A401A4323E06F4B1340C9B28905C02212040A401A431AE06C4B1340C9B256
:2036C000C904C02252030A401A4311E0684B1340C9B20904C02292020A401A4308E000BFFC
:2036E000FFFFFFDFFF7FFFFFFFFCFFFFFFFFFFF0C02109014250CA20325C2068C021090124
:203700004358AA491940D2B2D20380231B021A400A43C02109014250CB20325C2068C021A3
:2037200009014358A2491940D2B21302F82252011A400A43C02109014250B2782068436B16
:203740009C491940D2B2120380235B011A400A434263706B21680861B06B21684861F06BD2
:2037600021688861C820325C2068036892491940D2B2120480235B021A400A430260C920AE
:20378000305C002824D00022206803688B491940D2B2520480239B021A400A4302603A00E2
:2037A0002068436883491940D2B2120380235B011A400A43426023E0FFF7FFFF040C0000C9
:2037C000FFFF0FC00000F03FFFFFF8FFFF83FFFF3A002068036879491940D2B252048023B3
:2037E0009B021A400A43026000222068436871491940D2B2120380235B011A400A434260DA
:20380000D420305C002835D03A00206803686C491940D2B292058023DB031A400A4302601B
:203820003A002068036867491940D2B292068023DB041A400A4302603A00206803686249D3
:203840001940D2B292048023DB021A400A430260380061698A6C01239A43C0B20740174360
:203860008F6434E0FFFFFFF9FFFF3FFFFFFFE7FFFFFFFCFF00210B002268156850482840FF
:20388000DBB29B058025ED032B40034313600B00226815684B482840DBB29B068025ED0471
:2038A0002B40034313600B002268156846482840DBB29B048025ED022B400343136060692F
:2038C000826C01239A43C9B20F4017438764D520305C21680A68374B1340C0B20003802282
:2038E0005201104018430860D620305C21684A682E4B1340C0B2C003802212021040184343
:203900004860D720305C21684A68304B1340C0B280038022D201104018434860002723E08C
:203920002A00D2B2D02030583900C9B21423594341182000FFF746FC6D1C2A0092B2D02042
:2039400030583900C9B214235943435AD020305884463900C9B21420414360464018408847
:2039600018188242DCDB7F1C3800CC21715CC0B2884208D20020D02030583900C9B2142277
:203980005143455AD9E7200000F06EF92000FFF78BFB002021680A680D4B1340C0B2C00524
:2039A00080221204104018430860F1BDFF7FFFFFFFE0FFFFFFEFFFFFFFFFFEFFFFFFFDFF54
:2039C000FFFFBFFFFFFFFFFBFFFFFBFFFFBFFFFFFFFF7FFF80B5097889B2FFF7C0F90168FA
:2039E000C02212050A43026001BDF8B506000C00217889B23000FFF7B2F905000835217822
:203A000089B23000FFF747FA00210A000A001BE01600F6B23340032B15D12B681600F6B23E
:203A2000A619367A1E432E602D1D0CE01600F6B21E40022EECD12B681600F6B2A619367A29
:203A400036021E432E60521C1300DBB283421BD203231E00324209D129602B681600F6B213
:203A6000A619367A36061E432E60ECE71600F6B21E40012EDAD12B681600F6B2A619367A23
:203A800036041E432E60DEE7F1BDF8B506000C00217889B23000FFF762F905002868000CD5
:203AA0000007000FFFF7CEF9482160542868400D0100C907C90F281DC9B2002904D001686A
:203AC000C900C908616004E00168890C4905490D6160051D217889B23000FFF7DCF9002132
:203AE0000A0012E02A680B00DBB2E3181A722D1D0AE00B00DBB21A40022AF3D12A68120A55
:203B00000B00DBB2E3181A72491C0A000300D2B2DBB29A4216D203221300194206D12A6843
:203B2000120E0B00DBB2E3181A72EDE70B00DBB21340012BDDD12A68120C0B00DBB2E3186A
:203B40001A72E1E730688068F1BD30B500231A000A78D506ED0E01242200AA400D78402D46
:203B600011DB0221006800290AD0022904D005D3032907D1026705E0426703E0C26201E011
:203B80000263FFE723E00978202910DB0068002C0AD0022C04D005D3032C07D1026705E085
:203BA000426703E0C26201E00263FFE70FE00068002B0AD0022B04D005D3032B07D1026785
:203BC00005E0426703E0C26201E00263FFE730BD30B5002213000B78DD06ED0E0124230074
:203BE000AB400D78402D12DB0221006800290AD0022904D005D3032907D1026F05E0426F8B
:203C000003E0C26A01E0026BFFE71A4026E00978202911DB0068002C0AD0022C04D005D303
:203C2000032C07D1026F05E0426F03E0C26A01E0026BFFE71A4011E01100006800290AD06C
:203C4000022904D005D3032907D1026F05E0426F03E0C26A01E0026BFFE71A40002A01D0EA
:203C6000012000E0002030BD10B5017E032937D10021C9430A0002240368002C0AD0022CC2
:203C800004D005D3032C07D11A6705E05A6703E0DA6201E01A63FFE70A0001240368002C21
:203CA0000AD0022C04D005D3032C07D11A6705E05A6703E0DA6201E01A63FFE70022006835
:203CC000002A0AD0022A04D005D3032A07D1016705E0416703E0C16201E00163FFE73EE0BF
:203CE000017E022925D10021C9430A0001240368002C0AD0022C04D005D3032C07D11A67F5
:203D000005E05A6703E0DA6201E01A63FFE700220068002A0AD0022A04D005D3032A07D12F
:203D2000016705E0416703E0C16201E00163FFE715E0017E012912D10021C9430022006825
:203D4000002A0AD0022A04D005D3032A07D1016705E0416703E0C16201E00163FFE710BD8F
:203D600030B500231A000A78D506ED0E01242200AA400D78402D19DB02210068002910D01E
:203D8000022906D009D303290FD1816E0A4382660BE0C16E0A43C26607E0416A0A43426204
:203DA00003E0816A0A438262FFE733E00978202918DB0068002C10D0022C06D009D3032CCB
:203DC0000FD1816E0A4382660BE0C16E0A43C26607E0416A0A43426203E0816A0A438262CE
:203DE000FFE717E00068002B10D0022B06D009D3032B0FD1816E0A4382660BE0C16E0A43FB
:203E0000C26607E0416A0A43426203E0816A0A438262FFE730BDF9B58FB00D00179900205B
:203E200001200490012003900820009003230293022414240C94784C0B94FA24A4050A94E0
:203E4000C9B2002909D1754909915E2608931F217118491C0791069008E07049099126268A
:203E6000089307217118491C079106900192019800F0DEF8059001240D952EE0280000F0EF
:203E8000E7F80100380000F0EEF80700019800F0CFF80100380000F070F98021090400F0AD
:203EA000C5F939D8019800F0C3F80100380000F064F901000798A8420EDB059800F0B6F9BA
:203EC0000AD80494009505910C98A84204DB08000B9900F0BFF927D3641C0998A04223DB81
:203EE0000D9800F0A5F80500200000F0B1F80100280000F0B8F80700019800F099F80100E7
:203F0000380000F0B0F800F0B9F90500002D02D006988542B2DA07E0019800F089F8390010
:203F200000F02BF90100C5E710A80488200080B200F07EF80A9900F0BEF905000098B042EB
:203F400000DA009E0CE0380000F082F8290000F081F904D20296380000F07AF80500761E27
:203F60000898864216DB3000401C2D4948430099FEF784FE210089B2411A012903DB21006B
:203F800089B2471A02E0210089B20F1A210089B28842D8DA00980299401A401E0190214C5D
:203FA0000125169E1DE0310089B20F1A0CE01C4868430099FEF762FE310089B2411A0129BB
:203FC000F1DB310089B2471A380000F041F8210000F040F904D20395380000F039F80400D2
:203FE0006D1C0198A842E2DA0F9C04982060029800F0CAF90CA20CCA00F0D0F900F090FA2E
:20400000A0600298A168401AE060019820610398606011B0F0BD0000CDCCCC3DFF030000DC
:204020001027000000401C46333333333333E33F9D2102000AD002D4491E9218FCD5C90533
:20404000100A1206524100D3012A4841704700009D210200EED55242F446FFF7EBFF012209
:20406000D2071043604730B405004D400122D20715404B180418240E25D01B0E2CD0FF2CB0
:2040800031D0FF2B34D0E41A000209021043114343084808D10D1B1A02D2641EDB181B1815
:2040A000DB18834200D31B1A4941F9D37F3423DDFF2C05DAE40548086041284330BC704745
:2040C000FF20C005F9E728001B0E03D0FF2BF5D14902F3D0D043F1E7FF2C01D14002F9D106
:2040E000FF20C005E9E74002F4D1FF2BF8D1F1E728004902E2D0EDE70B0200202442DCD101
:204100005B129B1CD9D9D805D7E70122D20703004B402ED4431A01D2C01AC91830B44B1870
:204120000418240E1B0E22D0FF2C20D0E31A182B1DDC09021143C40D641E000210439446E1
:204140001925ED1A0A00AA40D940451801D36D08A41CE405D209280A2D062A436546AA417B
:20416000604103181B0EFF2B01D3C00DC00530BC7047514006E05140CCE70122D20703006D
:204180004B40F8D4431A03D2C01AC9185040514030B44B18090211430418240E1B0E40D08D
:2041A000FF2C3AD025009D410BD31ED8C50D4002401A0BD3ED050100400AC9059141684121
:2041C000D5E7C50D40024918401AD0D001214008491C0018FCD58C4204D36D1A000AED05D4
:2041E0004019C4E7E8051040C1E7182DBFDCAC1C0D00E140E5414D40012D4941C40D0002C2
:204200001043451A01D46D199543641EE405280A2D069541604130BC7047FF2BA7D1D84312
:20422000A5E72442A3D10020A1E7FEE70CB4012212060318DA4207D84B18DA4204D802001D
:204240000A43921802D281420CBC7047FCD088420CBC70470CB4012212060318DA4207D82B
:204260004B18DA4204D802000A43921802D288420CBC7047FCD08142FAE7FEE70122D2077C
:204280000118090E7F3910D449421F310FD4001805D2C0011043C84000D5D0437047C00129
:2042A0001043C84005D440427047002070470042F3D51000704730B405004D400122D20777
:2042C00015404B180418240E2ED01B0E32D0FF2C34D0FF2B3AD0E41800020902104311439C
:2042E000000A090A9446C2B24A43000AC3B24B43000A4843110A5B181A43D2B2190A091871
:2043000001D44918641E080A7F3C23DBFE2C08DAE40509061143634699416041284330BC47
:204320007047FF20C005F9E728001B0EFF2BF6D1D043F4E72800FF2CF1D1F9E74002F7D1D3
:20434000FF2B01D14902F3D1E005E7E7D8054902E4D0EDE743020020641CDFD15B129B1C36
:20436000DCD9D805DAE7FEE7010042221201D21E004207D002D4521E0018FCD5C10A400545
:2043800012058918704700000100EED54042F446FFF7EBFF0122D20711436047F0B50E00A4
:2043A0005E400125ED072E40B446AE0ADF184C18F44208D2F7420ED2640D01D07F0D12D1F0
:2043C00000206146F0BD05D1F74201D87F0D05D10020C143F0BDFBD1640DF9D00020C14324
:2043E000490549088FE0E419C902DB0229432B43DB0A460DC00231438E4630B487B295B28A
:204400007D432E0CADB2140C7C43A419260C240425439CB27C43A419190C7943270CC91925
:20442000A4B20F043C43090C000C97B247432E0CBE193543ADB2170C4743360CBF19A6B299
:20444000BF193E043543240C3E0C36199FB24743BF19BCB23E0C89191F0C47437F183E0466
:204460003443390C704680B297B247432E0CBE193543ADB2170C4743360CBF19A6B2BF19E6
:204480003E043543240C3E0C36199FB24743BF19BCB23E0C89191F0C47437F183E04344387
:2044A000390C77463F0C90B278432E0C80190604ADB22E43050CA0B22D18120C7A43501919
:2044C000020C80B2240CA4189AB27A43121914042043120C89181B0C7B43C91830BCEF0A97
:2044E000394203D1B61940414941641E6F12BF0DE41B0BDBFF19BC4211DA24050027420844
:20450000AE417841614166463143F0BD641C05D1401C6141CF0201D34908F4E750E75DE7E4
:204520004A1812D2400DC90208430121C9070843520D40210901521A521C06D452421F3232
:2045400001D4D0407047C017704700207047FEE700B50100C9B2802900DB7F20C0B200BDF2
:2045600000B50100C9B2F139092901D2012004E00100C9B2802900DB0020C0B200BDFEB5D4
:204580000400002528006E463F2030703078F0270F430740377072701800C0B2FFF7D8FFDF
:2045A000B070207800280FD0032003E00100C9B27554401C0100C9B20829F7DB082269463D
:2045C000E068A36D984704E003226946E068A36D984740B2FEBD7CB50300002001000100B2
:2045E00069460F220A700A78DC8AF025254315400D70020008E01C691500EDB2645D150031
:20460000EDB24D196C70521C1400E4B2DD8AA4B2AC42F0D31A78002A15D0020006E0140096
:20462000E4B2DD8A64190C196070521C1400E4B20725DE8AAD1BAC42F1DB08226946D868C4
:204640009B6D984706E0DA8A521CD2B26946D8689B6D984740B276BD1CB5040068461F2179
:2046600001700178E28A92B2120AF02313430B400370E18A417000210A00D2B2C9B208E02F
:2046800022690B00DBB2D25C0B00DBB2C3189A70491C0A00D2B2062AF2DB08226946E0683B
:2046A000A36D9847010049B2002904D1218B891D21830121A17640B216BDFEB50400002541
:2046C0002800C0B268462F2101700178A27EF02313430B400370E18A228B8E1A310089B2E5
:2046E000082900DB07262900C9B20AE02269238B0F00FFB2DB19D25C0B00DBB2C3185A709B
:20470000491C0A00D2B2330092B29BB29A42EDD3217800291AD02900C9B22900C9B207E06B
:204720000A00D2B233009BB2D21882185570491C0A00D2B207233700BFB2DB1B9A42EFDBC1
:2047400008226946E068A36D984706E03200521CD2B26946E068A36D9847010049B2002934
:2047600009D1218B89192183A17E491CA176A17E102900DBA57640B2FEBD70B5030000208F
:2047800004000F240D782600354205D0D2B2521E0D782540AA4208DA586D002802D099489F
:2047A000596D88470620C04315E00A78144042229C5208E00200D2B28A185278DC6B0500F8
:2047C000EDB26255401C0200D2B242241C5B92B2A242EFD3002070BD38B503000020040079
:2047E000D2B2082A08D0586D002802D08648596D88470620C04339E00A781202F0242401F8
:2048000014404A78A2181400A4B2082C08DA586D002802D07D48596D88470620C04325E001
:2048200040241C5B1500ADB2AC4208D2586D002802D07748596D88470220C04316E04224CD
:204840001A5308E00200D2B28A189278DC6B0500EDB26255401C0200D2B2062AF2DB06202A
:2048600044215852012046215854002032BDF8B50300002528004620185C0C782407240F2D
:20488000A04202D00320C0433EE04220185A44241C5B041B200080B2082800DB0724D2B242
:2048A000521E200080B2824208DA586D002802D05848596D88470620C04325E02A000BE059
:2048C000D86B1600F6B24427DF5BF6191700FFB2CF197F788755521C1000C0B2260080B258
:2048E000B6B2B042ECD34420185A0019442158524620185C401C462158544620185C102846
:2049000001DB46201D540020F2BD80B50100D2B2032A08DA486D002802D03F48496D884791
:204920000620C04300E0002002BD80B513009BB20A00C16800F001F802BDF8B50400002549
:204940002800002C02D10020C04359E0A08A190089B2884208D2606D002802D0C048616D15
:2049600088470220C0434BE03420205C012808D1606D002802D0BB48616D88470120C043BB
:204980003EE0E38228002083280007E00100C9B2515C26690700FFB2F155401C0100C9B22C
:2049A0001E0089B2B6B2B142F0D3E08A082804DA2000FFF710FE060020E02000FFF74CFE7E
:2049C0000600300040B2002818D12800A0832800A0772800E077E06D80472200203203C248
:2049E000083AE06D80470022643051412200283203C2083A2563012034216054300040B2C2
:204A0000F2BD0000D0AB0100FCAB010058AA010090AA010028AC010048AC0100FEB51400F4
:204A20001A001300DBB29B1E072B00D317E100252B00DBB22B00DBB2029408E0029C1E0037
:204A4000F6B2A45D6E461F00FFB2F4555B1C1C001600E4B2F6B2B442F0D32B00DBB207E0A1
:204A60006C461E00F6B21700FFB2F619A5555B1C1C00E4B208261700FFB2F61BB442EFDBFD
:204A80006F4604000E003878C0B20009002806D0022858D01BD3032800D19DE0DFE051203D
:204AA000205C012804D10520C0435021605401E050202554D2B269462000FFF75EFE40B2CE
:204AC000002803D1A663022051216054C7E05120205C012804D10520C0435021605401E0C9
:204AE00050202554D2B269462000FFF775FE01000222D24349B291420CD10720C043502191
:204B00006054512025540023002202212000FFF736FDA4E040B2002814D1A6630120512127
:204B2000605460784721605401234720225C00212000FFF724FDE06D804700226430514110
:204B4000A064E1648BE05120205C012804D00520C0435021605482E0A06B864200D07EE007
:204B6000D2B269462000FFF782FE0321C94302000B0052B29A4204D15020215451202554AB
:204B80006DE040B2002826D1E06D8047002264305141A064E1644420205A4221615A88424C
:204BA00003D302205121605415E06078002812D04720205C401E472160544720205C002898
:204BC00009D160784721605401234720225C00212000FFF7D4FC42E03420205C01283ED1CD
:204BE000D2B269462000FFF790FE40B2002835D1E06D80470022643051412200283203C221
:204C0000083A0F2039780140022906D10720C043206302203421605420E03978014001293B
:204C20000CD1E07F401CE077E07F022816DB0620C04320630220342160540FE03978014251
:204C40000CD17878002802D18048A08301E07878A083B878FFF784FCA077E577FFE7F7BDFA
:204C600038AB01006CAB010070B5002425005125455D022D02D00420C04325E0856B8668A7
:204C8000B54201D1012500E025000D704221415A1D000E00ADB2B6B2B54200D219002300AE
:204CA00007E0C56B1E00B6B2AD5D1E00B6B295555B1C1D000E00ADB2B6B2B542F1D3049A1B
:204CC000118051214454002070BD70B402000B0018781070587850705868506098689060BB
:204CE000D868D06018691061988A908200242000D08220001083200090762000908320005C
:204D000090772000D077002000211500203503C5083D1500283503C5083D146325003426F8
:204D200095559D69D5639D8B40269553250042269553250044269553250046269555250049
:204D4000472695559064D16420005021505451201454186A5065586A9065986AD06570BC74
:204D6000704738B504003420205C012856D1374DA08BA84202D0A08B00283DD0A07F002859
:204D80000ED0A07F002837D0E06D8047220020320CCA121A8B41002B2EDC01DB002A2BD259
:204DA0002000FFF78AFC40B2002822D1A08BA84202D0A08B4019A083E06D804700226430F2
:204DC00051412200283203C2083AE06D804702000B00A07F0021801859412200203203C2F2
:204DE000083A208BE18A884206D300203421605402E0022034216054E06D804722002832F2
:204E00000CCA121A8B41002B08DC01DB002A05D20120C04320630220342160545120205C19
:204E2000012811D1E06D8047A26CE36C121A8B41002B09DC01DB002A06D20220C04350217A
:204E4000605400205121605431BD0000FFFF000000B5BFF34F8F054805490860BFF34F8F94
:204E600000BFFDE701604260836070470400FA050CED00E038B504002F48A2688023D050E1
:204E8000C9B200295AD0022900D17FE06AD3042900D1A3E000D28DE0062900D1C6E000D274
:204EA000B0E0082900D1E9E000D2D3E00A2900D10CE100D2F6E00C2900D12FE100D219E197
:204EC0000E2900D152E100D23CE1102900D175E100D25FE1122900D198E100D282E114293F
:204EE00000D1BBE100D2A5E1162900D1DEE100D2C8E1182900D101E200D2EBE11A2900D1FC
:204F000024E200D20EE21C2900D147E200D231E21E2900D172E200D258E2202900D19DE294
:204F200000D283E2222900D1C8E200D2AEE2232900D1DBE2DDE200BF524553550120010059
:204F4000A26853680125AB43C9B20140194351600021A26853680125AB43C9B20840184397
:204F60005060C6E201200100A26893680125AB43C9B20140194391600021A2689368012549
:204F8000AB43C9B2084018439060B2E201200100A268D3680125AB43C9B201401943D160BD
:204FA0000021A268D3680125AB43C9B208401843D0609EE201200100A26813690125AB43ED
:204FC000C9B20140194311610021A26813690125AB43C9B20840184310618AE2012001006F
:204FE000A26853690125AB43C9B20140194351610021A26853690125AB43C9B208401843F4
:20500000506176E201200100A26893690125AB43C9B20140194391610021A26893690125F4
:20502000AB43C9B208401843906162E201200100A268D3690125AB43C9B201401943D16169
:205040000021A268D3690125AB43C9B208401843D0614EE201200100A268136A0125AB4399
:20506000C9B20140194311620021A268136A0125AB43C9B20840184310623AE2012001001B
:20508000A268D36A0125AB43C9B201401943D1620021A268D36A0125AB43C9B208401843D0
:2050A000D06226E201200100626813680125AB43C9B2014019431160002162681368012526
:2050C000AB43C9B208401843106012E201200100626853680125AB43C9B2014019435160DC
:2050E0000021626853680125AB43C9B2084018435060FEE101200100626813690125AB43CD
:20510000C9B20140194311610021626813690125AB43C9B2084018431061EAE1012001000E
:20512000626853690125AB43C9B20140194351610021626853690125AB43C9B20840184332
:205140005061D6E101200100626893690125AB43C9B20140194391610021626893690125D4
:20516000AB43C9B2084018439061C2E1012001006268D3690125AB43C9B201401943D16109
:2051800000216268D3690125AB43C9B208401843D061AEE1012001006268136A0125AB4379
:2051A000C9B201401943116200216268136A0125AB43C9B20840184310629AE101200100BB
:2051C0006268936A0125AB43C9B201401943916200216268936A0125AB43C9B208401843CF
:2051E000906286E1012001006268136B0125AB43C9B201401943116300216268136B0125BD
:20520000AB43C9B208401843106372E1012001006268536B0125AB43C9B201401943516332
:2052200000216268536B0125AB43C9B20840184350635EE1012001006268136C0125AB4322
:20524000C9B201401943116400216268136C0125AB43C9B20840184310644AE10120010064
:205260006268536C0125AB43C9B201401943516400216268536C0125AB43C9B208401843E8
:20528000506436E1012001006268936C0125AB43C9B201401943916400216268936C012527
:2052A000AB43C9B208401843906422E1012001006268136D0125AB43C9B2014019431165DD
:2052C00000216268136D0125AB43C9B20840184310650EE1012001006268136E0125AB434C
:2052E000C9B201401943116600216268136E0125AB43C9B2084018431066FAE0012001000F
:205300006268536E0125AB43C9B201401943516600216268536E0125AB43C9B20840184341
:205320005066E6E0012001006268936E0125AB43C9B201401943916600216268936E0125CF
:20534000AB43C9B2084018439066D2E0012001006268D36E0125AB43C9B201401943D16609
:2053600000216268D36E0125AB43C9B208401843D066BEE0012001006268136F0125AB4379
:20538000C9B201401943116700216268136F0125AB43C9B2084018431067AAE001200100BB
:2053A00062688023D3580125AB43C9B2014019438023D150002162688023D3580125AB4398
:2053C000C9B2084018438021505092E00120010062688423D3580125AB43C9B20140194312
:2053E0008423D150002162688423D3580125AB43C9B208401843842150507AE00120010035
:2054000062689023D3580125AB43C9B2014019439023D150002162689023D3580125AB4307
:20542000C9B2084018439021505062E00120010062689C23D3580125AB43C9B201401943B9
:205440009C23D150002162689C23D3580125AB43C9B2084018439C2150504AE001200100BC
:2054600062689423D3580125AB43C9B2014019439423D150002162689423D3580125AB439B
:20548000C9B2084018439421505032E0012001006268C823D3580125AB43C9B20140194359
:2054A000C823D15000216268C823D3580125AB43C9B208401843C82150501AE00120010008
:2054C0006268CC23D3580125AB43C9B201401943CC23D15000216268CC23D3580125AB4393
:2054E000C9B208401843CC21505002E0FFF7B0FCFFE70020A1688022885031BD0160426003
:20550000704770B50A79002A0DD0022A51D018D3042A00D1BDE000D283E0062A00D128E112
:2055200000D2EEE05DE10021006802691202120A20239A43C9B24901202319401143016132
:205540004FE10123026814692402240A2025AC43DBB25B0120252B402343136100221500DE
:2055600003681C692402240A1026B443EDB22D011026354025431D61150003681C69240231
:20558000240A0826B443EDB2ED000826354025431D61098803689C68240C240489B20C43C1
:2055A0009C600068C168090C090492B21143C16017E10122150003681C692402240A2026C9
:2055C000B443EDB26D012026354025431D6103681C692402240A1025AC43D2B212011025F2
:2055E0002A4022431A610022150003681C692402240A0826B443EDB2ED000826354025432A
:205600001D61098803689C68240C240489B20C439C600068C168090C090492B21143C160C2
:20562000DFE00122150003681C692402240A2026B443EDB26D012026354025431D6100251F
:2056400003681C692402240A1026B443EDB22D011026354025431D6103681C692402240A37
:205660000825AC43D2B2D20008252A4022431A610A8803689C68240C240492B214439C6051
:2056800049880068C268120C120489B20A43C260A7E00122150003681C692402240A202680
:2056A000B443EDB26D012026354025431D61002503681C692402240A1026B443EDB22D01E2
:2056C0001026354025431D6103681C692402240A0825AC43D2B2D20008252A4022431A610C
:2056E0004A8803689C68240C240492B214439C6009880068C268120C120489B20A43C26079
:205700006FE00122150003681C692402240A2026B443EDB26D012026354025431D611500BE
:2057200003681C692402240A1026B443EDB22D011026354025431D6103681C692402240A56
:205740000825AC43D2B2D20008252A4022431A610A8803689C68240C240492B214439C6070
:2057600049880068C268120C120489B20A43C26037E00122150003681C692402240A20260F
:20578000B443EDB26D012026354025431D61150003681C692402240A1026B443EDB22D0111
:2057A0001026354025431D6103681C692402240A0825AC43D2B2D20008252A4022431A612B
:2057C0004A8803689C68240C240492B214439C6009880068C268120C120489B20A43C26098
:2057E000FFE770BDF8B504000D000120030021684E698E4A3240DBB21B04802676023340ED
:2058000013434B612B7821680E68894A32400326B243DBB29B079B0F13430B60697822687C
:205820005368FF26B343C9B219435160A97822685368804E1E40C9B2090231435160EB786A
:2058400021684E687C4A3240DBB21E04FC239B03334013434B602A7921680B691B021B0A0F
:205860000427FF433B400426D2B2920032401A430A610100226810690002000A4023984378
:20588000C9B2890140231940014311612F202A5C6168886920239843D2B2520120231A4070
:2058A00002438A6130202A5C606881691C239943D2B293001C221A400A43826131202A5C5F
:2058C0006068816903239943D2B29207920F0A4382612A7B2168486908239843D2B2D200EB
:2058E00008231A4002434A61A91D2000FFF709FEA97B206842691740C9B289000E403E43CF
:205900004661A87B002809D0687B21684A6903239A43C0B28007800F10434861002135E0E0
:205920000800C0B240002818C37B0A0020681600F6B2B600861980277F00F6590F27BE43DE
:20594000DBB21B071B0F3343D2B2920080188022520083500800C0B240002818067C0A00FD
:2059600023681000C0B28000181880277F00C0594027B843F6B2B60140273E400643D2B2B8
:2059800090001818802252008650491C0800C0B21028C5DB002021684A69244B1340C0B236
:2059A000000480225202104018434861F1BD10B500210A0001221300037004231C0044705B
:2059C000302484700B24C4700C000471C18001810C0084720C0004730C00447382730A0091
:2059E0002F240255302283540A003123C2540A000BE01300DBB25B00C318DA730B00140029
:205A0000E4B2640004192374521C1300DBB2102BEFDB10BD0068C9B289004018C02149000A
:205A200040588004800C80B270470000FFFFFEFFFFFEFFFFFF00FFFFFFFFC0FFF0B502007E
:205A400052B2002A16D41822B94B040064B2A408A4001C59FF25C6001640B540AC43890163
:205A6000C9B2C5002A409140214340B28008800019501BE00F25AF4B1824020052B22A400F
:205A8000083A92089200060076B23540083DAD08AD005D59FF26C7002740BE40B5438901C5
:205AA000C9B2C0000440A14029439950F0BD80B5411E80225204914201D301200EE0401EE4
:205AC0009D49086003210020C043FFF7B7FF0020C34908600720C3490860002002BD10B5B2
:205AE000C14C200000F03AFAC02040002418200000F075FC00F00CF800F06CFD00F01EF924
:205B000000F055F8200000F08EFC00F0EAF910BDF0B585B001246E4620003070022777708B
:205B20002000B080B14D6A4607212800FDF752F8200030702000B0806A4613212800FDF7C9
:205B400049F86A4614212800FDF744F86A4615212800FDF73FF86A4616212800FDF73AF859
:205B60006A4617212800FDF735F82000307077700420B0806A4627212800FDF72BF834701E
:205B80006A4628212800FDF725F8994C220009212800FDF706F82068FA218900FDF771F8FF
:205BA000FFF785FF934800F07FFE05B0F0BD38B58D4C2500E03501220021280000F07DFEEA
:205BC00000220021280000F0B7FE01220121280000F073FE00220121280000F0ADFE0122BD
:205BE0000221280000F069FE00220221280000F0A3FE01220321280000F05FFE0022032103
:205C0000280000F099FE01220521280000F055FE00220521280000F08FFED83401220121E3
:205C2000200000F04AFE00220121200000F084FE01221021200000F040FE00221021200021
:205C400000F07AFE01220F21200000F036FE00220F21200000F070FE31BD80B5C0B20028B8
:205C60000BD002281FD013D3042832D026D3062845D039D307284DD057E00221A74800F04F
:205C800075FE002801D1012000E00020C0B24DE00321A24800F06AFE002801D1012000E076
:205CA0000020C0B242E001219C4800F05FFE002801D1012000E00020C0B237E00021974839
:205CC00000F054FE002801D1012000E00020C0B22CE00521914800F049FE002801D1012098
:205CE00000E00020C0B221E001218D4800F03EFE002801D1012000E00020C0B216E00F215B
:205D0000874800F033FE002801D1012000E00020C0B20BE01021824800F028FE002801D110
:205D2000012000E00020C0B200E0002002BD000000E400E01CED00E014E000E0F8B5A2B091
:205D40007848008869460881774803907748019002A9019800F0A8FF15A8FFF728FE012547
:205D600015A8057085730324210041730026310001730A21C1730B21417415A91A48FFF7DC
:205D800031FD6A4628211948FCF70BFF04A801F0E1F804AF3000387030003871FD7107200F
:205DA000F8702000B87102202C2178542D203C540098C0092821FCF764FFC821FCF761FFDE
:205DC0003881BE815A4C04A9200001F01BF9200001F028F86421019801F004F823B0F0BD97
:205DE00018E000E010E000E0C0300020C830002040500020FFFF000038B54E4C4E4D0021E2
:205E00002800FFF707FE206001212800FFF702FE606000F059F849490A78002A03D0022A61
:205E20003DD027D34FE0020092B2454B9A420CDB44480288521C02800288434B9A4218DBA6
:205E4000002202800120087013E080B23F4A90420CDA3C480288521C028002883A4B9A42B6
:205E600007DB002202800220087002E000203549088028E080B2FA22920190420BDA3148E1
:205E80000288521C028002882F4B9A4206DB002202800A7002E000202A49088013E080B287
:205EA0002B4A90420BDB27480288521C02800288254B9A4206DB002202800A7002E00020F5
:205EC00020490880FFE731BD1A48006821494843000BAF218900401880B2704717480078C2
:205EE000704700B585B0684600F061FA0120694602000A7000224A70CA7003000B714A716C
:205F000088714A72C82080010490FA20800003906946114800F086F905B000BDA0310020C8
:205F200098310020322D0100B8AC01002C3200208431002044500020C0300020A655002081
:205F400075400000A2550020210300003421000029230000D8D6000040320020F0B58BB090
:205F600004007D4D2A007D492000FFF7C7FA7C480590069000200790089009900A90794E54
:205F8000794F05A80390029778480190784800903300784A784920000830FCF7DEFD774923
:205FA0002000383001F03AF9754920003C3001F037F974492000403001F032F97249200086
:205FC000443001F02FF9714A71492000483001F02BF970492000543001F02AF96E492000CA
:205FE000583001F027F96D4920005C3001F024F932006B492000603001F020F90220694627
:20600000087404A80390029501970096594B574A644920008030FCF7E5FF634920009C30CF
:2060200001F004FA2A0061492000A03001F00CFA2A005F492000A83001F009FA5D49200032
:20604000B03001F007FA5C492000B43001F004FA5A492000B83001F001FA59492000BC3091
:2060600001F0FCF957492000C03001F0F9F956492000C43000F0D4FE544A55492000C830DE
:2060800000F018FC534A54492000D03000F012FC524A53492000D83000F00CFC514A524916
:2060A0002000E03000F006FC504A51492000E83000F000FC00962E4B3A004E492000F03046
:2060C00001F0D0F92A004C4980204000201801F00FFA2A00494984204000201801F008FA6A
:2060E000244B224A2449882040002018FEF7BAFE43498E204000201801F026FA4149B2206C
:206100004000201801F02AFA3F49B4204000201801F024FA2A003D49B6204000201800F021
:20612000C0FD3B49BA204000201801F031FA3949BC204000201801F02BFA3749BE20400026
:20614000201801F025FA3549C0204000201800F067F80BB0F0BD00BF00F0054000400240F4
:2061600000127A0000E0064000E8064000F8064000E4064000F0064000F0074000400740E3
:20618000003000400040004000C000400010024000800040009001400080014000500040DB
:2061A0000000024000800340006006400020074000300740007007400050074000000340C5
:2061C0000010034000D00040006002400050034000000640405003400010064080500340A5
:2061E00000200640C050034000300640005103400040064000D007400080054000900540A5
:206200000080074000C0024000D0024000E0054000A0064000B0064000C0064000A00740B5
:20622000016070477FB50400206801260068C2093000104022681268530932001A40236835
:206240001B685D0A33002B40C0B2002800D0ADE0D2B2012A00D0A9E0DBB2012B00D0A5E0A9
:206260000D0010220021684601F0B6F900987049014000912A78684603686E491940D2B2FE
:206280001304E022D2021A400A4302606A786846036869491940D2B2D20380231B021A408F
:2062A0000A430260EA786846036864491940D2B2120380235B011A400A4302606A7968467C
:2062C000016840239943D2B2920140231A400A430260AA796846016820239943D2B2520163
:2062E00020231A400A4302602A7A6846016802239943D2B2520002231A400A430260687AB0
:2063000069460A6801239A43C0B2304010430860AA78684603684A49194092B2920380231B
:20632000DB011A400A4302602A796846016880239943D2B2D20180231A400A430260EA79D9
:206340006846016818239943D2B2D30018221A400A4302603B48216848600099226811602D
:20636000296922689160216809688A0A31001140C9B20029F7D0216809684A0A31001140C5
:20638000C9B20029F7D0697800290FD02E492268516021684860E8682168C86020680068D5
:2063A000410A30000840C0B20028F7D07FBD01210A0002700022130043700B0083701300E6
:2063C000C3701300037113004371817111000172110041721D490161C260C271704700B579
:2063E00002680121126852090A40D2B2012A19D1144A03685A600268126880239A43036807
:206400001A60124A03689A6002681268D20A0A40D2B2002AF8D102681268520A0A40D2B2B2
:20642000002AF8D000BD08490068416070470000846FF8FFFFFFF8FFFF7FFFFFFFEFFFFF55
:20644000FFBFFFFF20C528D902A680B4FFFF0000F8B594B000200020694608704CE001A992
:206460002868FDF772FB42E001AE684600783070964D01A92868FDF7ABFB002837D0D020BE
:20648000205869460978142251434018407A0128E5D101A92868FDF758FB01A92868FDF7EA
:2064A000F4FA4820325C01A801000831884C98204001251828784C2358432018071D3800CD
:2064C00001F0AEF8029829784C225143605028784C214843201844214822B25C4254287855
:2064E000401C28702878202801D30020287068460078401C69460870764C68460078CC21B6
:20650000615C8842B0D315B0F0BD70B50100002420006F4BC14A9D18982252019A5C2E7872
:20652000B24211D04C2228784C26704318180E000100300001F074F82878401C2870287853
:20654000202800D32C700120C0B270BDF0B593B000242300DBB22500EDB2E4B200E0641C4E
:206560005C4D2600CC27EF5DF6B2BE420CD2D026AE59B4462700FFB2142677436646F61909
:206580007668B042EBD123002800D0306C4605681E00F6B214277E43AD5B25704825625582
:2065A0000068DBB214246343C01840680190D2B2684604000834200001F032F8434C69460C
:2065C0002068FDF712FA69462068FDF703FA002013B0F0BDFEB50025029591492A003C4C80
:2065E000200001F02BF8D8212A003A4C2600300001F024F88B4E30008030344908608A4FE4
:2066000001220921380000F058F901220921380000F092F900220921380000F09AF9834FDB
:2066200005220021380000F048F905220121380000F043F92000FCF7E4FC0820CC21605440
:206640007B48D0216050012001002170290061702900A1702900E17030216554C8216054CE
:2066600002AA0B2130000830FCF79BFA607801280BD101200190FA20C00000906D4B6E4AE9
:20668000029920001C30FDF7C6FB002001906B480090684B6A4A029920000830FDF7BBFB46
:2066A00021000A480068FCF7C1FD092000F0FCF8F7BD10B50400FFF711FC002804D108229A
:2066C00021006048FFF742FF10BD000034500020583C00205C4F00207CB505000824210047
:2066E00000226E46300000F0A9FF022001F008F869460978084369460870032001F000F83B
:20670000694609784000084369460870002000F0F7FF69460978800008436946087001204E
:2067200000F0EEFF69460978C000084369460870042000F0E5FF69460978000108436946F7
:206740000870052000F0DCFF694609784001084369460870062000F0D3FF69460978800155
:20676000084369460870072000F0CAFF69460978C00108436946087022006946280000F07B
:206780004FFF73BD30B593B02F4C2000FFF7A4FF20788006800E00280DD02C4D28886421C0
:2067A000FCF76CFA002902D12000FFF782FF2888401C288002E0002024490880062000F02C
:2067C0008FFF002804D1072000F08AFF002802D02000FFF76EFF1D480188FA2292009142A2
:2067E00001DB002101806846FFF78FFE01280FD100981749884203D000981649884207D1B3
:2068000068464421435C021D00991348FEF706F9124801F07AF813B030BD0000011300003E
:2068200004130000C0300020983100209031002050A801004C1D000080841E00C409000016
:2068400020A107000102000038500020A055002031070000DF0700002020002008200020EA
:2068600000B5010049B2002905D40121C006C00E81400B48016000BD00B50A4801680129E3
:2068800006DB0168491E01600068012800DA62B600BD000072B603480168491C016070474D
:2068A00000E100E06450002080B540B2FFF7D8FF01BD7047016042607047F0B51300DBB2DB
:2068C000002B1BD10B0004689D006659194D3540D2B21602E022D20032402A439B00E250D7
:2068E000012200688B00C3580424A343D2B29200042422401A43890042501AE000260C0015
:206900000568A300EB580427BB43F6B2B60004273E401E43A300EE5000688B00C358054C53
:206920001C40D2B21302E022D2001A40224389004250F0BDFFF8FFFF10B443685B690124BA
:206940008C40A343D2B28A401A434068426110BC704710B443681B6801248C40A343D2B2BF
:206960008A401A434068026010BC704710B502000020030052681469012213008B402340DE
:20698000002B00D01000C0B210BD00000068C00FC0B27047026852005208C9B2C907114398
:2069A000016070470268A14B1340C9B20A06FE21C90511401943016070470268A24B13402F
:2069C000C9B20A04FE21C903114019430160704702689E4B1340C9B20A02FE21C901114017
:2069E00019430160704702687F239A43C9B24906490E1143016070474068C00FC0B270470D
:206A0000426852005208C9B2C9071143416070474268864B1340C9B20A06FE21C905114092
:206A20001943416070474268874B1340C9B20A04FE21C90311401943416070474268834BE2
:206A40001340C9B20A02FE21C901114019434160704742687F239A43C9B24906490E1143D0
:206A600041607047C068C00FC0B27047C26852005208C9B2C9071143C1607047C2686B4B71
:206A80001340C9B20A06FE21C90511401943C1607047C2686C4B1340C9B20A04FE21C903FE
:206AA00011401943C1607047C268684B1340C9B20A02FE21C90111401943C1607047C26802
:206AC0007F239A43C9B24906490E1143C16070474069C00FC0B27047426952005208C9B277
:206AE000C90711434161704742697F239A43C9B24906490E1143416170478069C00FC0B2F7
:206B00007047826952005208C9B2C9071143816170478269454B1340C9B20A06FE21C905A9
:206B200011401943816170478269474B1340C9B20A04FE21C903114019438161704782699A
:206B4000424B1340C9B20A02FE21C901114019438161704782697F239A43C9B24906490E14
:206B6000114381617047C069C00FC0B27047C26952005208C9B2C9071143C1617047C2698D
:206B80002A4B1340C9B20A06FE21C90511401943C1617047C2692C4B1340C9B20A04FE2192
:206BA000C90311401943C1617047C269274B1340C9B20A02FE21C90111401943C16170479D
:206BC000C2697F239A43C9B24906490E1143C1617047806AC00FC0B27047826A5200520843
:206BE000C9B2C907114381627047826A7F239A43C9B24906490E114381627047006BC00FA8
:206C0000C0B27047026B52005208C9B2C907114301637047026B054B1340C9B20A06FE21BE
:206C2000C90511401943016370470000FFFFFF80026B054B1340C9B20A04FE21C90311406C
:206C40001943016370470000FFFF80FFFF80FFFF026B604B1340C9B20A02FE21C901114097
:206C6000194301637047026B7F239A43C9B24906490E114301637047406BC00FC0B270477E
:206C8000426B52005208C9B2C907114341637047426B7F239A43C9B24906490E114341635C
:206CA0007047016042607047F8B50600002E05D00D00002D02D02888002800D133E00027BE
:206CC0003C0010E06868210089B203224A43801842786868210089B203234B43C15C30002B
:206CE00000F022F8641C2000298880B28842E9D33C0013E06868210089B203224A438018DC
:206D00008078002809D06868210089B203224A4380184178300000F033F8641C20002988AF
:206D200080B28842E6D3F1BD70B506000C0015002900C9B2300000F034F8012801D1002099
:206D40001CE02800C0B28208AB079B0F224D1000C0B2000128181900C9B2890040580028A8
:206D60000BD02100C9B23068D2B21201AA18DBB29B00D2589047012000E00020C0B270BDC2
:206D800080B5C9B28B08154A1900C9B289005158002905D001210068DBB29B00D2589047DA
:206DA00001BD38B5020001242000C9B289080C4B0D00EDB2AD005D59002D09D01068C9B276
:206DC000890059588847012801D1200000E00020C0B232BDFF80FFFFB4A6010000AB0100AA
:206DE000C8AA010078B500231C0045686E6C012296430122E4B2144034436C64009302E068
:206E0000009B5B1C0093009B8B42F9D311004068436C0124A343C9B20A401A43426471BD30
:206E20000160704701210068026880239A43C9B2C901802319401143016070470021006890
:206E4000026880239A43C9B2C90180231940114301607047006801680122914301220A4363
:206E600002607047F3B581B000210A003AE06D462A70019D2D686E46367828277E43AE1922
:206E800037695E4E3E40C0B2000430436E46367828277E43AD1928611000019D2D68060035
:206EA000F6B228277E43AE193769554E3E40E4B224023443C0B22826704328180461100037
:206EC000019C24680500EDB22826754365192D69FF26B543DBB22B43C0B228256843201811
:206EE0000361521C1000C0B2022831DA0C000B0008000D0009E007E001261F003300AB40A9
:206F00003B43AE40064330006D1C2E00F6B2082EADDA029E1700FFB2FF00F6192F00FFB21A
:206F2000F65D002E05D0022E09D003D3032EE3D0E1E7E9E71E000123AB403343E4E701260B
:206F40001F003300AB403B43AE4026433400DBE7F7BD0000F0B500210A0002700A00427077
:206F60000A0082700A00C2700F2202710A0042710A00827101221300C371A24B03814181DE
:206F80000B0018E01D00EDB2ED0045192600F6B2AD192C260F00AF551D00EDB22D014519A6
:206FA0002600F6B27600AD19A981641C2500EDB2082DE7DB5B1C1C00E4B2022C01DA0C0024
:206FC000F4E72C23C2540A0011E00B001400E4B204193C2563551300DBB25B00C318D98755
:206FE0001300DBB25B00C31840241953521C1300DBB2002BE9D0F0BD00000000FFFF00FF4F
:20700000FF00FFFFF3B581B004002000FFF716FF0298008921684A68120C120480B2024362
:207020004A60029840892168CA68120C120480B20243CA6000212AE01300684601700298BC
:207040000D00EDB22D0140191500EDB26D00401986892568684600782827784328181F0058
:20706000FFB2BF00C0198069000C0004B6B230436E46367828277E43AD19DBB29B00EB1890
:207080009861521C1000C0B20828D5DB491C0800C0B2022801DA0022F4E7029801002C314E
:2070A0002000FFF7DFFE0298407821680A68564B1340C0B24004802292021040184308609D
:2070C0000298807821680A68504B1340C0B2C003802212021040184308600298C0782168DC
:2070E0000A684B4B1340C0B20203E020C0011040184308600298007921680A68454B1340F9
:20710000C0B20202F02000011040184308600298407921680A6820239A43C0B24001202371
:207120001840104308600298807921680A680C239A43C0B283000C201840104308600298D4
:20714000C07921680A6802239A43C0B24000022318401043086000252800290023E0029AFA
:207160000B00DBB25B00D218D28F1204029B0E00F6B276009B1940269B5B1A430B002668EC
:20718000DBB29B00F318CA2676009A51029A0B00DBB2D2183C23D25C002A03D002000120A0
:2071A00088401043491C0A00D2B2002AD7D02168C82252008A58FF239A43C0B21043C8229B
:2071C000520088502000FFF72DFE280021680A68114D2A40C0263603C0B280043040104381
:2071E00008602000FFF736FE2000FFF727FE0298007821680A681540C0B2800406402E4393
:207200000E60F7BD60EA0000FFFFFDFFFF7FFFFFFF8FFFFFFFF0FFFFFFFFF3FF016070470B
:207220000160704701607047416082607047000001607047016070470160704738B50400AB
:20724000216062600025A560E0208002E060802040052061802000026061200000F0C8F866
:207260002076E561207E002800D06561200000F001F831BD30B401221300046800210D002B
:20728000DBB25B0002252B402360130004680D00DBB21B0110252B402360130004680D000D
:2072A000DBB25B0120252B402360130004680D00DBB29B0140252B402360130004680D001E
:2072C000DBB2DB0008252B4023600068D2B2910004221140016030BC704730B5010000232A
:2072E0001800012214000D68E4B2E301802423402B600B681B68DB091340DBB2002BF8D011
:207300000B681B685B091340DBB2002B0CD10B681B681B091340DBB2002B05D1096809684E
:207320001140C9B2002900D01000C0B230BDF6B583B001000024200022006A46127C402A2C
:2073400000DB01200293029A002A00D1012000910100C9B2002935D100980068012500681A
:20736000C10928000840C0B2002801D1022029E00098FFF77FFF08232100009802682000C2
:20738000FF2001900E00F6B29619367F019FBE43DBB2019F1F403743C9B251180F77694663
:2073A000097C009A126823002B00DBB2D3181B7F8343C9B208401843EDB2511908770098D0
:2073C000FFF78BFF0100C9B200290ED121000AE00A00D21D009B1B682500D2B29A18127F9B
:2073E000029B5A54491C0829F2D3C0B205B0F0BD3EB5050008220021684600F0EDF800202D
:207400000400FF20694608706B46002200212800FFF78DFFC0B2002804D168460078800768
:2074200000D401242000C0B23EBD0000016000210168CA6E01239A43CA660068016C0A0093
:20744000D207D20F006C704701604260704701604260704701607047016070470160704793
:207460000160704710B4019C016042608360C46010BC704702692F4B1340C9B20A06F02132
:207480000905114019430161704702692A4B1340C9B20A04F0210903114019430161704779
:2074A0000269264B1340C9B20A02F0210901114019430161704702690F239A43C9B2090730
:2074C000090F11430161704742691C4B1340C9B20A02F0210901114019434161704742696F
:2074E0000F239A43C9B20907090F11434161704738B5050029606A60002408E01048210063
:2075000089B2425C0C21280000F006F8641C200080B20628F2D331BD80B51300DBB2062B96
:2075200006DAC9B24068074BD2B292009A58904701BD0000FFFFFFF0FFFFF0FFFFF0FFFF92
:20754000A8AC010068AC01000160002101714171282281543822815470470000016001684C
:207560000A6980235B0013430B6101680A6980239B0013430B61012101680A690223134383
:207580000B6100BF00BF00BF002100680161704701600168CA6A80231B021343CB6200BFA0
:2075A00000BF00BF00BF0A4B1340CB620168CA6A8023DB011343CB6200BF00BF00BF00BF1E
:2075C000044B1340CB6200210068016070470000FF7FFFFFFFBFFFFF10B504000800110021
:2075E0000200200000F02AF8200010BD70B4103A03D378C9103A78C0FBD2530701D318C987
:2076000018C001D508C908C0D20704D30B880380891C801C002A01D50B78037070BC704743
:207620008B0701D18307E1D0124205D00B78491C0370401C521EF9D1704700001206130AA5
:207640001A43130C1A4300BF094205D0830705D00270401C491EF9D1704700001300103901
:2076600006D330B41400150010393CC0FCD230BC490700D30CC000D504C0890002D30280BD
:20768000801C002900D502707047000000B5002001000CE04C4A0B00DBB2D0544B4A0B0073
:2076A000DBB2D0544A4A0B00DBB2D054491C0A00D2B2082AEEDB00BD00B50100C9B20829BC
:2076C00003DA0121414AC0B2115400BD00B50100C9B2082903DA01213D4AC0B2115400BD10
:2076E00000B50100002210000B00DBB2082B05DA364B0800C0B2185CC9B25A54C0B200BD31
:2077000000B50100C9B2082903DA2F49C0B2085C00E0002000BD70B50024250022E02A4E37
:207720002800C0B2305C012803D12800C0B2FFF7CDFF20002900C9B2705412E0C0B20028B6
:207740000FD124482900C9B24900415A0029E6D02900C9B24900415A491E2A00D2B2520087
:2077600081526D1C2800C0B208282BDA2800C0B2FEF773FA0100C9B20129DFD112492A0007
:20778000D2B28A5C012AD9D012482A00D2B25200825A521C2B00DBB25B00C2522A00D2B232
:2077A0005200825A142ADCDB01222B00DBB2CA5414212A00D2B2520081522800C0B2FFF715
:2077C0007BFFCEE770BD0000685000207050002078500020805000200021016041600A0090
:2077E0000272417270470022026041600121017242727047407A7047FEB505000E0014003B
:20780000082100226F463800FFF718FF2000C0B2782805D06F48295A6F482818FFF7E3FF13
:207820007920285C002814D02000C0B211280FD02000C0B212280BD02000C0B2312807D00C
:207840002000C0B27E2803D02000C0B27F2800D10AE068467F2101704670847003226946EC
:2078600028001830FDF761F8F7BD10B50022130000E0521C13009BB24468A3420AD2836897
:207880001400A4B2E4001B5D0C00E4B2A342F0D1012000E0002010BD70B505000C00210095
:2078A00028001830FDF711FA0120687000263000A870300078216854002000218422520133
:2078C000AA1803C2083AA08D44496852E08D44496852208E3F49685242482818FFF77CFF8C
:2078E00041482818FFF778FF3B482818FFF774FF3000300004E031002A187B23D154401C50
:20790000802149018842F6D370BD7CB50400002528006946888028002800280020001830A3
:20792000FDF71FFA01A8009080235B0122007B322100793120001830FDF796F940B2002863
:2079400039D17B20265C3100C9B22000FFF78DFF00282AD02B0000E05B1C606883422AD285
:20796000A068D900405C3100C9B28842F4D1A068D90040188078002806D07C20205CC0B296
:20798000C0097821605402E028007821605418007A2160546846828821007B312000A66860
:2079A000DB00F3185B68984705E011223100C9B22000FFF721FF08482018FFF71BFF012884
:2079C00006D101206070A57003482018FFF704FF73BD00008C100000A81000008810000032
:2079E0008A100000901000009C10000010B50400A26863681000401C834206D3206881549C
:207A0000521CA260E068401CE060A068616888420DD1A2682168206900F0CCFAA1688842F4
:207A200003D00020C043E06001E00020A06010BDF7B582B005001F0003980124012603E076
:207A40000499FBF71EF9761C04998842F8D2BE4200D23E0001950A9D0B98C0071BD4002DEA
:207A600019D00B98800705D5002F03D130206946087002E0202069460870002D0BD0AE425E
:207A800009D26D1E684601780198FFF7AFFF0198C0680028F1D50198C068002839D402E095
:207AA0007F1E04984443022FFAD203982100FBF7E8F804998842F4D203982100FBF7E1F8C7
:207AC0000100039A08006043101A03901248415C0198FFF78BFF0198C068002807D42000AC
:207AE0000499FBF7CEF80400002CE5D1FFE70B98C0070ED5002D0CD0002D0AD0AE4208D23E
:207B00006D1E20210198FFF771FF0198C0680028F2D505B0F0BD000080AC0100F1B584B081
:207B20000E001D00002E01D5704200E030000124039203E00399FBF7A1F8641C03998842AA
:207B4000F8DA02950298844200D2029C0A9D0B9F002D04D0002E01D4780700D56D1EB807F9
:207B600002D50298002810D0F8070ED4002D0CD0002D0AD0AC4208D26D1E20210498FFF775
:207B800035FF0498C0680028F2D50498C068002834D4002E06D5704206002D210498FFF769
:207BA00025FF05E0780703D52B210498FFF71EFF0498C068002821D4B807800F022811D12F
:207BC000029800280ED1002D0CD0002D0AD0AC4208D26D1E30210498FFF708FF0498C068F3
:207BE0000028F2D50498C068002807D401970095029B039A31000498FFF71AFF05B0F0BD2A
:207C0000F1B598B00C00160007A8029040200390002704971898069005972178641C08005B
:207C2000C0B2002808D00800C0B2252800D0C7E038000122110000E0CAE02378DBB2232B28
:207C400013D02B2B0CD02D2B02D0302B03D011E01043641C0FE0030002201843641C0AE01A
:207C6000030004201843641C05E0030008201843641C00E039000029DFD13A0005E0641C86
:207C80000A235A43C9B25218303A21780B00DBB2303B0A2BF3D33B002178C9B22E290DD1B0
:207CA000641C05E0641C0A256B43C9B25B18303B21780D00EDB2303D0A2DF3D3217801E080
:207CC000641C21780D00EDB26C2DF9D00D00EDB2682DF5D0C9B225296BD0582934D0632962
:207CE0000AD0642914D0702952D073293AD075291CD0782928D061E030683060306801684B
:207D00003068001D3060C9B202A8FFF76FFE55E0316831603168096835682D1D3560019020
:207D200000920A2202A8FFF7F9FE47E0316831603168096835682D1D3560019000920A22C8
:207D400002A8FFF775FE39E0316831603168096835682D1D356001900092102202A8FFF752
:207D600067FE2BE030683060306805683068001D306029786D1C0800C0B2002807D0C9B203
:207D800002A8FFF733FE05980028F2D5FFE715E030683060306801683068001D306000201D
:207DA0000190082000900823102202A8FFF740FE04E0252102A8FFF719FEFFE7641C03E015
:207DC000C9B202A8FFF712FE0598002800D424E7059801280BDB0498002804D0049A07A942
:207DE000189800F0E7F80598049940180590059819B0F0BD0CB480B502AA00926A46FFF7F1
:207E0000FFFE019904B0084710B5494C0320206160614848A0614849E1618021C9002162B8
:207E20000021A1626162E1622066444860661020A0662167E166616741A1E01D00F0D8F8D4
:207E40004049200000F0D4F82020A07110BDF8B584B004000D00160000200190E76820690E
:207E6000874202D2C01B401E03E0A168C91B0818401EA168C91B884201D3A068C01BB0427E
:207E800001D2009000E000966068C0190099039129000290039A0298FFF7C2FB0298019863
:207EA00000994018019000982D180098361A00983F18A068874200D10027E760002ECED1AF
:207EC000019805B0F0BDF8B504000F001500E668A068801B0090009885420AD260688019B5
:207EE0002A00390007003800FFF79AFB7019E06010E0009A6068861939003000FFF790FBB1
:207F000000982D1A66682A00009839183000FFF787FBE560F1BD00B50169C2688A4204D31A
:207F20008068401E801A401801E0881A401E00BD905000209CAC01003851002038550020CC
:207F400052545400B0AC0100F8B516000F002549182250430818050018356869002803D07F
:207F600002281DD00ED322E02800FFF7D4FFB04201D2002405E03400320039002800FFF78B
:207F8000A2FF15E02800FFF7C6FFB04201D2040000E03400220039002800FFF794FF07E098
:207FA000320039002800FFF752FF040000E000242000F2BD70B504000D00160009480078FB
:207FC000002801D1FFF720FF320029002000EFF31084012383F31088FFF7B6FF84F31088B5
:207FE00070BD00009050002080B5FFF70DFF01BD31B48B0707D00B780370002B20D0401CA4
:20800000491C8B07F7D1164CE501830722D104C9131B93432B4205D104C004C9131B934333
:208020002B42F9D0FF231A42027009D0120A1A42427005D0120A1A42827001D0120AC270B9
:2080400031BC70470270120A4270120A8270120AC270001D04C9131B93432B42F2D0E1E7FB
:2080600001010101002202604160012101724272704770B504000E0015003448215A344818
:208080002018FFF7EFFF7820205C012806D02A00310092B220001830FCF747FC70BDFEB594
:2080A00005000E001400082100226F463800FFF7C5FA2000C0B2782805D02448295A24484A
:2080C0002818FFF7CFFF7920285C002814D02000C0B211280FD02000C0B212280BD0200002
:2080E000C0B2312807D02000C0B27E2803D02000C0B27F2800D10AE068467F21017046706A
:2081000084700322694628001830FCF70EFCF7BD7CB56C46AE4D2E682660DBB2042B14D3D9
:20812000069C0B0004210D00258014008078DBB2834204D100222000FFF780FA05E0684643
:208140000A0001002000FFF76BFA73BD8C100000A810000001207047F8B584B006000C004A
:208160001500002008210020009002AF009A3800FFF764FA00206946C8800020002028009B
:20818000B1687A22B25CD2008918497880B289B2884205D2132227213000FFF780FF14E1C3
:2081A0007078012805D1222227213000FFF777FF0BE184204001301803C8FA22D2000023BB
:2081C000994208DC01DB904205D2372227213000FFF765FFF9E0200041784906490E6A4628
:2081E000117167216A4611726946097902AA517069460979C90776D50027380075490870C3
:208200003C0000E0641C2000C0B2042833DA724D684600792100C9B20901695C8842F1D11A
:208220002000C0B20001281880782100C9B209016918497888421ED28420400130180CC8D0
:2082400008382000C0B200012818083003C8121A8B41624800218B4208DC01DB824205D21D
:20826000362227213000FFF71AFFAEE02000C0B2000128184770E4B2042C05DB31222721C6
:208280003000FFF70CFFA0E0062301A8801C0090DBB202A8821C684601793000FFF738FFD5
:2082A0006846C088002818D06846C288921C92B202A93000FFF7DDFE6846007945490870F5
:2082C0006846C088464908806846C28802A8811C444C2000FFF7A4F977E0312227213000ED
:2082E000FFF7DDFE71E03B4C694609792278521C914205D0242227213000FFF7D0FE64E02E
:20830000AD1EADB20095831C3548028835492078FFF720FFC0B2012821D1022202A9300041
:20832000FFF7A7FE00200100217069460979491EB17001000A00D2B2042A46DA264A6B4639
:208340001B790C00E4B22401145DA34205D103000C00E4B2240112195370491CEAE7352251
:2083600027213000FFF79BFE00232AE01A4A20781900C9B20901515C884221D11800C0B23C
:20838000000110184078401C1900C9B20901511848701800C0B20001101880781900C9B2A2
:2083A00009015118497888420AD284204001301803C81D00EDB22D015219083203C2083A55
:2083C0005B1C1800C0B20428D0DB05B0F0BD0000BCAC0100A8550020000000201027000086
:2083E000A455002048550020002202604160012101724272704770B504000E0015002548C9
:20840000215A25482018FFF7EFFF7820205C012806D02A00310092B220001830FCF785FACC
:2084200070BDFEB505000E001400082100226F463800FFF703F92000C0B2782805D01548A7
:20844000295A15482818FFF7CFFF7920285C002814D02000C0B211280FD02000C0B2122899
:208460000BD02000C0B2312807D02000C0B27E2803D02000C0B27F2800D10AE068467F2112
:208480000170467084700322694628001830FCF74CFAF7BD8C100000A810000000B500285F
:2084A000FFD000BD00B50028FFD000BD00B50028FFD000BD00B50028FFD000BD00B5002818
:2084C000FFD000BD00B50028FFD000BD00B50028FFD000BD00B50028FFD000BD00B50028F8
:2084E000FFD000BDF3B5FFB086B006001400002503952800280028002800032069460870A2
:208500008020800001902A0005AF01993800FFF795F82800694608812000B1687A22B25C34
:20852000D2008918497880B289B2884205D2132231213000FFF775FFE5E0869841784906ED
:20854000490E6A46517081780902C2788918241F6A4694806A469288002A01D0001D0390F8
:208560002C0000E0641C20006A461278C0B2904229D266482200D2B214235A43825A0B00C7
:208580009BB29A42EED171782200D2B214235A4382189278914222D12100C9B214225143C0
:2085A0004118C97800290ED02100C9B2142251434018C078B178884205D033223121300085
:2085C000FFF72FFF9FE0200069460978C0B288420BD3312231213000FFF723FF93E02222EA
:2085E00031213000FFF71DFF8DE08020800004902A0005AF04993800FFF720F8684640789F
:20860000012804D066D303284CD027D362E03F4D02A8009080239B0005AA6846818803989C
:2086200084462700FFB214204743E81987686046B8470120E4B214214C4329190871684661
:20864000008904284CDB6846007D712848D16846028905A93000FFF7CEFE54E02B482100C0
:20866000C9B21422514340180079002819D002A8009080239B0005AA6846818803980190C9
:20868000224884462700FFB2142047436046C019C7680198B8471D48E4B214214C430019F2
:2086A0000571CCE7194D2000C0B2142148432818007900280DD002A8009080239B0005AAF4
:2086C000684681880398E4B214277C432C192469A047B4E7122231213000FFF7A2FE12E026
:2086E00068460089032809D105A801787F2905D1827831213000FFF794FE04E0242231211A
:208700003000FFF78EFE7FB008B0F0BD8C010020002202604160012101724272704770B51C
:2087200004000E001500AE48215AAE482018FFF7EFFF7820205C012806D02A00310092B2DD
:2087400020001830FCF7F1F870BDFEB505000E001400082100226F463800FEF76FFF200013
:20876000C0B2782805D09E48295A9E482818FFF7CFFF7920285C002814D02000C0B21128CB
:208780000FD02000C0B212280BD02000C0B2312807D02000C0B27E2803D02000C0B27F284D
:2087A00000D10AE068467F210170467084700322694628001830FCF7B8F8F7BDF6B5FFB0A0
:2087C00082B00500002000200026002000200027802189000020009001AC009A2000FEF75F
:2087E0002DFF82A80088A9687A22AA5CD2008918497889B2884205D2132222212800FFF742
:20880000A4FFEAE082A80088401EC00705D5132222212800FFF799FFDFE082A80088400853
:2088200080B2002805D1132222212800FFF78DFFD3E0622001A9320092B28854761C012002
:208840006946088079E0300080B22969220092B214235343C91889894018801C6249884205
:2088600000DB9FE02869210089B214224A4380188078052800D19BE068782969220092B20D
:2088800014235343C918C978884200D290E02869210089B214224A4380188289D2B2286975
:2088A000210089B214234B43C018816828002F69BC462700BFB214237B436746FB181B6943
:2088C0009847012701A881996A461288895C320092B28154761C81996A46128889184978FC
:2088E000320092B28154761C684646802869210089B214224A43801882892869210089B2E7
:2089000014234B43C018816801A86B465B88C6183000FEF785FE684640882969A4B214227A
:2089200062438918898946183800C0B2002845D068460088801C694608806846008882A930
:20894000098888423AD2819869460988405C000281996A461288891849780843002427005D
:2089600000E0641C2100AA8A89B29142DCD22969220092B214235343C95A020092B2914285
:20898000EFD1A8782969220092B214235343C9180979884200D156E7332222212800FFF741
:2089A000D4FE1AE0142222212800FFF7CEFE14E0222222212800FFF7C8FE0EE0FFB2002F5B
:2089C00006D0320092B201A92800FFF7A8FE04E0312222212800FFF7B8FE7FB004B0F0BDFF
:2089E0008C100000A810000001020000002202604160012101724272704770B504000E00C4
:208A000015009548215A95482018FFF7EFFF7820205C012806D02A00310092B220001830D6
:208A2000FBF783FF70BDFEB505000E001400082100226F463800FEF701FE2000C0B278285D
:208A400005D08548295A85482818FFF7CFFF7920285C002814D02000C0B211280FD020002D
:208A6000C0B212280BD02000C0B2312807D02000C0B27E2803D02000C0B27F2800D10AE0AE
:208A800068467F210170467084700322694628001830FBF74AFFF7BD70477047704770475E
:208AA000F6B5FFB082B004000D00002630003000300002206946087080218900320001AF0E
:208AC0003800FEF7BBFD82A80088A1687A22A25CD2008918497889B2884205D213222F21C7
:208AE0002000FFF7A0FFB3E06078012805D122222F212000FFF797FFAAE0280041780902A1
:208B000082788918C2786B465A70350000E06D1C2A006B461B78D2B29A4220D2504A2B00E2
:208B2000DBB214277B43D35A0F00BFB2BB42EED12900C9B2142359435118897800290ED05E
:208B40002900C9B21423594351188978A278914205D033222F212000FFF765FF78E02900D2
:208B60006A461278C9B2914205D331222F212000FFF759FF6CE001A96F220A7042784A700F
:208B800082788A70C278CA7069464978002902D003291BD057E032482900C9B214225143CC
:208BA0004118CE722900C9B2142251434118096900290AD0EDB214214D43401900698047F3
:208BC000042201A92000FFF718FF41E0244E82A909882A00D2B214235A43B218127A121D42
:208BE000914205DA22222F212000FFF71CFF2FE001212A00D2B214235A43B218D172290015
:208C0000C9B21422514371180A7A011D2800C0B214235843301847683800FEF701FD28002E
:208C2000C0B2142148433018C06800280AD0EDB2142045437019C0688047042201A92000CD
:208C4000FFF7DBFE04E031222F212000FFF7EBFE7FB004B0F0BD00008C100000A8100000DB
:208C6000640100200100050000000000000000000000000003000500000000000000000061
:208C8000000000001100050000000000000000000000000063000500000000000000000056
:208CA000000000000100000031070000DF070000B107000050320020000200005034002095
:208CC00008080000000000004D65010031A301003200F401881300001A620400500000006A
:208CE000000000001B63040050000000000000001603F00050000000000000001703F0003F
:208D000050000000000000008873C00050000000000000000100C1005000000000000000E6
:208D20000101C10050000000000000000121C10050000000000000000127C10050000000B4
:208D4000000000000128C10050000000000000000129C10050000000000000000131C100AB
:208D600050000000000000000041C10050000000000000000151C1005000000000000000EE
:208D80000063C10050000000000000000069C10050000000000000000181C1005000000052
:208DA000000000000136C20050000000000000000064C10050000000000000000067C100CD
:208DC000500000000000000092F000005055002002000000998A01009B8A010020F00000A0
:208DE00052550020020000009D8A01009F8A010000FF0301000000009D840100A584010009
:208E0000AD84010001FF030100000000B5840100BD840100C584010002FF03010000000051
:208E2000CD840100D5840100DD84010086F106010000000060550020010000003BA40100F0
:208E400087F1060100000000615500200800000041A4010080F10601000000006955002079
:208E60000800000031A4010093F106010000000071550020040000004BA4010095F1060122
:208E800000000000755500201000000055A4010091F1060100000000855500201800000043
:208EA0005FA4010088490870704730B5010089B2142927DA0021854A0B000400A4B20C25C9
:208EC00065435419237103009BB20C245C4313191B1D1C78102525431D7003009BB20C2428
:208EE0005C4313191B1D1C78402525431D7003009BB20C245C431319D98080B20C234343F6
:208F0000D018017230BD30B5010000221000100010000DE06D4B1400A4B20C2565435B1975
:208F20001B795B065B0EDBB20B4200D0401C521C13009BB2142BEDDB80B230BDF2B5010031
:208F4000002318001800180023E01E00B6B20C277743EE59360C0700BFB2CE55401C1E0092
:208F6000B6B20C277743EE59360A0700BFB2CE55401C1E00B6B20C277743ED590600B6B2F7
:208F80008D55401C6406640E0500ADB24C55401C5B1C1C00A4B2142C11DA4C4D1C00A4B237
:208FA0000C266643AC1924792600F6B21642EFD06E4636880700BFB23F1DBE42C5DA80B278
:208FC000F2BDF0B50200002318001800180023E01E00B6B20C277743EE59360C0700BFB259
:208FE000D655401C1E00B6B20C277743EE59360A0700BFB2D655401C1E00B6B20C2777437E
:20900000ED590600B6B29555401C6406640E0500ADB25455401C5B1C1C00A4B2142C0DDA01
:209020002A4D1C00A4B20C266643AC1924790E00B6B20700BFB23F1DBE42C9DA80B2F0BD3E
:2090400010B5002421002249401A04D09D3817D02F382CD035E00EE01C48210089B20C225D
:209060004A43805880214903884203D2200080B2FFF71BFF641C200080B21428ECDB20E0C8
:2090800010E01248210089B20C224A438058114940188021C903884203D2200080B2FFF791
:2090A00004FF641C200080B21428EADB09E004E0200080B2FFF7F9FE641C200080B21428C0
:2090C000F6DB10BD00000000A75500207400002033FFFF000000C0FF00220260416001210B
:2090E00001724272704770B504000E0015002548215A25482018FFF7EFFF7820205C012898
:2091000006D02A00310092B220001830FBF70DFC70BDFEB505000E001400082100226F4670
:209120003800FEF78BFA2000C0B2782805D01548295A15482818FFF7CFFF7920285C0028F0
:2091400014D02000C0B211280FD02000C0B212280BD02000C0B2312807D02000C0B27E28E0
:2091600003D02000C0B27F2800D10AE068467F210170467084700322694628001830FBF789
:20918000D4FBF7BD8C100000A81000008020704710B5010000200200012200E0521C130035
:2091A000DBB2052B08DA04239B1ADB000C00DC40002CF3D00520801AC0B210BDF8B584B063
:2091C000040013000022100015001500160016001600160016006778012F05D12222342130
:2091E0002000FFF796FF8EE09C46A7687A23E35CDB00FB185B786746BFB29BB29F4205D2A5
:20920000132234212000FFF784FF7CE00191019989780907090F6B46197001998978C9B22A
:2092200009096B4659706946097800290BD069460978052907D269464978002903D069461C
:209240004978052905D3312234212000FFF761FF59E0110007E00002019B0F00FFB2DB19A6
:20926000DB78C018491C0B006F463F78DBB2BB42F1D30AE02902019B6D462D781700FFB2C8
:20928000ED195B19DB78CD18521C11006B465B78C9B29942EED3002D05D122223421200046
:2092A000FFF737FF2FE000F087F8280000F087F8012000F08AF8FFF769FF05002800FFF759
:2092C00067FF02A9742233009BB2CA54761C320003011600B6B28B55521C012308E0C61AC9
:2092E000F7002E00FE401700BFB2CE55521C5B1C06001F00F6B2FFB2BE42F0D292B202A94C
:209300002000FFF7F0FE05B0F0BD0000002202604160012101724272704770B504000E008B
:2093200015007948215A79482018FFF7EFFF7820205C012806D02A00310092B220001830E5
:20934000FBF7F3FA70BDFEB505000E001400082100226F463800FEF771F92000C0B278285E
:2093600005D06948295A69482818FFF7CFFF7920285C002814D02000C0B211280FD020003C
:20938000C0B212280BD02000C0B2312807D02000C0B27E2803D02000C0B27F2800D10AE085
:2093A00068467F210170467084700322694628001830FBF7BAFAF7BD55490860704755494B
:2093C000086070475348006870475349087000200100524A11700100514A11705149086043
:2093E00070474D48007870474E4800687047F0B5FFB082B004000E001500002210006946AF
:2094000008808021890001AF3800FEF717F96078012805D1222236212000FFF794FF6EE044
:2094200028000100A2687A23E35CDB00D218527889B292B2914205D2132236212000FFF7C3
:2094400082FF5CE034490978012902D002294BD050E0334972780A70304B0A781D78AA4281
:209460000BD00A781D786D1CEDB2AA4205D0732236212000FFF767FF41E001AA76256F468D
:209480003F88D5556D462D886D1C77782E00B6B297556D1C2A000D781E78B54205D192B29A
:2094A00001A92000FFF739FF29E01E4D194E3768BC462F680600B6B2BE19B61E6746B742E2
:2094C00005D2712236212000FFF73DFF17E02E6880B2801E301828600878187092B201A956
:2094E0002000FFF71AFF0AE0312236212000FFF72AFF04E0242236212000FFF724FF7FB081
:2095000002B0F0BD000000008C100000A81000005455002058550020AA550020AC550020C2
:20952000AB5500205C550020002202604160012101724272704770B504000E001500784809
:20954000215A78482018FFF7EFFF7820205C012806D02A00310092B220001830FBF7E5F9CA
:2095600070BDFEB505000E001400082100226F463800FEF763F82000C0B2782805D06848A5
:20958000295A68482818FFF7CFFF7920285C002814D02000C0B211280FD02000C0B21228F5
:2095A0000BD02000C0B2312807D02000C0B27E2803D02000C0B27F2800D10AE068467F21C1
:2095C0000170467084700322694628001830FBF7ACF9F7BDF2B582B00400150008210026A0
:2095E00032006F463800FEF729F83000A0687A21615CC90040184078ADB280B2854205D29E
